:020000022000DC
:1060000000000420990B06009F94020091F002000A
:106010009F9402009F9402009F94020000000000E1
:106020000000000000000000000000009F9402003B
:106030009F940200000000009F940200CDFC02002B
:1060400051E302009F940200F10F0300B1A002008F
:10605000C1A002009F940200150503009F94020056
:106060009F940200A1FA020091FA02006507030062
:106070009F9402009F9402009F9402009F9402004C
:106080009F940200750703009F9402009F940200F2
:106090009F9402009F940200918A05009F94020041
:1060A0009F9402009F9402009F9402009F9402001C
:1060B0009F9402009F940200000000000000000076
:1060C0009F9402009F9402009F9402002501030008
:1060D000850703009F9402009F940200C1620300A1
:1060E00001100300BDA202009F9402009903030067
:0860F000000000009F94020073
:1070000040F8044B40F8045B40F8046B40F8047B04
:1070100040F8048B40F8049B40F804AB40F804BBF4
:1070200040F804CB40F804DB6846704781F000412B
:1070300002E000BF83F0004330B54FEA41044FEA5D
:10704000430594EA050F08BF90EA020F1FBF54EAF8
:10705000000C55EA020C7FEA645C7FEA655C00F094
:10706000E2804FEA5454D4EB5555B8BF6D420CDD65
:107070002C4480EA020281EA030382EA000083EAE8
:10708000010180EA020281EA0303362D88BF30BD88
:1070900011F0004F4FEA01314FF4801C4CEA1131DE
:1070A00002D0404261EB410113F0004F4FEA03333D
:1070B0004CEA133302D0524263EB430394EA050FC8
:1070C00000F0A780A4F10104D5F1200E0DDB02FA37
:1070D0000EFC22FA05F2801841F1000103FA0EF2CB
:1070E000801843FA05F359410EE0A5F120050EF191
:1070F000200E012A03FA0EFC28BF4CF0020C43FAC2
:1071000005F3C01851EBE37101F0004507D54FF0CE
:10711000000EDCF1000C7EEB00006EEB0101B1F51E
:10712000801F1BD3B1F5001F0CD349085FEA300064
:107130004FEA3C0C04F101044FEA445212F5800F6F
:1071400080F09A80BCF1004F08BF5FEA500C50F10C
:10715000000041EB045141EA050130BD5FEA4C0CEF
:10716000404141EB0101013C28BFB1F5801FE9D24C
:1071700091F0000F04BF01460020B1FA81F308BF6F
:107180002033A3F10B03B3F120020CDA0C3208DD3B
:1071900002F1140CC2F10C0201FA0CF021FA02F116
:1071A0000CE002F11402D8BFC2F1200C01FA02F186
:1071B00020FA0CFCDCBF41EA0C019040E41AA2BFAB
:1071C00001EB0451294330BD6FEA04041F3C1CDA73
:1071D0000C340EDC04F11404C4F1200220FA04F093
:1071E00001FA02F340EA030021FA04F345EA03013D
:1071F00030BDC4F10C04C4F1200220FA02F001FAFF
:1072000004F340EA0300294630BD21FA04F0294680
:1072100030BD94F0000F83F4801306BF81F4801119
:107220000134013D4EE77FEA645C18BF7FEA655C8C
:1072300029D094EA050F08BF90EA020F05D054EA5E
:10724000000C04BF1946104630BD91EA030F1EBF63
:107250000021002030BD5FEA545C05D14000494167
:1072600028BF41F0004130BD14F580043CBF01F55A
:10727000801130BD01F0004545F0FE4141F4700140
:107280004FF0000030BD7FEA645C1ABF194610461B
:107290007FEA655C1CBF0B46024650EA013406BF1C
:1072A00052EA033591EA030F41F4002130BD00BFDB
:1072B00090F0000F04BF0021704730B54FF4806498
:1072C00004F132044FF000054FF0000150E700BF19
:1072D00090F0000F04BF0021704730B54FF4806478
:1072E00004F1320410F0004548BF40424FF0000165
:1072F0003EE700BF42004FEAE2014FEA31014FEAA8
:1073000002701FBF12F07F4393F07F4F81F06051F6
:10731000704732F07F4208BF704793F07F4F04BF41
:1073200041F40021704730B54FF4607401F000451E
:1073300021F000411CE700BF50EA010208BF70477E
:1073400030B54FF000050AE050EA010208BF70476F
:1073500030B511F0004502D5404261EB41014FF4D8
:10736000806404F132045FEA915C3FF4D8AE4FF0E0
:1073700003025FEADC0C18BF03325FEADC0C18BFC3
:10738000033202EBDC02C2F1200300FA03FC20FA14
:1073900002F001FA03FE40EA0E0021FA02F1144461
:1073A000BDE600BF4FEA4102B2F1E04324BFB3F5AE
:1073B000001CDCF1FE5C0DD901F0004C4FEAC0026C
:1073C0004CEA5070B2F1004F40EB830008BF20F050
:1073D0000100704711F0804F21D113F13872BCBF0A
:1073E00001F00040704741F480114FEA5252C2F15F
:1073F0001802C2F1200C10FA0CF320FA02F018BFA8
:1074000040F001004FEAC1234FEAD32303FA0CFCFA
:1074100040EA0C0023FA02F34FEA4303CCE77FEA89
:10742000625307D150EA01331EBF4FF0FE4040F4D3
:107430004000704701F0004040F0FE4040F4000082
:10744000704700BF024B1A6912681A61704700BF8B
:10745000D04E0120C460056146618761C0F81C8080
:10746000C0F82090C0F824A0C0F828B0C0F82CD0F4
:1074700080ED0C8B80ED0E9B80ED10ABC0F808E02A
:107480000AF094B82DE9F0412A4C00250326D4F8DF
:10749000EC700021013143189A0803F00303BA5C31
:1074A0005B0042FA03F303F00303022BF2D0D4F89B
:1074B000F83009018A0803EB001089B300EB82025F
:1074C0000368190729D1D4F8F810994225D8D4F8BF
:1074D000FC709F4221D95B1A48BF0F331B11D4F8AF
:1074E000ECE04FEA930C03F003011EF80C80490016
:1074F00048FA01F707F00307012F0ED106FA01F150
:1075000041EA080104EB85083F2D0EF80C109ABFE4
:107510000135C8F80831C4F8047104309042CFD165
:107520002DB1013D04EB8503D3F80801AFE7BDE8B9
:10753000F08100BFD04E01202DE9F0473B4CD4E94B
:107540003E120023C0E90233C0E90433521AC0E9F5
:1075500000231D4683619C461F4619461A469A46DB
:1075600099469E46D4F8EC6016F80A304FEA49096D
:1075700043FA09F303F00303012B4DD0022B47D04C
:10758000002B3ED0D4F8F0600132B2EB860F4FEA08
:1075900086080FD0D4F8EC604FEA920A02F0030993
:1075A00016F80A304FEA4906334113F0030301D0BD
:1075B000012BD7D1012911D0022902BF466901361A
:1075C000466186698E4238BF816190450FD0012B9C
:1075D00026D04FEA920A02F00309C3E70669013692
:1075E000066186698E4238BF81619045EFD177454B
:1075F00000D9C7602D014FEA0C13C0E90153BDE863
:10760000F0870CF1010CC0F808C001371946B9E742
:10761000013545600131B5E7013545601946B1E7EF
:10762000BE4501D2C760BE460027D2E7D04E01203A
:1076300050F8310010B1043818BF01207047000025
:10764000054B5B695A68824204D8801A043053F8AB
:10765000200070471B68F5E7D04E0120014441F23D
:107660000553884204D3D8B2012838BF012070479F
:1076700010F8012B03EB43135340F2E708B5FFF773
:10768000DFFF023008BD08B5FFF7DAFF43780B6073
:10769000023008BD43688B422CBF591A002141605B
:1076A000704700002DE9F74F89469DF830101746C6
:1076B0000D9A11F0DF0F0646A2EB07023DD03029EC
:1076C00025490CA813BF804688464FF0100A4FF09A
:1076D000010A13F0800535D002EBD2746510A2EBDD
:1076E0006404002D35DDAB46DA45524673683068D8
:1076F000A8BF5A46414601929847019AABEB020B4C
:10770000BBF1000FF0DC2FB1736830683A46494690
:1077100098473D44002C0CDD2544A2455746A8BFA0
:107720002746736830683A464146E41B9847002C68
:10773000F3DC284603B0BDE8F08FDFF820804FF07F
:10774000100AC6E713F0010401D11546C9E7144633
:10775000D9E70025D7E700BF2D1407001C14070048
:107760002DE9F04389B006460020119D9DF8488020
:10777000139F8DF80F000AB381421ADA2D228DF87B
:107780000F204942109A08ACA2F10A000DF110092D
:10779000B1FBF3FC03FB1C12092A8CBF1218303218
:1077A00004F8012D4C458E4661460ED07345EFD945
:1077B0000BE0A80727D52B228DF80F200029E1D157
:1077C00030238DF81F300DF11F0415F040099DF88E
:1077D0000F301CD023B30122CDE900822B460DF1DE
:1077E0000F013046FFF75EFF013F814608AACDE951
:1077F00000872B46121B21463046FFF753FF4844B3
:1078000009B0BDE8F0836A07D8D52022D4E7002B61
:10781000ECD004AA9442E9D904F8013C013CE5E724
:107820009946E3E790F9001003780029024601DB4E
:107830001846704703F07F004023184206D112F823
:10784000013F03F0C001802904D0704720EA030003
:107850005B08F2E703F03F0343EA8010EFE7431CC5
:1078600018460133027802F0C002802AF8D070472F
:1078700001440346002099421A4600D87047127806
:1078800002F0C002802A03F1010318BF0130F2E7C1
:107890007F289DBF024B185CC0F34000002070475A
:1078A000149A06007F289DBF024B185CC0F3C000ED
:1078B00000207047149A06007F289DBF024B185C79
:1078C000C0F3800000207047149A06007F289DBFF7
:1078D000024B185CC0F3001000207047149A060099
:1078E0007F289DBF024B185CC0F3401000207047FA
:1078F000149A060008B50246FFF7E8FF00B12032EF
:10790000104608BD08B50246FFF7EAFF00B1203A6D
:10791000104608BD10B501440246E52400209142FE
:1079200003D8B0FA80F0400915E012F8013B20B10D
:107930001B0611D5431ED8B2F1E7BF2B09D9F72B8F
:1079400009D8DB0803F0060344FA03F303F003004D
:10795000E5E71B06E3D510BD0020FCE702398142B4
:107960000B4603D20233181A401070471A880239A6
:10797000002AF4D0F6E7B2EB131F70B54FEA1314E8
:1079800015D9121B03F00F0301EB440115460E46F7
:10799000012D31F8024B18BF3468DC40A4B2013D20
:1079A00020F8024BF3D104B9013A104670BD002211
:1079B000FBE7F0B5059F0024D21B2646A74210D155
:1079C00000EB470C01EB47010024A24214D10CEB61
:1079D00042031EB101212CF812100233181A401074
:1079E000F0BD31F8145033F814C06544354420F824
:1079F00014502E0C0134E1E731F8145035442CF8C2
:107A000014502E0C0134E0E7F0B4049F0025D21B83
:107A10002C46AF420BD100EB470601EB4705002394
:107A20009A420FD106EB4201F0BCFFF797BF31F845
:107A30001560344433F81560A41B20F81540241455
:107A40000135E6E735F813100C4426F813402414EA
:107A50000133E5E710B500EB410002EB410209B943
:107A6000084610BD30F8023D32F8024D1B1B002BBA
:107A700002DB04D10139F2E74FF0FF30F1E70120DA
:107A8000EFE710B5D0E90121034601EB42020020E7
:107A9000914204D31B78DB0748BF404210BD32F847
:107AA000024D44EA0040F3E72DE9F04371B19F181D
:107AB000D0E901940025A4F102084FF0010EAC4674
:107AC0001A44B9F1000F03D1BDE8F0831F46EFE778
:107AD00038F8024F0CF1100C44EA0545BCF1070FD1
:107AE00002DC09F1FF39ECE70678ACB2F60742BFD9
:107AF000E4435EFA84FE1FFA8EF4E4B248BFCEF38C
:107B0000072E49B17E1E07F8014CB342DCD0ACF120
:107B1000080C2D0A3746E1E73E4606F8014B96422F
:107B2000F4E70000D0E901329FED0C0A9FED0C7ADA
:107B300002EB43039A4205D30378DB0748BFB1EE5B
:107B4000400A704733F8021D07EE901AF8EEE77A04
:107B5000E0EE077AB0EE670AECE700BF0000000035
:107B600000008047D0E9023293423DBF5A1C826038
:107B700018784FF0FF30704790F8703083B1036988
:107B8000C3614369036283694362836E1A78026149
:107B90005A7842619B7883610323A0F87230704762
:107BA000C2690261026A4261426A82614366F4E725
:107BB00010B502690A2A04463BD1836A0133836205
:107BC0000123E36263692361A369636194F8703000
:107BD000002B36D0B4F87230626E93421FBF591C2E
:107BE000A26EA4F87210D35C08BF0023A36163697E
:107BF0000D2B08D1A3690A229342626103D1D4E913
:107C000001039847A061A369013306D163695A1C37
:107C100003D00A2B1CBF0A23A36194F87030ABB1C8
:107C200023699BB984F870302046BDE81040FFF707
:107C3000A3BFC36A092A04BF073323F00703013334
:107C4000BFE7D4E901039847A061D0E710BD70B544
:107C500004460D4600262269531C01D1304670BDF2
:107C60000A2A08D115B1636B002BF7D02046FFF725
:107C70009FFF0126EFE71046FFF70AFE18B12046E6
:107C8000FFF796FFE7E7232A08D12046FFF790FF8A
:107C900023695A1CDFD00A2BF7D1DCE75C2ADDD13F
:107CA00063690A2BDAD12046FFF782FFE7E7D0E9C4
:107CB0000432013B036152F8230070470369C94352
:107CC0001944436953F821007047B0F59F7F07D0EE
:107CD00010F0010306D043080CBF012000207047BC
:107CE0000120704718467047B0F5AF7F07D010F0FD
:107CF000010306D0430814BF012000207047012073
:107D0000704718467047000010F0010204D040F0A0
:107D10000100086001207047A8B110F003030FD1E3
:107D20000279372A0ED183680B6013F00100F1D17C
:107D30009A0708D11868044BC31A58425841704733
:107D40001046704718467047800A070010B5036850
:107D500013B91360184610BD9C0702D010600120B3
:107D6000F9E71C798C42F9D103F1080111605868D8
:107D7000000AF0E730B5058D04460022954201D88F
:107D8000002030BDE36A03EBC20043688B42F8D0A9
:107D90000132F3E7838B426A01339BB28383918C78
:107DA000994238BF93847047F7B51E4659B111F018
:107DB000030511D14F68FCB294420DD13F0A01F185
:107DC0000804BD4201DB03B0F0BD54F8041B019070
:107DD0000135B0470198F4E7334603B0BDE8F04001
:107DE00018470000024B89689722FFF7DDBF00BFEC
:107DF000F5710400024B89686722FFF7D5BF00BF09
:107E0000BB58050031B1026801F00303134304BFFE
:107E10000B680360704770B504460D46104619465E
:107E2000FFF7A8FF037833B96D681A4620462B4642
:107E3000BDE870401847012BF6D02D684288022B10
:107E40002046AC4608BF0023BDE8704018BF0123A0
:107E5000604737B50DF105040B46214602F07F055A
:107E6000D20904F8015DF9D1091B984701AD01461B
:107E70002346AB4205D19DF804201B1BC25403B01E
:107E800030BD13F8012B62F07F0201F8012BF0E7FF
:107E90004379026A032B88BF036B114494BF0346E6
:107EA0009B1801621846704710B50C460121FFF778
:107EB000EFFF047010BD4279836A032A88BF426ACB
:107EC000194484BFD218036B816294BF03469B1888
:107ED0001846704710B50C460121FFF7ECFF0470FF
:107EE00010BD000013B504460192FFF7F3FF019A9D
:107EF0000349204602B0BDE81040FFF7AABF00BF0B
:107F0000B77E020030B4C36815465C8B9A8B038F32
:107F10001444C28E14445A1C02871A194379042B44
:107F200004BFC36B43F8225030BCFFF7DBBF2833DC
:107F3000D9B2FFF7D7BF38B50D4603211446FFF776
:107F4000BAFF4470240A0570847038BD38B543798F
:107F5000032B81BF846AC369C4F1FF2404F57F0445
:107F600084BF53F82230FD340D464FF003018CBF1F
:107F7000E4180024FFF79FFF4470240A0570847002
:107F800038BD38B54379032B81BF846AC369C4F512
:107F9000FF4453F8223088BF7D340D464FF0030173
:107FA0008CBFE4180024FFF786FF4470241205708C
:107FB000847038BD4379012B09D083681944C368A4
:107FC00081605A8C9142C8BF5984002383717047E5
:107FD00070B501211D4606461446FFF7EBFF45B973
:107FE0000F2C06D8A4F15001C9B2BDE87040FFF7CC
:107FF00071BF05F1190122463046C9B2BDE8704093
:10800000FFF770BF70B514460E461B340121FFF711
:10801000D1FF3246E1B2BDE87040FFF78CBF70B5CA
:108020004FF0FF311D4606461446FFF7C3FF45B922
:108030000F2C06D8A4F14001C9B2BDE87040FFF78B
:1080400049BF05F1220122463046C9B2BDE8704061
:10805000FFF748BF70B514460E4624344FF0FF3189
:10806000FFF7A8FF3246E1B2BDE87040FFF763BFFB
:1080700070B514460E462A340021FFF79BFF3246A6
:10808000E1B2BDE87040FFF756BFF7B5DDE908760D
:10809000C91AD4B243EA07220546A1EB470101926F
:1080A0005EB10239FFF786FF611C019AC9B228460A
:1080B00003B0BDE8F040FFF715BFFFF77BFF019A63
:1080C0002146F4E713B501910021FFF773FF019AF0
:1080D0001D2102B0BDE81040FFF72DBF10B54FF0D5
:1080E000FF31FFF767FFBDE810402121FFF7F2BE27
:1080F00038B50D460021FFF75DFF4379012B05D010
:10810000032B9EBFC369826A43F8252038BD13B58F
:1081100001910121FFF74EFF019A162102B0BDE83F
:108120001040FFF708BF10B50121FFF743FFBDE87E
:1081300010401821FFF7CEBE10B50121FFF73AFF1E
:10814000BDE810403021FFF7C5BE10B54FF0FF313C
:10815000FFF730FFBDE810403221FFF7BBBE10B57E
:108160000021FFF727FFBDE810403321FFF7B2BE23
:1081700010B50021FFF71EFFBDE810403421FFF7C6
:10818000A9BE13B501910021FFF714FF019A352113
:1081900002B0BDE81040FFF7F4BE10B54FF0FF315C
:1081A000FFF708FFBDE810404121FFF793BE38B547
:1081B0000C1E14BF03210021FFF7FCFE002C18BF8A
:1081C0004721BDE8384008BF4221FFF783BE10B504
:1081D0000021FFF7EFFEBDE810404421FFF77ABE13
:1081E000302937B50C461AD031291BD10125072477
:1081F0004FF0FF310190FFF7DDFEA4F12901019856
:10820000C9B2FFF767FE019875B10021FFF7D2FEF2
:108210000198D32103B0BDE83040FFF75BBE0125D4
:108220000624E5E70025E3E703B030BD70B5032A77
:108230000D46144614BFC5F1010101215034FFF76A
:10824000B9FE2A46E1B2BDE87040FFF74BBE10B55B
:108250006FF00101FFF7AEFEBDE810405421FFF7BB
:1082600039BE2DE9F74F05460C46904699461BB19D
:108270000B7E43F008030B76A4F81E806B6A1B7814
:10828000002B4DD159EA0803A86A4CD10121FFF710
:1082900091FE6269602103B0BDE8F04FFFF732BE86
:1082A000DB6A03EBC70B13F83730033B012B1AD8FB
:1082B0004FF0000A14E0E36A03EBCA0213F83A3005
:1082C000042B0BD1DBF804105368994206D1BBF89C
:1082D0000220A86A0023FFF77BFE01360AF1010A9B
:1082E000238D5345E7DC01376B6A1A8DBA42D7DC20
:1082F000002EC7D059EA0803A86AF5B21AD1C6F110
:1083000001010190FFF756FE626962210198FFF7B3
:10831000F9FD0198294603B0BDE8F04FFFF7DABD3B
:1083200000273E46E0E74FF0FF31FFF743FE62696A
:108330006121B0E7F1430190FFF73CFE62696321E0
:10834000E4E70000F8B504460E4611461A4600233D
:1083500085794769837143610D4BFFF725FDA3685C
:10836000A3B9E18A39B1A28A2AB9A06AFFF75EFFF0
:10837000A06AFFF7D8FEA38AE28A31462046FFF7BB
:1083800070FF003D18BF0125A5716761F8BD00BFF2
:108390003973040007B5CDE900230B4664220021A0
:1083A000FFF773FE03B05DF804FB10B54FF0FF312B
:1083B000FFF700FE0123BDE8104083715B21FFF74A
:1083C00089BD38B50C464942FFF7F4FDC268137EFB
:1083D00043F0040304F15D011376BDE83840C9B2EF
:1083E000FFF778BD2DE9F74F10EE104A002C9DF8ED
:1083F0003050044624DAB4EE400AF1EE10FA1FD6EB
:108400002D2504F8015BB1EE400A9FEDC47AF0EE31
:10841000C07AF4EE477AF1EE10FA02F0200E14DD85
:108420008EF0490323708EF046058EF04E03637084
:10843000A570E31C00221A70181A03B0BDE8F08F73
:10844000002DE2D004F8015BDFE7B4EE400AF1EE64
:1084500010FA08D74EF04E028EF04105227065707A
:10846000E31CA270E6E7002B42F02002B8BF06230F
:10847000672A02D1002B08BF0123251A491B10EEE1
:10848000105A002D01F1FF3748D1662A38D15D1C02
:10849000AF424FF00006D8BFCB1E591C6627B4462A
:1084A0003546652F23EAE37840F0098108F10101A0
:1084B000002301934FF02E0BB2EE047A019B8B4206
:1084C000C0F20681662A40F03381A94280F286819B
:1084D00096B10A2195FBF1F301FB135593FBF1F2E1
:1084E00001FB12324EF0450E3032303584F800E098
:1084F0006670A270E570043400232370201A9CE794
:108500005D1DAF42D8BFCB1F652A17464FF0000153
:1085100040F0CF802B268C460D46C2E7B5F17E5F3A
:108520006FD2DFED7F7ADFF80082DFF800A2B4EED1
:10853000E70AF1EE10FA4FF00006ACBF4FF0310938
:108540004FF030094FF0200C3546B8EC017AB4EE0C
:10855000C07AF1EE10FAC4BF0AEB060B9BED007A6D
:1085600006F10406C4BF654420EE070A182E4FEA40
:108570006C0CEAD110EE106AB6F17E5F27D2B4EE31
:10858000E70AF1EE10FA1DDB002D14BF2D262B2675
:10859000B7EE000A662A03D0672A28D1042D26DC0C
:1085A000672A04BF05F1FF369B195E1CB742D8BF8E
:1085B000CB1E84F8009063B9013419461E464FF073
:1085C000FF3C58E0F2EE047A20EE270A01352D2612
:1085D000E0E72E216170302619460234013D6AD051
:1085E00009B90E46EBE704F8016B0139F6E78F1F76
:1085F000BB4202DB672A60D0CB1F174600218C46A6
:108600004FE70026DFF82481DFF81C914FF0200CA3
:108610003546F8EC017AF4EEC07AF1EE10FA9CBF20
:1086200009EB060ADAED007A06F104069CBF654400
:1086300020EE270A182E4FEA6C0CEAD1FDEEC07A24
:1086400017EE906A092EC2BFDFED367A013520EEB3
:10865000270A662A11D1AF4217DD591901318F421D
:1086600005DC7F1B012FA7F1020308BF0023E918D7
:108670000131AC460026662713E7652A05D0672A34
:108680000CD0174600212B26B9E78E1FB34200DB22
:10869000CB1F00212B268C46652702E71E1DB74203
:1086A00000DC8B1F9D4201DB6727EBE7691C5B1A2F
:1086B000DDE70E462FE72E4681E73B469DE7672F15
:1086C0007FF4F6AE002BDABF012188464146EFE683
:1086D000FDEEC07A04F1010A17EE903A002BA8BF14
:1086E00003F13009019BACBF5FFA89F94FF0300903
:1086F000634584F8009006D1B8F1000F03D004F16F
:10870000020A84F801B0F8EEE77A019B30EE670ABE
:10871000013320EE070A01935446CFE6FFFF7F7F27
:10872000F8FF7F3FCDCCCC3D00D5060018D5060024
:10873000F1EE047AB4EEE70AF1EE10FA28DB611EDE
:108740004FF030090B782E2B8C4601F1FF31F9D018
:10875000A3F1300ABAF1090F2CD90CF1010C9CF8E5
:108760000030302B14D19CF801102E292FD1662F08
:108770002DD02D2E8CF800108CF8013025D1013D24
:1087800008BF2B2623469C4523D331238CF8003089
:10879000672A7FF49DAEB8F1000F3FF499AE2346EF
:1087A0001C46013B14F8012C302AF9D02E2A08BFB0
:1087B0001C468DE6392B03D001338CF80030CEE710
:1087C000604581F80190BDD1C9E70135DAE7013490
:1087D000D8E713F8011C03F80119D4E7F1EE047A85
:1087E000B4EEE70AF1EE10FAA9DA71E600F003033D
:1087F000022B05D1034B0340981F18BF012070477F
:1088000000207047070080FF50F8210010B10438A5
:1088100018BF01207047704708B5C307024608D447
:10882000074B0340062B06D0FFF7E0FF28B910687E
:1088300008BD0448FCE70448FAE70448F8E700BF2D
:10884000070080FF800A0700040E070028080700C1
:1088500038B5816804460846FFF7DEFF43690546E0
:1088600005209847E168B1EB600F0ADA49002B6AEE
:10887000A068042241F001019847E3680133E360F6
:1088800038BD0020FCE708B5FFF7C6FFBDE808408B
:10889000C088FEF7F3BE7047044B0B60044BC1E980
:1088A00001300023CB600846704700BF240C07004E
:1088B0005188020013B504460192FFF7ADFFC36A69
:1088C0003BB1019A20469847B0FA80F0400902B0C7
:1088D00010BD1846FBE7062806BF480040F001001F
:1088E00000207047042803D0052808D000207047D6
:1088F0008A68054B0548002A08BF184670478868F3
:10890000400040F001007047A0E10600ACE1060025
:10891000074BC1E900300023C1E90233054B02686F
:108920009A4202BF4368C3F317238B60084670471F
:1089300098990600340B0700136870B56BB944684A
:10894000A51C50F825509C4207D055F82360B14231
:1089500004D1023350F82330136070BD0133F2E7C5
:1089600013685BB940F22633994208D1436823F07B
:10897000030343F00203A3F1FF4313607047B1F513
:10898000197FFBD18368F2E7044B0B60037A0B710C
:1089900043688B600023CB60084670473CBD0600EF
:1089A000044B0B6001230B7100238860CB600846E9
:1089B000704700BF3CBD060038B585680B680246AD
:1089C0000C46AB4201D3002009E01946D068FEF7FF
:1089D0002FFE591C20B12160D06800EBC30038BDC8
:1089E0000B46EEE7042803D0052809D00020704785
:1089F0004B68074833F00F03064B08BF1846704713
:108A00004868C0F31B10400040F00100704700BFF1
:108A1000ACE10600A0E1060010B4C4680023A4463F
:108A20005DF8044B604700221146FFF7F5BF0000D8
:108A300038B504461546FFF7EFFE074BC2689A4269
:108A400018BF2469A36813B90B602B6038BDE38895
:108A50000B60A368F9E700BF2975030001F1FF432C
:108A600023F0030307EE903A072805D8DFE800F06B
:108A7000051D04040704101800210846704710481B
:108A80001049F5EE407AF1EE10FA08BF0146F4E71E
:108A9000FDEEE77A17EE901A490041F00101ECE78C
:108AA000F5EEC07AF1EE10FAE7D5F1EE677A17EE3F
:108AB000901A21F0030141F00201A1F1FF41DCE72E
:108AC000A0E10600ACE10600C30706D5401000286F
:108AD0000DDB14BF012000207047836853B1037978
:108AE00013F0010F14BF4FF0FF30012070474FF01B
:108AF000FF30704718467047044B0B60044BC1E9C8
:108B000001300023CB600846704700BF240C0700EB
:108B1000158B0200D0E9022391688B423BBFD268DB
:108B200052F823200022013338BFC360104670473B
:108B300000487047A8E1060043681847C268002A49
:108B400005DDD0E90113994206DB00230AE0FCD0E1
:108B5000D0E901139942F8DD41684B000A4443F023
:108B6000010342601846704710B5D0E90142C3685E
:108B70000348C1E90223C1E90004084610BD00BF53
:108B8000901C0700820708D10068064B984206D067
:108B9000054BC31A584258417047002070470120C6
:108BA000704700BF140D070064080700044B0B60FA
:108BB000044BC1E901300023CB600846704700BF79
:108BC000240C0700C98B020038B58268C16855685B
:108BD0000346A94201D3002008E0D068FFF714FE45
:108BE0004C1C20B1DC60D36853F8210038BD21460D
:108BF000EFE7000010F0030203D10168084B99422F
:108C000009D010F0010306D13AB90068054BC31A28
:108C1000584258417047012070471846704700BFBE
:108C200058050700800A070010B50446FFF7E2FF69
:108C300028B92046FFF7DAFD00F0010010BD012041
:108C4000FAE70000044B0B60044BC1E9013000233C
:108C5000CB600846704700BF240C0700AD8C0200B3
:108C6000884230B513D20378303B092B0FD800234C
:108C700013600A2510F8014B1368303C05FB0343D1
:108C80008142136003D00378303B092BF2D930BD09
:108C9000054A0240062A02D1C008FEF7F4BC8268E9
:108CA0000A60C068704700BF070080FF13B5044624
:108CB00001A98068FFF7ECFFE268019B9A423FBF81
:108CC000835C5B0043F0010001322CBF0020E260B6
:108CD00002B010BD73B50546084601A9FFF7D8FFDD
:108CE000019B064613B3134B9D4221D0124B9D426C
:108CF0004FF0000405D1224613E0305DA847A8B12B
:108D00000134019BA342F8D80C4802B070BD315D1C
:108D10000846FEF7C7FD18B10846A847024628B125
:108D20000134019BA342F2D8002AEDD10448ECE7BC
:108D30000024E0E7CD780200E1780200ACE1060013
:108D4000A0E1060001460148FFF7C4BF9178020088
:108D500001460148FFF7BEBFA57802000146014861
:108D6000FFF7B8BFB978020001460148FFF7B2BF6C
:108D7000CD78020001460148FFF7ACBFE178020060
:108D8000012A13B50C460AD101A9FFF781FF019B07
:108D9000636042232060A360002002B010BD002366
:108DA000C1E900334FF0FF338B600120F5E700008D
:108DB000044B0B60044BC1E901300023CB60084633
:108DC000704700BF240C07008961050013B50446F5
:108DD000084601A9FFF75CFF042C04D0052C09D03C
:108DE000002002B010BD019A0648074B002A08BFB8
:108DF0001846F6E70199FEF73BFD400040F0010000
:108E0000EFE700BFACE10600A0E10600D0E90223D5
:108E100051688B4237BF991C002252F82120013340
:108E200038BFC36010467047044B0B60044BC1E968
:108E300001300023CB600846704700BF240C0700B8
:108E40000D8E0200F8B50E46114C1249124B8842A5
:108E50001AD0C268A24203D0306001242046F8BD77
:108E6000406B98B102689A42F1D1476800F1080559
:108E700005EB87070024BD42F0D255F8040B3146BC
:108E8000FFF7E0FF0444F6E70024E7E70446E5E7E0
:108E900081F70400AC0B0700B80E0700F0B50C46D4
:108EA00085B054F8046B019200220392054603A991
:108EB0003068FFF7C7FF0398019BC7682246691E09
:108EC000B8473061014805B0F0BD00BFA8E1060019
:108ED0002DE9F041134E144F0D46A8421CD010F05E
:108EE00003031BD10268B2421AD1406B90B10368F0
:108EF000BB42F2D1044654F8043F00EB830000F17A
:108F0000040854F8040FA045E7D92946FFF7E0FF0D
:108F10000028F6D0BDE8F0810120FBE70020F9E74A
:108F20001846F7E7F40E0700B80E0700830707D1CD
:108F30000268064B9A4203D1C268054B9A4202D09E
:108F40000449FFF7C5BF0120704700BFF40E0700BA
:108F5000297503009CFD060008B5FFF75DFCBDE820
:108F60000840FFF7E3BF38B504460D46FFF7F4FFAE
:108F700018B12046FFF750FC044629462046BDE8BC
:108F80003840FFF7A5BF70B504460D46FFF744FC17
:108F90000646FFF79DFF20B1AE4200D0246920466F
:108FA00070BD0446FBE7000010B5044608460A49B8
:108FB000FFF7E9FF042C03D0052C08D0002010BDDA
:108FC0008268064B0648002A08BF1846F7E7806803
:108FD000400040F00100F2E7BC0A0700A0E10600F3
:108FE000ACE106000C4970B5FFF7CDFF836803EBD9
:108FF000D37149109B0000229142A3F1040301DCCC
:10900000064870BDC468E65854F8225044F82260FF
:10901000C4680132E550EFE7BC0A0700A8E106008A
:1090200010B50446FFF7F8FB0422036A2046BDE8AA
:109030001040184713B504460192FFF7EDFB019A63
:10904000036A204602B0BDE81040184710B5044638
:10905000FFF7E2FB0022036A2046BDE810401847F4
:1090600013B504460191FFF7D7FB019A83692146A6
:109070002E2002B0BDE81040184710B5044608463F
:10908000FFF7CAFB006B18B10388A34218BF00208A
:1090900010BD014640F20E30FFF7EFBF2DE9F0475B
:1090A0001E4681468A461546FFF7F3FF9DF820705D
:1090B000D0E9018317F0020F4FF0000418BF984663
:1090C000346007F001076DB133462A4651464846E1
:1090D000C04738B1431C08D133680B2B02D10CB107
:1090E000002333602046BDE8F0871FB982442D1A63
:1090F0000444E8E70446F5E7014BD868704700BF31
:10910000D04E0120014B9868704700BFD04E01201F
:10911000024B0348002283F80A227047D04E0120F8
:10912000A8E10600024B0348012283F80A22704797
:10913000D04E0120A8E10600044B054A93F80A022C
:10914000044B002814BF104618467047D04E01202B
:10915000ACE10600A0E1060000B589B001A8FEF769
:10916000EBF90398400040F0010009B05DF804FB02
:1091700000B589B001A8FEF7DFF90298400040F081
:10918000010009B05DF804FB034A0448B2F8083254
:10919000013BA2F808327047D04E0120A8E106003A
:1091A000034A0448B2F808320133A2F80832704783
:1091B000D04E0120A8E1060010B50268002312F885
:1091C000011B01F07F04090644EAC313F7D40260CF
:1091D000184610BD0138013910F8012F11F8013F70
:1091E0008AB163B97F2A07D80B4B9B5C13F00C0F35
:1091F0000FD15F3A53425341C3F1010306E09A4253
:10920000EAD000207047B3FA83F35B0903F0010052
:1092100070470123F0E700BF149A0600002813DD11
:10922000002908DD6FF0404393FBF1F18142ACBFB0
:109230000020012070474FF0404393FBF0F088423C
:10924000D4BF002001207047002905DD4FF04043C6
:1092500093FBF1F18142F3E70028EBD06FF040433C
:1092600093FBF0F0E2E7782820D86D2807D8622831
:1092700017D0662817D0612808BF07207047A0F1D3
:109280006E030A2B12D8DFE803F01011111106113A
:10929000111108110A000D2070470B2070475C2047
:1092A0007047082070470C2070470A2070471FB590
:1092B0008388C2889A42044610D3172B15D90123FC
:1092C000009300F1080103AB00681822FFF7E6FEE7
:1092D000039B80B2A08043B938B1E380E088431C8F
:1092E000E3800444207A04B010BD4FF0FF30FAE769
:1092F000BFF34F8F0549064BCA6802F4E06213437F
:10930000CB60BFF34F8F00BFFDE700BF00ED00E073
:109310000400FA052DE9F04F00228578DFF8A4C09B
:10932000DFF8A4E0072416461746038803F1FF3848
:10933000424505DB0B44084603F8017CBDE8F08F8D
:109340004FF00009CA46C8464B465B0015F0800F37
:1093500008F1010818BF43F001035FFA88F884B9E7
:10936000741CE6B250FA84F4A5780724BAF1000F11
:1093700001D053450AD31CF808B00BEB4A0AD94474
:10938000E3E76D00013CEDB2E4B2EFE74B44A3EB41
:109390000A0301EB02081EF803307F2B04DC8B5418
:1093A00001231A4492B2C0E74FEAA31903F03F0326
:1093B00063F07F0369F03F0901F8029088F80130FB
:1093C0000223EEE7E8D7060092650700034B1B680F
:1093D000DB0700D500BE0020704700BFF0ED00E0C5
:1093E0000120704708B50B7803F06003202B0FD1E4
:1093F000084B8A88187890420AD14A78202A05D1E9
:10940000054A1AB1991D0020AFF30080012000E049
:10941000002008BD7426012000000000024B1B68DC
:10942000DB0700D500BE7047F0ED00E0002070477C
:109430004DDF70474EDF70474FDF704750DF70479A
:1094400012DF704748B9064BD3F8D80030B1034655
:10945000C0680028FBD1986870470020704700BFA3
:10946000D04E0120012808B50BD8FFF7EBFF38B12B
:10947000836943B1808800F03000203818BF012094
:1094800008BD0020FCE71846FAE7807A400040F06B
:1094900001007047C07A400040F001007047FEE7CD
:1094A00061DF70474BDF704730B5084A52F8D03F54
:1094B0003BB19C6884421C6804D15D688D4201D137
:1094C000146030BD1A462346F2E700BFD04E01209B
:1094D000B1DF7047B2DF704730B5124D044600204F
:1094E000E8B14378FF2B18D0C388033323F003037C
:1094F00008331844A84210D84378002BF0D04378A2
:109500008B42EDD1FF2907D0037803F00103A3427A
:10951000E6D143889342E3D130BD0020FCE7024806
:10952000EDE700BFFB1F0F0004A00E004288437848
:10953000007843EA022340EA032070470B0A0170D7
:1095400043700B0C090E8370C1707047036A0239B7
:10955000023B8B4283BFC389406B01FB03000020A9
:109560007047836A02680433D289490AB1FBF2F179
:10957000186830B1814202D3091A0833F8E75868F5
:109580000844704700F10B010022D30143EA520363
:1095900010F8012B52FA83F38842DAB2F5D1104663
:1095A0007047CA7E8B7E032843EA022301BF487DB1
:1095B0000A7D42EA002243EA024318467047C2F39A
:1095C00007238A76CB760378032B01BF120C0A752A
:1095D000120A4A757047000010B50749002331F898
:1095E000024B84429AB203D00133802BF7D11A4642
:1095F00002F18000C0B210BDB08B060070B51E4BEA
:109600001E4AB0F5805F28BF1346191D31F8043C8F
:109610000A46ABB1984213D331F8024C250AE6B2A0
:1096200053FA84F4A04221DA082D09D8DFE805F0C6
:1096300005090F11131517191B00C01A31F8100076
:1096400070BDC31A03F00103C01A80B2F8E71038E6
:10965000FBE72038F9E73038F7E71A38F5E7083044
:10966000F3E75038F1E7A0F5E350EEE70431002DC1
:10967000CCD102EB4603C8E756B8060048BA06004C
:10968000830705D16422B0FBF2F302FB13034BB94D
:109690004FF4C872B0FBF2F302FB1300B0FA80F093
:1096A0004009704701207047084B4A1E10B533F837
:1096B000114033F812300229A4EB030403D1FFF761
:1096C000DFFF00B10134204610BD00BF10BB060013
:1096D0004B4BA0F59E00A0F5D05070B590FBF3F475
:1096E00003FB14000028BCBF00F5A83004F1FF34D0
:1096F0004FF03C02B8BF00F5C0704FF46163B0FB9F
:10970000F3F30B71B0FBF2F302FB1300B3FBF2F5C2
:1097100002FB1535A31C072293FBF2F2C2EBC20237
:109720009B1A48BF0733002CB8BF04F50E34CB7129
:10973000BABF04F2B1244FF0FF330023887148F61A
:10974000AC623048B4FBF2F2042A08BF032200FBEB
:10975000024440F2B5562C4894FBF6F6192E08BF89
:10976000182600FB06444D7140F26D1594FBF5F58B
:10977000042D08BF03256FF4B67000FB05409C0064
:10978000234402EB820203EB830302EB82021B0100
:1097900003EB820303EB86032B449BB203F5FA62CF
:1097A0001A4D0A80002215F9014B844224DDD2B201
:1097B000941CE4B20B2C8ABF0A3A8C708A708A78A7
:1097C000134C02F10102D2B202F1FF3588BF03F25D
:1097D000D17300F1010034F8154088BF0B80C3B28B
:1097E000022A0888CB708A701C4403D9FFF748FF0F
:1097F00000B101340C8170BD001B0132D3E700BF02
:10980000805101005471FFFF4BFAFFFF04BB0600BB
:1098100010BB0600002910B514680CDA2144036857
:10982000002BBCBF1B19036003688B42D4BFC91A4D
:109830000021116010BDA14228BF2146EFE7012998
:109840001DBF16224FF0FF301A6000207047000045
:1098500000487047A8E10600064B1B68082B06D19C
:10986000054B1B68032B02D8044AD05C70470020CC
:10987000704700BF3001001034010010888A0600D4
:1098800041DF704729DF704728DF704707B50023A5
:109890000DF107008DF80730FFF7D2FD9DF80700A6
:1098A000003818BF012003B05DF804FB10B5FFF7C6
:1098B000EDFF054C18B9207004E0FFF7E1FF2378B5
:1098C000012BFAD0207810BD89510120074B10B52B
:1098D00001241C70FFF7D6FF28B9FFF7E7FF023815
:1098E00018BF012010BD0020FCE700BF89510120F6
:1098F000F0B508B3204E002133463546984204D0D7
:109900000131082903F10803F8D11C4A04681768DB
:109910004368BC4223F00303234415D14C1C05EBE0
:10992000C10513600021072C02DC55F8086F26B131
:1099300001B1136000230360F0BD696821F00301E9
:109940000B4401340121EEE70D4A17689F42F1D123
:1099500005EBC10314600021B34202D053F8085D47
:109960001DB10029E6D01460E4E7596821F0030135
:10997000641A0121F0E700BFC4460120D84A012043
:10998000EC4A012010B5084C206858B1FFF7B0FF31
:10999000064B93F85010002262F3C301226083F853
:1099A00050105A6210BD00BFA0510120F4220120C6
:1099B0002DE9F0431A4B1B4CD3F800C0D4F800E05B
:1099C000AEEB0C0282420646994611DB82070FD1AC
:1099D000154F00290BBF01204FF0FF300023072354
:1099E000B84657F833207AB11D18EBB2072BF8D9D7
:1099F000002007E0AEEB020247F83320226008EBBC
:109A0000C3035E60BDE8F08307EBC30026F00302EA
:109A10000029EFD1624447F833C0C9F80020EEE7CF
:109A2000EC4A0120D84A0120C4460120054B064AD1
:109A30001B681068834203D00021C01AFFF7B8BF2B
:109A400000207047EC4A0120D84A0120064B1868D4
:109A5000082802D104331B6823B9A0F10D03584232
:109A600058417047012070473001001042DF7047B5
:109A700043DF704744DF704707B5FFF707FF48B182
:109A800001A8FFF7F7FF0198003818BF012003B0C5
:109A90005DF804FB4FF08043D3F80C0400F0011094
:109AA000A0F1011358425841F1E700004309012297
:109AB00000F01F0002FA00F02033024A42F82300AF
:109AC000704700BF00E100E00028ACBF00F160403B
:109AD000064B4FEA4111B4BF00F00F0000F56140A2
:109AE000C9B2B4BF195480F80013704714ED00E0F8
:109AF00003681F2B83BF03F01F03036001484FF06F
:109B0000A04070470003005007B5019001A8FFF77F
:109B1000EFFF019B03F5E073032240F8232003B01D
:109B20005DF804FB07B5019001A8FFF7E1FF019B79
:109B300003F5E073022240F8232003B05DF804FB34
:109B400007B5019001A8FFF7D3FF019A01239340C5
:109B5000C0F8083503B05DF804FB07B5019001A813
:109B6000FFF7C6FF019A01239340C0F80C3503B0FC
:109B70005DF804FB10B5014690F82000FF2805D0E1
:109B80008B7F1BB9CB7F5BB1FFF7E7FF0023084654
:109B90004B770B72BDE8104050F8083B49681847F6
:109BA000FFF7CEFFF2E7000038B504791D49242302
:109BB0006343CA180546127F92B3CB5823B100689D
:109BC00040F30730FFF772FF24236343CA18CB58D2
:109BD0002D687BB1144BC5F80833537F53B1012373
:109BE0006B61D5F80431002BFBD0242303FB041355
:109BF00000225A77242303FB041393F82100FF2843
:109C000001D0FFF78FFF0023C5F80035074B9D42B9
:109C100004BF01225A60242303FB041100230B77A5
:109C200038BD00BF204D01205201080000F0024065
:109C30000023435082B043580193019B02B0704708
:109C40000B7B032B2DD8DFE803F025291D028A6842
:109C5000154B9A4204D1D0F84C350A699A4209D181
:109C60008A6840F202239A421BD1D0F84C354A69E7
:109C70009A4216D000230622C0F80035C0F800250D
:109C800018467047D0F84C350A699A42F2D1D0F89C
:109C90003C35ECE7D0F84C350A69E9E7D0F83C35BB
:109CA000FAE70120704700BF000204002DE9F843E5
:109CB0009846002380F82E30D36803F06043B3F158
:109CC000005F06460C46154603D0824F3846BDE875
:109CD000F883814BC1F8083390F82F3003F0FF0967
:109CE00023B183687D4FC1F80433EFE7012380F887
:109CF0002F30944600F10C07BCE80F000FC7DCF8CA
:109D000000303B6086F830906B78C4F888354FF4AB
:109D100082712046FFF78CFF4FF49271FFF788FFA6
:109D2000C4F85095C4F840952B78032B00F2B1800D
:109D3000DFE803F07A9C5E022B6903F06043B3F125
:109D4000005FC2D14FF48073C4F800326B68EA68D8
:109D5000C4F844254FF4A871C4F84835FFF768FFEC
:109D60004FF4B071FFF764FF4FF4A471FFF760FF89
:109D700001232362A360D4F85031002BFBD04FF4B1
:109D8000A8712046FFF754FFAB682A69C4F8442540
:109D9000C4F84835524BB3604FF482730822514FD8
:109DA000297803291CBF0121A1503268002A75D1EE
:109DB000012223441968002974D0D4F8C434C4F8AB
:109DC000C434002286F82F20002B79D0464A474F12
:109DD00013F0010F18BF174613F0020F02F1010232
:109DE00018BF174613F0040F414B18BF1F466DE70D
:109DF0006B68EA68C4F84425C4F848352B6903F059
:109E00006042B2F1005F7FF460AFAA68C4F83435F5
:109E10004FF48453C4F83825C4F8003240F20223CA
:109E2000B36001232362B7E76B68EA68C4F844258E
:109E3000C4F84835B8F1000F0ED04FF48073C4F861
:109E40000032274BB3604FF4A471FFF7F1FE4FF4DB
:109E5000A47301222262A1E74FF40073C4F8003218
:109E600040F20223B3604FF48273F2E76B68EA6852
:109E7000C4F83425C4F838354FF48053C4F80032A0
:109E800040F20223B3600123236200224FF4827365
:109E900085E7184F4FF48273082281E7B368C4F84E
:109EA000043313E7D4F82411002983D04FF49271BE
:109EB0002046FFF7BDFE4FF482732262626178E7AD
:109EC00031462046FFF7BCFE084B002808BF1F465E
:109ED000FCE600BF0A00AD0B02029C010B00AD0BBB
:109EE000000204000000AD0B0000AE0B0100AD0B42
:109EF0000200AE0B0400AD0BF0B5D0F8243187B0F2
:109F000004460D46ABB14FF49271FFF791FED0F8C5
:109F1000043173B9AB68C0F808330223AB60AB6897
:109F2000C0F8043301230362436185F82E3007B083
:109F3000F0BDD4F804316BB34FF48271204605F1C3
:109F40000C07FFF775FE0FCF01AE0FC63B683360FD
:109F500095F82E303BB929462046FFF771FE80F078
:109F6000010085F82E004FF4B0712046FFF760FE27
:109F70004FF4AE71FFF75CFE95F8303013B195F8F1
:109F80002E30CBB10023C4F80032AB60224BC4F8B2
:109F9000083311E04FF4A4712046FFF749FE2B7BF4
:109FA000EBB905F10C070FCF01AE0FC63B6833606C
:109FB00095F83030002BE6D0D4F8C434C4F8C4345B
:109FC0009A071ED501238DF8003095F830300BB973
:109FD00085F82F30D5E9003168469847A7E74FF458
:109FE0000073C4F8003240F20223AB6003F1CE7379
:109FF000C4F80833AB68C4F804330123A3602362B8
:10A0000095E713F0050F01D00223DCE795F82E3019
:10A01000002BD8D00423D6E702029C0103790B4918
:10A020000268342000FB0313094900209860C2F83D
:10A030000813D2F8001221F4BC51C2F80012C2F881
:10A040000005012283F82D20704700BF804D0120BC
:10A0500002029C0170B50679144D34237343EA184B
:10A06000044692F82D20FAB1EB5823B1006840F372
:10A070000730FFF71BFD2046FFF7D0FF342303FB1B
:10A08000065393F832304BB92368D3F80805FFF72D
:10A0900049FD2368D3F80C05FFF744FD342303FB87
:10A0A0000655002385F82D3070BD00BF804D01207E
:10A0B00001490248FFF720BF804D012000300040D9
:10A0C00002494FF04020FFF717BF00BFB44D0120F9
:10A0D0000023435082B043580193019B02B0704764
:10A0E0001FB50123CDE901218DF80030D0E900131F
:10A0F0006846984705B05DF804FB00002DE9F04183
:10A100002F4E0579242303FB0563044693F8202092
:10A11000002A52D05B6843B103682A4AC3F8082377
:10A12000006840F30730FFF7C1FC2268D2F8003224
:10A1300023F02003C2F80032236801225A6020680D
:10A140004FF4AC71FFF7C4FF2368DA602368D3F8DB
:10A150005821002AFBD00022C3F8002523684FF0C5
:10A16000FF32D3F80C05D3F81485D3F80815D3F8CB
:10A170001075C3F80C25C3F8142523689042C3F862
:10A180000825C3F8102501D0FFF7CCFCB8F1FF3F3C
:10A1900002D04046FFF7C6FC7A1C02D03846FFF7D3
:10A1A000C1FC4B1C02D00846FFF7BCFC242303FB78
:10A1B0000565002385F820306B60BDE8F08100BFA5
:10A1C000E84D01201003420007B5019001A8FFF7F8
:10A1D0008FFC019B00EB8300D0F8003723F4403361
:10A1E00043EA0141C0F8001703B05DF804FB07B56E
:10A1F000019001A8FFF77CFC019BD0F81005D84026
:10A2000000F0010003B05DF804FB0000054B4FF0C7
:10A21000FF32072843F8202084BFC01880F84C2064
:10A22000704700BF304E01200E4B034493F92420A9
:10A23000072A02DD0021FFF7C7BFD3B2072B10D8D2
:10A24000930003F1804303F5C043D3F8101521F0C8
:10A250000101C3F81015012303FA02F2024BC3F8FF
:10A2600008237047304E01200060004010B50E4AB0
:10A27000537903F0FF01A3B90C4B1960116821B1A8
:10A28000012454710A4AC2F8044300F1804000F5E9
:10A2900024300122026011B91A68002AFCD0054856
:10A2A00000E0054810BD00BF984E0120009102401B
:10A2B000009002400000AD0B0B00AD0B054A136887
:10A2C00033B1054B0020587110601A689968104727
:10A2D000704700BF00910240984E01206DDF70472B
:10A2E00072DF704773DF704774DF704775DF704748
:10A2F00078DF70477ADF70477BDF70477CDF70471D
:10A300007DDF70478ADF70478BDF70478CDF7047D7
:10A310008FDF704790DF7047A5DF704760DF7047C1
:10A3200069DF704767DF704710DF704711DF7047E4
:10A330000388102B03D01B2B03D000207047838889
:10A340000B8001208870704721290DD005D8112974
:10A350000AD0122908D039B17047312904D04129D7
:10A3600002D0222900D0704701707047A3DF7047E8
:10A37000ABDF7047ADDF7047AEDF704770B5EFF30E
:10A38000108672B60D4A94680123A4B993600C4BF1
:10A390000C4DD3F8801029401160C3F88050D3F8D9
:10A3A000841051604FF0FF32C3F88420047006B966
:10A3B00062B6002070BD0370F9E700BF2051012094
:10A3C00000E100E0FC06FFBDC38802899A420BD081
:10A3D0005A1C92B20168C280CB5C818891429CBFBA
:10A3E0000022C280184670474FF0FF30704710B50A
:10A3F00002898488531C9C4298BF0023C4889C42D5
:10A400001DBF0468A15403814FF0FF3018BF002026
:10A4100010BDC288038982B09B1A0193019B002B57
:10A42000BFBF019A83889B180193019880B202B044
:10A430007047000010B5084B9A685AB150B9EFF355
:10A44000108172B6054A1C6814605C68546098609C
:10A4500001B962B6002010BD2051012000E100E0EA
:10A46000F7B504460DF107000F461646FFF786FFC5
:10A4700000250C34AE4205D89DF80700FFF7DAFF3F
:10A4800003B0F0BD795D2046FFF7B1FF0135F1E77C
:10A49000034610B51A88392A08460DD0502A1AD119
:10A4A0004A68D988928A914204D11A8A03F112012A
:10A4B000FFF7D6FF01200FE01C7B012CFAD14A6880
:10A4C0005989928A914204D1DA8903F11001FFF788
:10A4D000C7FF204600E0002010BD00004368014691
:10A4E00013B10248FEF7E0BF704700BF91A402001D
:10A4F00076DF70477EDF70477FDF704786DF70470B
:10A500009BDF70479DDF70479EDF7047B5DF704768
:10A51000406878B1406868B1837953B1C06848B188
:10A52000406838B100884FF6FF73C01A18BF012089
:10A5300070470120704718B143680BB11888704705
:10A540004FF6FF707047A4DF704770B505460C46A4
:10A550008E18B44200D170BD21782846FFF747FF1E
:10A56000002806DA2846FFF72FFF21782846FFF754
:10A570003EFF0134EDE770B506460C468D18AC423F
:10A5800000D170BD3046FFF71FFF04F8010BF6E75E
:10A59000F0B5838B002187B0044680F82310002B90
:10A5A0003CD0626894F82250978A94F82020C08B9F
:10A5B00094F821600432F5B104EB8202CDF8091061
:10A5C00052688DF80D1002A98DF80860ADF80A7078
:10A5D000ADF80E300492FFF7C9FE50B994F8203060
:10A5E000A083013303F0010384F82030012384F8B1
:10A5F000233007B0F0BD04EB8202ADF806300DF158
:10A600000603049302A95368ADF808708DF80A6038
:10A61000ADF80C500593FFF7AFFEDEE71846E8E70C
:10A62000F0B585B08389ADF8062002329A4205461E
:10A630000E4620D80DF10D00FFF7A0FE05F108042D
:10A640002046A989FFF7E5FEBDF80630081A023357
:10A6500098424FF0020210DB0DF106012046FFF791
:10A6600074FF20469DF806203146FFF76EFF9DF8E7
:10A670000D00FFF7DFFE05B0F0BD0DF10E01204625
:10A68000FFF779FF0027BDF80E20BBB29A42D7D959
:10A690002046FFF799FE0137F5E738B50446CD8B24
:10A6A000A3889D42084606D12388392B05D023F084
:10A6B0000403382B15D0002005E04B6862899B8A83
:10A6C0009A4201D0012038BDE28904F11001FFF760
:10A6D000A7FF237B022BF5D161892846FFF733FFC3
:10A6E000F0E7FFF755FFEDE738B5034608461A884F
:10A6F000502A03D0572A24D0002038BD4468D98876
:10A70000A58A9A888D420FD1C18B4FF6FF74A14262
:10A7100007D1C2831A8A03F11201FFF781FF0120DA
:10A72000EBE79142E8D1F5E7648C8C42F7D1C48B1A
:10A730004FF6FF718C42F2D15B8ADB07EFD5C28303
:10A74000EDE7FFF725FFD7E7A8DF7047AADF7047DF
:10A7500062DF704764DF7047A1DF7047ACDF70478E
:10A76000012070471020704790F8203033B982687C
:10A77000D2F8041111B18377C2F80431807F704799
:10A780000C4B984211D00AD8A3F57F43F73B98426F
:10A790000DD0013398420CBF102000207047064BAB
:10A7A00098420CBF052000207047132070470520F9
:10A7B000704700BF0100AE0B0200AE0BFF280CD0AB
:10A7C0004109064A012300F01F0003FA00F052F885
:10A7D000213023EA000342F821307047BC490120B0
:10A7E00010B54368044643B11879FFF79BF96368D5
:10A7F0001879FFF7E3FF0023636010BD70B50E4BBF
:10A800000122002604465A60C3F80065FF2590F82F
:10A810002100FFF7D3FF94F8220084F82150FFF7BE
:10A82000CDFF94F8230084F82250FFF7C7FF034BB5
:10A8300084F823501E6070BD00500240DC4A0120A5
:10A8400010B5837AFF2B04460ED04068FFF702FC58
:10A85000A07AFFF7B3FF607AFFF7B0FFFF23A37280
:10A860006372636800221A7210BD10B5437AFF2B21
:10A8700004460DD04068FFF797F9607AFFF79EFF16
:10A88000A07AFFF79BFFE07ABDE81040FFF796BF84
:10A8900010BD00004109064A012300F01F0003FA21
:10A8A00000F052F82130184342F82100704700BFF1
:10A8B0000C51012003790649580903F01F020123B6
:10A8C000934051F82020134341F82030704700BFD7
:10A8D000BC4901204CDF704720B1034B800143F09D
:10A8E00001031847704700BF30BC060010B5094C83
:10A8F0002046FEF7A5FD237823B1BDE810400648A9
:10A90000FFF73CBD72B6BFF35F8F044A1368013393
:10A91000136010BD8A510120E04A0120045101203A
:10A9200030DF704731DF7047184B53F8203000227A
:10A93000022110B5C3F80025C3F80425C3F810158B
:10A940004FF4FA41C3F81425C3F80C25C3F80815D1
:10A950000F4901EBC004C3F820450424C3F8244583
:10A96000C3F82825C3F82C25C3F84025C3F844258F
:10A97000C3F84825C3F84C254FF4004321F8303084
:10A9800001EBC00043808380C38010BD3C1C0700E6
:10A990004051012001F5AC714FF0FF3340F82130F8
:10A9A000002303F5AC7250F82220013205D10133A7
:10A9B000042BF6D10023C0F80035704710B543686A
:10A9C00004467BB1007AFFF7ADF8617A6068002336
:10A9D000636001F07F01FFF7DDFF207AFFF7EEFEF5
:10A9E000FF23237210BD30B543684181D3F8205551
:10A9F000447AD3F8082504F07F0451434FF6FF73DF
:10AA0000B1FBF3F36FEA43436FEA534325F8143085
:10AA1000436801229A6030BD2DE9F84F00251646A3
:10AA20009DF828B004460F462A469A46002B7CD053
:10AA30004949A946012347F6FB70B1FBF3F8B8FB7F
:10AA4000FAF8A8F1040C844568D8DFF814C1002195
:10AA50005CF8040BD0F8003513F00F036FD0BBF196
:10AA6000000F67D1D0F80835984563D1D0F80C3580
:10AA70004B455FD15B4603F5AC7E50F82EE0BEF14E
:10AA8000FF3F54D15AB201256060002861D0637A3B
:10AA900062F3060363723B7923723846FFF70AFFBD
:10AAA000637A207AC4F80CA06BF3C7136372FFF7C4
:10AAB0002BF863680022C3F80025DDB96368274AD4
:10AAC00093420CD002F5A04293423BD002F5805253
:10AAD000934239D002F53042934237D10325E8B290
:10AAE000FFF722FF63680022C3F80C95C3F8042522
:10AAF000C3F80885637A6268397903F07F0303F548
:10AB0000AC73204642F8231063680122C3F8002585
:10AB10003146FFF768FF0020BDE8F88F09F1010911
:10AB2000B9F1080F4FEA430387D10220F4E701335C
:10AB3000042BA0D1013104298AD10020A4E71A46B0
:10AB40001D46A1E70125CAE70225C8E74FF0FF35FA
:10AB5000C5E70420E0E700BF0024F40000C0014086
:10AB60003C1C070003685B684FF0FF32C3F86025A8
:10AB70000368187AFEF7F1BF10B5174B53F8202081
:10AB8000FAB11079FFF733FBC1B250794C00FFF7EF
:10AB90002EFBE4B24140937954FA81F1C9B2CB1A49
:10ABA00003F00303012B0DD1D3790133D37192F953
:10ABB00007309171032B0ADD936801339360002302
:10ABC000D37110BD032BF2D1D379013BEEE70333F0
:10ABD000F7DA9368013BF1E7BC440120052801BF87
:10ABE000024A136803F50013136070478451012073
:10ABF0001FB5134BD3F80405124B1B6801A903EBD7
:10AC0000D000FEF765FD9DF807309DF806001B0497
:10AC100043EA40539DF8080043EAC0239DF8090029
:10AC200043EA40139DF80A0043EA5003BDF80400CC
:10AC3000A0F2BC7043EA406005B05DF804FB00BFC1
:10AC40000040024084510120807D400040F001001E
:10AC5000704700008068024B002808BF1846704704
:10AC6000A8E1060008B5FFF739FC014808BD00BFA0
:10AC7000A8E1060043683BB193F85A200348044B0F
:10AC8000022A08BF1846704700487047A0E1060036
:10AC9000ACE106008068024B002808BF18467047E8
:10ACA000A8E106004068704708B54368014613B143
:10ACB0000248FEF7F9FB024808BD00BF9BA6020050
:10ACC000A8E106008079034A034B002814BF104610
:10ACD00018467047ACE10600A0E10600C079034ABF
:10ACE000034B002814BF104618467047ACE106001D
:10ACF000A0E106008068024B002808BF1846704794
:10AD0000A8E106008088400040F001007047000084
:10AD1000C30747BF401007EE900A00F1FF4020F044
:10AD200003034CBFF8EEE77A07EE903A9FED337AD3
:10AD3000F4EEC77AF1EE10FA82B00EDDDFED306A84
:10AD400067EEA66AFCEEE66A16EE903A1B0206EE85
:10AD5000903AF8EE666A77EEE67ADFED2A5AF4EE7C
:10AD6000E57AF1EE10FAF0EE086A13D567EEA67AEE
:10AD700037EE677AFCEEE77ABCEEC77A8DED017AA2
:10AD80009DF80430CDED017A9DF80400000440EAFE
:10AD900003201AE09FED1C6AF4EEC67AF1EE10FA79
:10ADA00018D577EEE57A67EEA67A37EE677AFCEE8D
:10ADB000E77ABCEEC77A8DED017A9DF80430CDEDCF
:10ADC000017A9DF8040040EA0340400040F0010091
:10ADD00002B0704777EEC67A67EEA67AFCEEE76AB5
:10ADE00077EE677ACDED016AFCEEE77A9DF80430E4
:10ADF000CDED017A9DF80400C9E700BF00007F4354
:10AE00000000803B0000AA4200002A4308B5FFF77B
:10AE1000E7FC014808BD00BFA8E1060008B50868C6
:10AE2000FFF7DEFC004808BDA8E1060008B5086889
:10AE300090F82330FF2B01D0FFF7E0FC004808BD5D
:10AE4000A8E1060038B5084B0C681B680025C3F85C
:10AE500000552079FFF7B2FC60792571FFF7AEFC51
:10AE60006571024838BD00BF44220120A8E10600F8
:10AE700008B5FFF7E5FC014808BD00BFA8E10600E2
:10AE800008B50868FFF7DCFC004808BDA8E106002B
:10AE900008B5FFF7EAFC014808BD00BFA8E10600BD
:10AEA00008B50868FFF7E1FC004808BDA8E1060006
:10AEB000037A1BB9012303720148704701487047A8
:10AEC000ACE10600A0E10600064BD3F8B83093F8D9
:10AED000250093F824204000D2B283F8252040F0CA
:10AEE00001007047D04E0120F0B5134D3124013CD4
:10AEF00014F0FF0411D1114D3124013C14F0FF0472
:10AF000019D02E466F68B84205F10805F5D140F218
:10AF1000BB20086040F2F52109E02E466F688742A9
:10AF200005F10805E3D10020086040F29B11116093
:10AF30003268D2081A60F0BDB0B00600B4DA06007C
:10AF400008B5FFF7D3FC014808BD00BFA8E1060023
:10AF500000487047BC13070008B50868FFF72EFDCE
:10AF6000004808BDA8E1060008B5FFF727FD014825
:10AF700008BD00BFA8E10600024BC3F8B4000248B8
:10AF8000704700BFD04E0120A8E10600024B0348E5
:10AF900000221A70704700BF08470120A8E1060090
:10AFA000044B054801221A70044B03F138029A65DC
:10AFB000704700BF65510120A8E10600D04E012076
:10AFC00080687047C06870470079034A034B0028C7
:10AFD00014BF104618467047ACE10600A0E1060019
:10AFE0004079034A034B002814BF104618467047A7
:10AFF000ACE10600A0E10600F7B587689DF8206087
:10B000009DF82440042F04D1857C15B1E40844F058
:10B01000E004456A79435DB1042F08BF077C0D4405
:10B0200008BFEC55477BEA55877BEB55C77BEE5550
:10B03000056A29448568042D11D1857C6DB907EE18
:10B04000904A90ED067AF8EEE77A67EE877AFCEEA2
:10B05000E77ACDED017A9DF80440057C4C5507EE6A
:10B06000902A90ED067A447BF8EEE77A67EE877ACD
:10B07000FCEEE77A17EE902A07EE903A0A55F8EEC2
:10B08000E77A90ED067A827B67EE877AFCEEE77AC4
:10B0900017EE903A07EE906A8B54F8EEE77A90ED4F
:10B0A000067AC27B67EE877AFCEEE77A17EE903A73
:10B0B0008B5403B0F0BD000000234360004870478C
:10B0C000A8E1060000697047007B7047807B7047ED
:10B0D000704730B5039C85682560446849B1857B1D
:10B0E000B2FBF5F105FB1122017BD2B2C90802FBCC
:10B0F00001441C60002030BD10B501241470427B57
:10B100001A70029B82681A6001B1847B039B1C70D9
:10B1100010BD000000234360C3600148704700BFBA
:10B12000A8E10600806A7047807E704790F824008E
:10B13000704710B500241470827E082A94BF002244
:10B1400001221A70029B4FF400721A6021B190F82C
:10B150002430039A137010BD0123FAE70023C0E9DD
:10B1600001330148704700BFA8E1060040697047FD
:10B17000C07C7047007C704710B500241470827C3E
:10B180001A70029BC2681A6019B1C37C039A1370CB
:10B1900010BD0123FAE7008B07EE900AFBEEE87A78
:10B1A00017EE900A20F0030040F00200A0F1FF40EB
:10B1B0007047002210B5144690F82410D3B299427B
:10B1C00000D810BD00EB83030132DB6A9C60F3E71B
:10B1D000406A704790F82D00704710B50024147035
:10B1E00001221A70029B046A1C6009B190F82D209C
:10B1F000039B1A7010BD836813B10430FFF7F0BAD7
:10B200007047000008B5FFF7F6FF014808BD00BF12
:10B21000A8E1060008B50868FFF7EDFF004808BD83
:10B22000A8E1060030B5838899422CDA00292ADB90
:10B23000C3889A4227DA002A25DB838984685A4327
:10B24000837BDD080FD1C57B41FA05F52A440569EA
:10B25000008C294001FB0333C3F1200154F8223054
:10B26000CB40184030BD012D04EB820201D1505C6F
:10B27000F8E7022D02D132F81100F3E7042D02D1D4
:10B2800052F82100EEE70020ECE70000C1EB01419D
:10B29000084480EA50310C4B9FED0C7A01FB01F021
:10B2A0004EF64D4202FB0030094B01FB003020F00E
:10B2B000004307EE903AFAEEE07A67EE877AFCEE0A
:10B2C000E77A17EE900A70471F07310100007F43AD
:10B2D0000DDD0852C20CC0F3C403400943EAC22387
:10B2E00000F4FC60184340BA80B27047020C13238C
:10B2F0005343C2B2FF213632B3FBF1F3B2FBF1F29A
:10B30000C0F307201344B6225043B0FBF1F01844B9
:10B31000C0B27047C2B2030C9342194610B538BF91
:10B320001146C0F30724A14238BF21469342184674
:10B3300028BF1046A04294BF081A081B10F0FF0057
:10B3400010D0C9B28B420ED1A21AF0232824624336
:10B3500092FBF0F292FBF3F003FB1020002800DADE
:10B36000F030C0B210BD8C4207D1D21A02EB4002BD
:10B370002823534393FBF0F0F0E78A4203D11A1BD2
:10B3800002EB8002F4E70020EBE700000079034ABB
:10B39000034B002814BF104618467047ACE1060066
:10B3A000A0E10600436800221A727047C08840007E
:10B3B00040F0010070478088400040F00100704775
:10B3C000042806D0052806D18868400040F0010016
:10B3D0007047024870470020704700BFACE106008C
:10B3E00090F95030816A30B5002BB4BFB0F91240EB
:10B3F000B0F91040B0F90C30858923449CB28B7BA6
:10B40000C3B191F905204B8812FB05F21A4412B220
:10B41000A0F8462091F90530498813FB04F30B444A
:10B420001BB29A42D2BFA0F84A30A0F84A20A0F836
:10B43000463030BD91F904200B8812FB05F21A4406
:10B4400012B2A0F8442091F90430098813FB04F3E8
:10B450000B441BB29A42D2BFA0F84830A0F8482053
:10B46000A0F84430E5E790F95030816A30B5002B00
:10B47000B4BFB0F91040B0F91240B0F90E30C58930
:10B4800023449CB28B7BC3B191F904200B8812FB3F
:10B4900005F21A4412B2A0F8442091F90430098848
:10B4A00013FB04F30B441BB29A42D2BFA0F84830FE
:10B4B000A0F84820A0F8443030BD91F905204B8811
:10B4C00012FB05F21A4412B2A0F8462091F9053099
:10B4D000498813FB04F30B441BB29A42D2BFA0F875
:10B4E0004A30A0F84A20A0F84630E5E72DE9F041BF
:10B4F00090F82E309A07044622D4BDE8F0816368A4
:10B5000053F83500830710D10368B34212D190F885
:10B510005030C0F8288023F0140343F0140380F85F
:10B520005030FFF75DFFFFF79EFF0135638D9D42B1
:10B53000E5D3E2E7BB42F8D1414600F00BF8F4E76F
:10B54000024E034F002500F10808EFE758C9060036
:10B5500034C506000A1E90F82E3018BF012262F38F
:10B56000410380F82E309B0730B428D58C7BB0F98E
:10B570002420B0F9263014B114461A4623460C880C
:10B5800091F9045005FB024202814A8891F9054075
:10B5900004FB032343810B7990F8282013FB02F36B
:10B5A00003734B7913FB02F343738B7B83750B7B24
:10B5B00003754B7B43758B7913FB02F3837330BCAC
:10B5C000FFF794BFB1F90030B0F900209A42C8BF2C
:10B5D0000380B1F90230B0F902209A42C8BF43801B
:10B5E000B1F90430B0F904209A42B8BF8380B1F9B0
:10B5F0000630B0F906209A42B8BFC380704710B534
:10B60000B0F900301380B1F90040A342B8BF23461F
:10B610001380B0F904309380B1F90440A342A8BF6D
:10B620002346B2F9004093809C4218DAB0F9023008
:10B630005380B1F90240A342B8BF23465380B0F90A
:10B640000600D080B1F906309842A8BF1846B2F97A
:10B650000230D0808342ACBF0020012010BD00200A
:10B66000FCE7028883889B1AC2884088101A9BB224
:10B6700080B2584370474FF4B473F0B591FBF3F5C3
:10B6800005FB131100250123B0F84220066CB0F829
:10B690004040A0F84410456280F82A30058680F8C2
:10B6A000325021B1B42920D140F201130386002386
:10B6B00090F832C04363C36340F20113038590F8EE
:10B6C000301090F8313025B217B2BCF1000F16D00F
:10B6D0000787458719B18284FF2280F828201BB193
:10B6E000C484FF2380F82930F0BDB1F5877F80F84E
:10B6F00032300CBF80F8313080F83030D7E78663C5
:10B7000019B1FF21848480F82810002BECD0C2846A
:10B71000E7E7000038B5054643680C4619BB174AF1
:10B7200092F82E10C1F3400089071BD5934222D115
:10B7300038BD33B193F82E206FF3410283F82E20E9
:10B7400054B105F124012046FFF704FF94F82E3090
:10B7500043F0020384F82E3001236C6085F85830E2
:10B760000120E5E714469C42FAD094F82E20920777
:10B77000DFD50020DCE7002BDCD1D9E78C210120CC
:10B78000836900681847036A006818472DE9F04F7D
:10B790008DB004460593BDF858300693199B079267
:10B7A0005A88029290F84A20B3F800A0B3F80490A7
:10B7B000DB889DF85C809DF860600393072A0D4646
:10B7C0000ED80823B3FBF2F290F84B30534390F8B5
:10B7D0005020002A00F0B780BAFBF3FAB9FBF3F966
:10B7E0002046FFF7CDFF002E08BF46468DF82850B3
:10B7F0000125B8F1000F40F0AF800095E76920689F
:10B800000AAB42464146B847AB464546AA1C04929D
:10B81000B4F84620B4F95430FF2A00F2A080DAB21E
:10B820005AFA83FA0CAB2B4403F808AC531E994424
:10B830006A1C0CAB134403F8089C05F102090AAB1F
:10B840002068E769CDF8009032465946B84720464F
:10B85000FFF799FF059BB3F5807F1BD04FF0010ADE
:10B8600020468DF82730FFF78BFF2068E769CDF879
:10B8700000A00DF1270332460021B847C9F3470362
:10B8800020680093E7690AAB32465146B847204624
:10B89000FFF779FF2046FFF773FF079B8DF82830ED
:10B8A000B8F1000F07D1012300932068E7690AABC4
:10B8B00042464146B847B4F84820B4F95630FF2A0A
:10B8C0000CAA0CA902EB050005F101020A4411467D
:10B8D00063D8029DDAB255FA83F300F8083C531E90
:10B8E000039A134401F8083C049B206800933246F5
:10B8F0000AAB5946E569A8472046FFF744FF069B77
:10B90000B3F5807F1CD04FF0010820468DF827301A
:10B91000FFF736FFE5692068CDF800800DF12703B9
:10B9200032460021A847049B2068E569C3F347031A
:10B93000009332460AAB4146A8472046FFF723FF53
:10B940000DB0BDE8F08F029AB2FBF3F20292039AB7
:10B95000B2FBF3F3039343E74FF0000B56E79AB2C1
:10B960001AFA83FA531E0CAA2A44CAF3072102F8D2
:10B97000081C691C0CAA0A44A81C02F808AC0CAAF2
:10B980004B440244C3F3072102F8081C0CAA2A44C2
:10B9900005F1040902F8053C51E7029F9AB217FA33
:10B9A00083F3C3F3072C039F00F808CC013A01F896
:10B9B000083CA91C0CAB0B441744C7F3072103F840
:10B9C000081C2B1D04930CAB1D4405F8057C8BE76C
:10B9D00038B5054634301446FFF711FE10B395F81C
:10B9E0004A20072A1ED80823B3FBF2F395F84B2010
:10B9F00095F8505013FB02F3DBB2A5B1B4F9002067
:10BA000092FBF3F103FB112109B1521A2280B4F920
:10BA1000042092FBF3F103FB112119B113445B1ACB
:10BA2000A380284638BDB4F9022092FBF3F103FB52
:10BA3000112109B1521A6280B4F9062092FBF3F188
:10BA400003FB11210029EDD013445B1AE380E9E7E1
:10BA500040687047A1F120035E2B2DE9F0410E46AE
:10BA600002D8D8B2BDE8F081C568078A4FF0000857
:10BA70002F44BD425FFA88F401D3FF20F2E7284645
:10BA8000FBF7D0FE01462846FBF7E9FE8E4205464D
:10BA900008F10108EDD104F15F00C0B2E2E70268ED
:10BAA000034610783E2805D83B2805D8212806D023
:10BAB000402070474028FBD101321A6070473E2079
:10BAC000FAE7000010B50C68606818B1FEF788FE50
:10BAD00000236360004810BDA8E1060010EE102AA4
:10BAE0006F4822F00043834282B04FEAD27111D9ED
:10BAF000B3F1FF4F79D8002940F0CF80DFED697AAC
:10BB0000B4EEE70AF1EE10FA47DDDFED677A20EEDA
:10BB1000270A6AE0654883425CD9654A93423CD86B
:10BB20009FED647A91BB30EE477ADFED637A0123B3
:10BB300037EE670A37EE407A37EE677AB6EE005A8C
:10BB400060EE054A9FED5D6ADFED5D6A60EE247A86
:10BB5000E7EE866AB7EE006AF0EE465AE6EEA75ABE
:10BB6000F0EE656AF0EE085AE4EEE65AF1EE084AA5
:10BB7000E0EE654A76EEE56AC6EEA45A65EEA75A8F
:10BB8000BBBBD0EE257A30EE670A2EE030EE077AA6
:10BB9000DFED4C7A4FF0FF33CAE7B6EE007A0029AA
:10BBA000FEEE007A08BFF0EE477A9FED477ADFEDB0
:10BBB000426A40EE077A9FED3F7AFDEEE77A17EE94
:10BBC000903AF8EEE77AA7EEC70A67EEA67AB0EEEB
:10BBD000407AADE7B3F14C5F09D212F0FF4F04D1C8
:10BBE00060EE007ACDED017A019B02B07047002330
:10BBF000A4E775EEC75A5A1C90EE257A77EE677A5D
:10BC000006D170EE676ABEEE000AA6EE850AECE782
:10BC1000012B16D1BDEE007AB4EEC70AF1EE10FA90
:10BC200006D530EE050A37EEC00AF8EE007A6EE768
:10BC300030EE670AF0EE007AA0EE276AB0EE460A10
:10BC4000D3E703F17F02D205382B06EE902A10D9F4
:10BC500030EE670A802B70EE067A05BF9FED120A60
:10BC600077EEA77A26EEA70A27EE800A30EE460A7C
:10BC7000BBE7C3F17F02D20507EE102A162BCDBF1A
:10BC800037EE877A30EE670A36EE476A30EE470ABB
:10BC900030EE060A20EE260AA7E7BFEE000AA4E768
:10BCA00043B895418071B1420000007F1872B13EE7
:10BCB0009115853F8071313FD1F717371030CF3A5A
:10BCC000688808BDD1F717B73BAAB83F10EE103A05
:10BCD000A3F50002B2F1FF4F59D35A0006D160EE2E
:10BCE000007ABFEE007A87EE270A7047002B04DA4D
:10BCF00030EE407ADFED2B7AF5E7DFED2B7A60EE60
:10BD0000277A6FF0180117EE903A284A9FED285ACB
:10BD10009FED284A1A44D30D7F3B0B4406EE903A20
:10BD2000254BC2F31602134407EE903AB7EE000A11
:10BD300077EEC07AB0EE007A37EE877AF8EEE66AF0
:10BD4000C7EE875A9FED1D7A9FED1D0A65EEA54A45
:10BD500026EE800A24EEA46AA6EE075A9FED197A11
:10BD6000A6EE047A27EE247AA5EE067AB6EE006AED
:10BD700027EE866AA6EE277AA7EE250AA6EE670AC0
:10BD800030EE270ADFED107AA6EEA70A7047B3F16E
:10BD9000FF4F06D2B3F17E5F01D00021B5E79FEDE2
:10BDA000010A7047000000000000004C0DFB4A0033
:10BDB00013CECC3EEEE9913EF304353F269E783E0D
:10BDC000D1F71737AAAA2A3F8071313F08B5FFF78C
:10BDD0007DFFDFED027A80EE270A08BD8E5D1340FD
:10BDE00008B5FFF773FFDFED027A80EE270A08BD82
:10BDF0001872313F10EE103AC3F3C752A2F17F011F
:10BE0000162982B013DC002913DB124A0A411A42B8
:10BE10000DD0DFED117A30EE270A002B8DED000AF0
:10BE2000A8BF9B18009923EA020300EE103A02B063
:10BE30007047DFED097A30EE270A002B8DED010AFD
:10BE4000019A04DB5A0018BF4FF07E53EDE74FF024
:10BE50000043EAE7FFFF7F000000807B10EE103A0E
:10BE6000C3F3C752A2F17F01162982B013DC002967
:10BE700013DB124A0A411A420DD0DFED117A30EE7F
:10BE8000270A002B8DED000AB8BF9B18009923EA02
:10BE9000020300EE103A02B07047DFED097A30EE8F
:10BEA000270A002B8DED010A019A04DA5A00054A8F
:10BEB00018BF1346EDE70023EBE700BFFFFF7F004D
:10BEC0000000807B000080BF10EE103A23F000429B
:10BED000B2F1FF4F70B502D3A0EE000A70BD002A88
:10BEE000FCD0002B04DA70EE407A87EEA70AF5E763
:10BEF00013F0FF424FEAE35129D0C3F3160242F494
:10BF00000002CB07A1F17F0058BF52000023401070
:10BF1000520019241E464FF0807175189542DEBFFD
:10BF20006E18521B5B18013C4FEA42024FEA510166
:10BF3000F3D112B1013323F001035B1003F17C5301
:10BF400003EBC05300EE103AC8E75B000132180261
:10BF5000FBD5013A891AD0E710EE103A23F00043DE
:10BF6000B3F1485F04DAFDEEC07A17EE903A5BB3A6
:10BF700020EE007ADFED157A9FED156AA7EE276AAD
:10BF8000DFED147AE6EE077A9FED136AA7EE876A73
:10BF9000DFED127A60EE076AE6EE077A30B99FEDC0
:10BFA000106AA7EE276AA6EE260A704767EEE67AC1
:10BFB000B6EE006AE0EE867AD7EE870ADFED097A00
:10BFC000E6EEA70A30EE600A704700BFD3C92E2FF5
:10BFD000342FD7B21BEF3836010D50B98988083C91
:10BFE000ABAA2ABEABAA2A3E10EE103A23F00043B9
:10BFF000B3F1485FB7EE006A05DAFDEEC07A17EEDE
:10C00000902A002A3DD060EE005ADFED1F7A9FEDA6
:10C010001F7ADFED1F6A1F4AA5EEA77A9342DFED74
:10C020001E7AE7EE257A9FED1D7AA7EEA57ADFED61
:10C030001C7AE7EE257AB0EE667AA7EEA57AF6EEE0
:10C04000006A65EEA67A67EE256A20EEC07AA5EE54
:10C05000A67A04DC37EEC77A36EE470A7047114AF3
:10C060009342DABF03F17F4306EE903AF5EE026A9F
:10C0700077EEE67A36EE660A77EEC77A30EE670A32
:10C080007047B0EE460A70474ED747ADF6740F3191
:10C09000ABAA2A3D9999993E7CF293B4010DD03711
:10C0A000610BB6BA0000483F10EE103A23F0004290
:10C0B000B2F1465F16DAFDEEC07A17EE901A39BB80
:10C0C000431C134306D1F0EEC07AB7EE007A87EE38
:10C0D000270A7047012800F0A080FFEE007A87EE63
:10C0E000800A70474D498A4212DBDFED4D7A002B02
:10C0F000B8BFB1EE400A37EEC00ADFED4A7AB8BFEA
:10C10000F1EE600A77EEE00A30EE800ADFED460AD3
:10C110009FED466ADFED466ADFED465A3F4920EE65
:10C12000007A8A4267EE077AE7EE866A9FED426AF6
:10C13000A6EEA76ADFED416AE6EE276A9FED406A48
:10C14000A6EEA76ADFED3F6AE6EE276A9FED3E6A3C
:10C15000A7EEA56ADFED3D5AE6EE275A9FED3C6A51
:10C16000A5EEA76ADFED3B5AE6EE275A9FED3A6A45
:10C17000A5EEA76AF0EE467AE7EE876A20EE076A38
:10C18000F0EE667AF0EE606AE7EE866ADFED337A0B
:10C19000E6EE870AE6EE270A30EE207A1DDB07EE90
:10C1A000900AF8EEE77A27EE076A37EE277A9B17B0
:10C1B000C6EE076A03F00203C3F10103B0EE007A92
:10C1C00076EEE00A70EE600A00EE103AE0EEC77A12
:10C1D000B8EEC00A20EE270A704701281BD0FFEEF8
:10C1E000007AC7EE876A1E4B17EE102A1A4006EE39
:10C1F000102A16EE902A36EE400A134070EEC00A5E
:10C2000000EE103AF7EE007AE6EE007AE0EE807A81
:10C21000A7EEA60A7047B0EE470A704740A12C3F30
:10C22000DA0F493F68212233000000005FAE9BB760
:10C2300045F4A3388453D937C8261A3A16696B3B9C
:10C24000A427B33C8988083E7AC09538B93781392C
:10C2500048DEBE3A1F37113CD10D5D3DABAAAA3E68
:10C2600000F0FFFFDFED0A7A9FED0A7ADFED0A6A40
:10C27000A0EE277ADFED097AE7EE007AB7EE007AD2
:10C28000A0EE267A67EE807A87EE870A704700BFB5
:10C290006BD30DBCBA132FBDAEE534BF75AA2A3ED1
:10C2A00010EE102A08B522F00043B3F17E5FB0EE25
:10C2B000406A12D319BF76EE467A9FED1F7ADFED02
:10C2C0001F7A9FED1F7A12BF87EE276AE0EE077A8A
:10C2D000B0EE676AB0EE460A08BDB3F17C5F0BD2E0
:10C2E000A3F50003B3F1645FF4D320EE000AFFF777
:10C2F000B9FFA6EE006AEDE7B0EEC06AB7EE000A3D
:10C3000030EE466AB6EE000A26EE000AB1EEC06ACA
:10C31000FFF7A8FF002AF0EE007AA0EE066A9FED74
:10C32000090AA6EE270A9FED066A36EE406AB8BFF4
:10C33000B1EE466ACEE700BF0000000000008003B7
:10C34000DA0FC93F6821A2B308B510EE103A23F006
:10C350000042B2F17E5FF0EE405A10D308D19FED5B
:10C36000300A9FED306A002BA8BFB0EE460A08BD28
:10C3700070EE405ADFED2B7A87EEA50AF7E7B2F1AF
:10C380007C5F11D2B2F14A5F9FED276A44D920EE5B
:10C39000000AFFF767FFDFED257AE0EE657A35EEFC
:10C3A000E70A36EE400AE2E7002BB7EE000AF6EEA7
:10C3B000007A14DA35EE800A20EE270AF1EEC05A30
:10C3C000FFF750FF9FED1A6AA0EE256A9FED160A4F
:10C3D00075EE865A30EE650A30EE000AC7E730EE99
:10C3E000650A20EE270AB1EEC05AB0EE407A15EE8B
:10C3F000103A23F47F6323F00F0306EE103AA6EE03
:10C40000467A75EE067AC7EE275AFFF72BFFE0EE65
:10C41000055A36EE250ADFE7B0EE460AA7E700BF69
:10C42000DA0F494000000000DA0FC93F6821A2334B
:10C430006821A2B310EE102A22F00043B3F1994F05
:10C4400082B04FEAD2700ED3B4EE400AF1EE10FA89
:10C4500007D69FED410ADFED417A002808BFB0EE14
:10C46000670A02B070473E498B420BD8B3F1665F52
:10C470005AD212F0FF4FF4D160EE007ACDED017A7E
:10C48000019BEEE7374A9342F0EEC07A37D8A2F527
:10C49000D002934229D8F0EE006ABFEE007AA7EEF0
:10C4A000A67A002377EEA67A87EE270A5A1C60EE5A
:10C4B000006A9FED2D6ADFED2D7ADFED2D5A26EE15
:10C4C000A67AE7EE067A9FED2B6AA7EE876ADFED84
:10C4D0002A7AE7EE257A67EE877AE6EE267A60EE2C
:10C4E000277A24D130EE670ABBE7B7EE007A77EE01
:10C4F000C76A77EE877A012386EEA70AD6E71F4A36
:10C5000093420BD8F7EE086AB7EE007AA7EEA67A48
:10C51000022337EEE66A86EE070AC7E7BFEE007A27
:10C5200087EE270A0323C1E74FF0FF33BEE7144A23
:10C53000144902EB830201EB830393ED007A77EE5B
:10C54000C77A37EEC00AD2ED007A37EEC00A00286B
:10C5500087D0B1EE400A84E7DA0FC9BFDA0FC93FCE
:10C56000FFFFDF3EFFFF973F25AC7C3D0DF5113E01
:10C570004712DABDA9AAAA3E98CA4CBEFFFF1B40CB
:10C58000F4990600049A060070B510EE105A25F0D2
:10C5900000440123B4F1FF4FB0EE403A0646036079
:10C5A00004DB60EE003AB0EE630A70BD34B9DFED33
:10C5B000CA7AB7EE007AC7EE273AF4E7B4F1E45F3F
:10C5C0000BDA002DBEBF4FF0FF330360B1EE400A1F
:10C5D000FFF77CFBF1EE403AE5E7002D80F2C082E8
:10C5E000B4F1964FE3DAB4F17A5F9FEDBC5A78DA92
:10C5F000DFEDB90A20EE050A0020FFF7ADFCF0EEF2
:10C60000403AF5EE403AF1EE10FAD0D023EE230A8C
:10C61000B0EEC00A85EE000AFFF758FBF5EEC03A0F
:10C62000F1EE10FA4CBF4FF0FF330123B4F17E5FFF
:10C63000F0EE402A336000F08D82B4F1804FB1EE0D
:10C64000433A00F087826B0000F1D281A44B9C42F8
:10C6500000F3F380B0EE430AFFF738FBA14B9C4296
:10C66000F1EE407A40F39B80F7EE003A33EEC33AA6
:10C6700023EE037ADFED9C6A9FED9C6ADFED9C3A26
:10C68000A7EE266ADFED9B6AE6EE076A9FED9A6ADF
:10C69000A6EE876ADFED996AE6EE076A9FED986A73
:10C6A000E6EE873ADFED976AE7EE066A9FED966A57
:10C6B000A6EE876ADFED956AE6EE076A9FED946A5B
:10C6C000A6EE876ADFED936AE6EE076A63EE833AC9
:10C6D000E6EE873AB6EE007AE3EE473A73EEA73A13
:10C6E000F5E1B1EE407AB0EE470AFFF7B7FBB4EEE2
:10C6F000407AF1EE10FA19D0B6EE000A27EE007A71
:10C70000B0EE470AFFF7AAFB37EE400A30EE000A08
:10C71000F0EE407AFEEECF7A17EE903A062B39D83B
:10C72000DFE803F02312121F1F2B2B00DFED7A7AB4
:10C7300077EEC37A17EE903A03F0010307EE903AD2
:10C740009B00B8EEE70AE9E7F6EE007A37EEC00A9A
:10C75000DFED610A20EE050AFFF746FCF1EE403AF4
:10C760004FE7F7EE007A37EEC00ADFED5B0A20EE06
:10C77000050A0020FFF7F0FBF0E7F7EE087A30EE4D
:10C78000670ADFED550A20EE050AFFF72DFCB1EE32
:10C79000400AE3E7F0EE007A30EE670AE5E75F4B28
:10C7A0009C4264DDDFED5E3A73EE633A63EEA34ACA
:10C7B0009FED5C6ADFED5C6ADFED5C5A9FED5C5AD1
:10C7C0009FED5C0A24EEA37AE7EE066A9FED5A6AB3
:10C7D000A6EE876ADFED596AE6EE076A9FED586AB2
:10C7E000A6EE876ADFED576AE7EE265ADFED566A56
:10C7F000E5EE876ADFED555AE6EE875ADFED546ABB
:10C80000E5EE876ADFED535AA7EE255ADFED525A5F
:10C81000E5EE075A9FED515AA5EE875ADFED505AC3
:10C82000E5EE075AE5EEA36ADFED4E3AE6EEC73ACB
:10C83000D4EE863A73EEC03A50E74B4B9C4206DD8D
:10C84000F0EE003A33EEC33ADFED237A10E7474BC0
:10C850009C4206DDDFED463ADFED1F7A73EE633A68
:10C86000A4E7F7EE007A33EE673ADFED1B7ADFEDEF
:10C87000416A9FED417A9FED416AA3EE267ADFED92
:10C88000406AE7EE036A9FED3F7AA6EE837ADFED1A
:10C890003E6AE7EE036A9FED487AA6EE837ADFED03
:10C8A0003B6AE3EE066A9FED3A6AA6EE836ADFED25
:10C8B000396AE6EE036A9FED386AA6EE836AF7EE00
:10C8C000006AE6EE036A27EE037AC7EE263ABEEE6A
:10C8D000007AE3EE073A01E700000000DB0F494071
:10C8E0006666663F1F4A3B3FA283D3376797673927
:10C8F0003F239E3DA1549C3A7E02F23B01F0893DCC
:10C90000752C3C384584E23834B6053AC66E3D3B5A
:10C910001599A83C661AA53E0000004B07336D3EF2
:10C920000C5BEC3E6B7BA53976F4B7BA67F8663AD8
:10C9300085300DBACDCDF83D07E7C73B474D06BD65
:10C940005EB9F73E27F9A3B9FE7771BB3D37933C3B
:10C950003C2117BEF7E9AF399916143BFEFC28BC01
:10C96000155A843D521CE63117A6DD3F1FA69D3F98
:10C97000C316BB3F5E3C5B3C78756A3EDBD5523BE1
:10C98000B24B7A3FE73ABA3FF400223FAF72D53D4F
:10C99000DFEF443F2D390840BE2E1D4067FF0538AC
:10C9A000B435F13ABDD7F536E440DA3CE6DC153E65
:10C9B0007ACCA63E5A245C3E3F239EBDD6EE4B3A2F
:10C9C00054BF983C6E0F303EC5D0383F3B2DB23F30
:10C9D000E8C4D5BAD23D5B3A1D7FD63E5C061CBA90
:10C9E000FD0C503A610B36BBABAAAA3D000000001B
:10C9F000B4F1824FB7EE002A7BDABDEEC36A5FED79
:10CA0000197A1FED197A5FED196AF8EEC63A16EE3B
:10CA1000103A33EE633A033BA3EE277A5FED1E7ABA
:10CA2000E7EE037A1FED1F7AA7EE837A5FED207A97
:10CA3000E7EE037A1FED217AA7EE837A5FED227A83
:10CA4000E7EE037A1FED237AA3EE267A5FED246AE0
:10CA5000E7EE036A1FED257AA6EE837A5FED266A7C
:10CA6000E7EE036A1FED277AA6EE837A67EE837AF4
:10CA7000A7EE032AC7EE823AF6EE007AE3EE273AF3
:10CA8000042B24D8DFE803F0322F2C290300F1EE29
:10CA9000087A33EE270AF1EE047A73EE277A67EE0E
:10CAA000807AB1EE000A33EE000A60EE277AB0EE2B
:10CAB000080A33EE000A20EE270AF0EE007A33EE81
:10CAC000273A23EE000AFFF701F973EE803A002DB2
:10CAD000BFF669AD72EEE33A65E5B7EE000ADAE754
:10CAE000F7EE007ADDE7F7EE007AE0E7B7EE000A4E
:10CAF000E3E7B0EE430AFFF7E9F8B4F1B94F30EEDF
:10CB0000420A24DA82EE037A1FED4F6A5FED4F6A24
:10CB10005FED4F3A67EE077AE7EE866A1FED516ADE
:10CB2000A6EEA76A5FED526AE6EE276A1FED536A2A
:10CB3000A6EEA76A5FED546AE6EE276AF6EE007A83
:10CB4000E6EE873A33EE673AE3EE003ABFE763EE8C
:10CB5000003ABCE75FED5B3ABCE75FED5C3A22E58B
:10CB6000B4F17E5FF9D0B4F1804FF6D05FED612A69
:10CB700069E500BF07B501A8FFF706FD03B05DF842
:10CB800004FB422905D1835C00EE103AB8EE400A5E
:10CB90007047622905D1835600EE103AB8EEC00AFC
:10CBA0007047482902D130F81230EDE7682902D1E8
:10CBB00030F91230F0E700EB820090ED000A704788
:10CBC000044B0B60044BC1E901300023CB600846E5
:10CBD000704700BF240C07004564040008B50069D5
:10CBE000FBF768FE80F00100C0B208BDF0B501F0AF
:10CBF0001F014368C1F11F0523FA05F58B4043600F
:10CC000083685E1A002E4FEA550586602CDAC268EA
:10CC1000032AA1EB030129DD04682746631C036096
:10CC200017F8023B1B06C0E90073677843EA074325
:10CC3000E71C43600760A77843EA0723271D43608A
:10CC40000760E47823434360043A20238360C26092
:10CC5000436806F1200223FA02F21543826803FAC0
:10CC600001F11644866041602846F0BD0023436010
:10CC7000144647684CB9C2F10303DB0007FA03F31B
:10CC8000D200C0E902244360E2E7036803F1010C2B
:10CC9000C0F800C01B783B431B02013C4360E8E73F
:10CCA000F0B510B94FF0FF30F0BD0368002BF9D09C
:10CCB0000A78FF2AF6D14C7804F0E002E02AF1D19C
:10CCC000E20814F0180F1ABFD24302F00102022248
:10CCD0001A704C78C4F34104C4F104045C604D78CC
:10CCE000ED4305F001059D608F783F09DF608E7888
:10CCF000C6F381061E618D78C5F340055D618D78B0
:10CD000005F001059D61CD78AD091D7791F803C04F
:10CD1000CCF3011CC3F820C091F803C0CCF3C00CC5
:10CD2000C3F824C091F803C0CCF3800CC3F828C02A
:10CD300091F803C0032E0CF0030CC3F82CC0B1D043
:10CD4000042CAFD00F2FADD0DE2454434A2212FB67
:10CD50000642384E012D16445E6303D00022032D97
:10CD60001A6262D00222C0F8BC271A781C6902EB52
:10CD700042022244304C54F82220C0F8C0271A78CE
:10CD8000002A0CBF02250125C0F8C4571A785C6838
:10CD900002EB4202013C2244284C34F9122092FB5F
:10CDA000F5F2C0F8C8275A68C0F8D0271C7880F878
:10CDB000D447DE68002E30D05A68013AC2EB021523
:10CDC0002D2202FB045434441D4D35F814404FF419
:10CDD0007A7514FB05F4C0F8B8471D691C78C5EBDB
:10CDE000051502FB0452DD682A44164D35F9122060
:10CDF0001D7F6400032D18BF0134134D35F9144015
:10CE00005D69121B9C68002C18BF0224043A121B97
:10CE1000002D18BF0132C0F8CC279A683AB18A8831
:10CE200052BA92B21A6306203EE701229BE71A63C8
:10CE3000042039E7C692070090920700B4920700D9
:10CE40001C6807006C950700609507002DE9F04FFE
:10CE500087B0CDE90323109B052B8C4600F3078395
:10CE6000C3F1060E00F17C01031F53F8042F42FAB0
:10CE70000EF299421A60F8D1C56F0368D0E90F1419
:10CE80005A195B1B7D4D85FB03630D195B00091B64
:10CE90007B4C84FB0161541904604901794C521B9D
:10CEA00084FB02525200C2635A1802645B1A84FB6C
:10CEB00003235B00856FC3674368816B446C5A1919
:10CEC0005B1B714D85FB03630D195B00091B6F4CE8
:10CED00084FB016154194460C9006D4C521B84FBF2
:10CEE0000252520082635A1842645B1A84FB032385
:10CEF0005B00456F83678368416B846C5A195B1BC9
:10CF0000644D85FB03630D195B00091B624C84FBB8
:10CF1000016154198460C900604C521B84FB0252A9
:10CF2000520042635A1882645B1A84FB03235B003D
:10CF3000056F4367C368016BC46C5A195B1B584D7E
:10CF400085FB03630D195B00091B564C84FB0161D3
:10CF50005419C4608900544C521B84FB0252520085
:10CF600002635A18C2645B1A84FB03235B00C56E1C
:10CF700003670369C16A046D5A195B1B4B4D85FB3E
:10CF800003630D195B00091B494C84FB01615419B3
:10CF900004618900474C521B84FB02525200C2625A
:10CFA0005A1802655B1A84FB03235B00856EC36617
:10CFB0004369816A446D5A195B1B3F4D85FB0363CE
:10CFC0000D195B00091B3D4C84FB01615419446140
:10CFD00049003B4C521B84FB0252920082625A1859
:10CFE00042655B1A84FB03239B00456E836683695D
:10CFF000416A846D5A195B1B324D85FB03630D1921
:10D000005B00091B304C84FB0161541984614900A9
:10D010002E4C521B84FB0252920042625A188265C7
:10D020005B1A84FB03239B00056E4366C369016A98
:10D03000C46D5A195B1B264D85FB03630D195B00FC
:10D04000091B244C84FB01615419C4614900224C22
:10D05000521B84FB0252120102625A18C2655B1A0B
:10D0600084FB03231B0103661C4FDFF874B000F13F
:10D07000A00300F12002059334E000BF51C2134029
:10D08000FB22855172464F40BD45B340CF200B6D0A
:10D09000103CE1426D2DFA419057D941449F91488F
:10D0A0002134F943968DFC5E630ECB52C41BCC46F3
:10D0B000971AD84A2E40E264F09C9D4AB31D7D7CAD
:10D0C000A924E2431137AE4F26CF6F6BC1923C6E5D
:10D0D000A71E6056EBF64C5F044E9E512CBB06001B
:10D0E0009A79825A52F8203C52F8044C3E6E191933
:10D0F00052E905851B1B86FB034308EB05067C6E86
:10D100005B00A8EB050884FB08584FEAC804BD6E15
:10D1100001EB0608891B85FB01611E19490000917E
:10D1200001961B1B85FB03435B0052F8089C02938E
:10D1300052F81C3C52F8185C52F80C6CF96E03EB78
:10D140000904A3EB090381FB039305EB0609396F7F
:10D150005B00AD1B81FB05A504EB0906D7F874A0A5
:10D160006D00A4EB09048AFB049403EB0509A400F9
:10D170005B1B8AFB03539B00A8EB06058BFB05A5F5
:10D180000099A1EB040A8BFB0A1A4FEA4A0142F804
:10D19000141C0099214401EB4A0142F8181C019922
:10D1A00046446D0042F8206C42F81C5CA1EB09017A
:10D1B0008BFB0141029C029D1C444900EB1A8BFB36
:10D1C0000353019E04EB43045D00B14401EB4303B0
:10D1D00042F80C3C09EB0406059B42F8106C0C4429
:10D1E00042E902452032934207F118077FF47AAFF3
:10D1F000DDE903329C1A002A04F0070404F5806478
:10D2000014BF4FF000084FF4885808EB84050CEB6E
:10D21000050703683B624CF80530039B466814BF62
:10D220004FF48852002202EB83020CEB02031E62D1
:10D230004CF80260466E426F3244466C1644C3F8A6
:10D240002061C3F80061416B466A0E44C3F8206256
:10D25000C3F80062416D0A44C3F82023C3F80023D9
:10D26000466FC26E32444669C3F82064C3F8006456
:10D27000466D1644C3F82065C3F80065C16A466B65
:10D280000E44C3F82066C3F80066C16C0A44C3F8B4
:10D290002027C3F80027C66EC26F3244C668C3F8A1
:10D2A0002068C3F80068C66C1644C3F82069C3F848
:10D2B0000069C16BC66A0E44C3F8206AC3F8006AED
:10D2C000C16D0A44C3F8202BC3F8002BC269C66F96
:10D2D000C3F8202CC3F8002CC26D3244C3F8202DB3
:10D2E000C3F8002DC26BC3F8202EA5F57C61C3F8EE
:10D2F000002EC3F8206F0CEB0102C3F8006F4468E6
:10D3000014624CF80140446E816F466C21440E4417
:10D31000C2F82061C2F80061466A846B3444C2F8E6
:10D320002042C2F80042866D3144C2F82013C2F890
:10D3300000138169C2F82014C2F80014846F816E52
:10D34000866D21440E44C2F82065C2F80065866BE4
:10D35000846A3444C2F82046C2F80046866C3144E0
:10D36000C2F82017C2F800178168C2F82018C2F866
:10D370000018846E016F866C21440E44C2F8206947
:10D38000C2F80069866A046B3444C2F8204AC2F8C5
:10D39000004A066D3144C2F8201BC2F8001B016927
:10D3A000C2F8201CC2F8001C046F016E066D2144F7
:10D3B0000E44C2F8206DC2F8006D046A066B344456
:10D3C000C2F8204EC2F8004E046C2144C2F8201F5F
:10D3D000C2F8001FBEF1000F46D05CF80510CEF178
:10D3E0001F044FF0004041FA04F820FA0EF0CE1767
:10D3F000B8EBE17F00F1FF3018BF80EA060101FAC7
:10D400000EF139624CF8051003F1200503F5815344
:10D4100055F8201C41FA04F7B7EBE17F4FEAE176BB
:10D4200018BF80EA060101FA0EF1296045F8201CB8
:10D4300005F58075AB42EBD102F1200102F5815276
:10D4400051F8203C43FA04F6B6EBE37F4FEAE3756C
:10D4500018BF80EA050303FA0EF30B6041F8203C85
:10D4600001F580718A42EBD107B0BDE8F08F4FF033
:10D47000000E01E538B10023002801DA1846704794
:10D4800001334000F8E72023F8E700002DE9F04FD2
:10D490000446594D5948DFF89091884603F003013E
:10D4A0009B1089B01F2B05EB81159C4650F821106D
:10D4B0000291A8BF4FF01F0C1C2B1946A8BF1C21BE
:10D4C0006E68033121EAE1710E410596AE680E41A6
:10D4D0000696EE68002046FA01F104EB8202049001
:10D4E00007910392019054F8046B454A164226F0C6
:10D4F000004114D108AA02EB810151F8102C0199C6
:10D50000002E41EA0201B8BF524248F8042B039AA8
:10D510000191A242E7D1019809B0BDE8F08F394AE4
:10D5200016420AD1002B55F82110BABFCCF10002E7
:10D5300001FA02F241FA0CF2E1E7334A164214D141
:10D540001039324A029F52F8212082FB0717ACF1B2
:10D55000030100294DDA49426FF0004242FA01FE10
:10D56000BE45CCDB07FA01F2C9E74A04B2F1006F0D
:10D57000B6BF4A0500210421B2F1005FBCBF920092
:10D580000231234F2348B2F1804FBCBF520001311A
:10D59000BA42214FC8BF38468346204F2048D4BFE7
:10D5A000BE4686469246584680FB0ABADEF80470AC
:10D5B0005744924687FB0ABADEF8087057449246F1
:10D5C00087FB0ABADEF80C70574487FB02A2DEF82C
:10D5D00010703A4459F8217082FB07E74FEAC70EF2
:10D5E000029F8EFB07270F4A52F82110ACEB010176
:10D5F000AFE747FA01F282E760180700501707000B
:10D60000FCFFFF7FF0FFFF7FC0FFFF7FA017070039
:10D610009979825AA9BDA029632185101C1707009A
:10D620000817070060170700801707002DE9F74F5C
:10D630000368816982680469066AD0F80CC05B1AC5
:10D640000193C1694369591A131BA3EB060B02EB43
:10D65000040E364B83FB0C5C45684769EF1BC569BC
:10D660007F1B83FB0757324DF04685FB0838314B53
:10D67000324483FB0292361B85FB0646744683FBCD
:10D680000454DFF8B4A08E468AFB0E3E4368C56999
:10D69000DFF8A8902B4489FB035345680093436946
:10D6A0001D448AFB053589FB01A1036899468369FE
:10D6B00009EB630A019B0AEB4C09AAEB4C0C03EB48
:10D6C0006B0A009B520002EB48025B00490003EB2F
:10D6D0004E0EC1EB450509EB020171446400C4EB39
:10D6E000460601600AEB470141600CEB0601941904
:10D6F0002944A5EB0E038160ACEB0401C91AC1609B
:10D700000199A9EB04044E446244A1EB0B011C44B3
:10D71000751BAAEB4707A2EB0E020161446185610C
:10D72000C761026203B0BDE8F08F00BFA1EBD96E04
:10D730008BBE0D627E1A3A1649DD4652322E0E7E9F
:10D740002DE9F0410568C4688269436A066BC06BC5
:10D75000DFF87CC0361A9B1BD21AA41A1B1A2D1B89
:10D76000E41A6D1064108CFB027205EB6607AD1BAA
:10D7700007EB4206A7EB42078CFB032304EB600296
:10D780004FEA430CDFF84CE002EB43038EFB0383CC
:10D79000201A9B000C4C84FB00E00C4C8000A2EB98
:10D7A0000C0284FB02C2F4180C602C184C60281A7E
:10D7B00007EB8204F31AA7EB82028C60CA6008614F
:10D7C0004B61BDE8F08100BF9A79825A83FB20212A
:10D7D000A1EBD96E1D75A37B022A2DE9F0415AD128
:10D7E0003B4B826883FB02423A4E846986FB0454B9
:10D7F00022440A60384C426884FB0252374FC569A4
:10D8000087FB05C52A444A60026883FB0252056A09
:10D8100086FB05752A448A60314F026887FB0252F5
:10D82000304D066A85FB06C63244CA604FF060463A
:10D83000426886FB02C2D0F81CC086FB0CEC624436
:10D840000A61826885FB02C2D0F818C087FB0CEC25
:10D8500062444A61426983FB02C28A61026984FBB5
:10D8600002C2CA61C26883FB02420A62C36887FBC4
:10D8700003234B62036986FB03238B62436985FBA9
:10D880000323CB620023C1E91033C1E90E33C1E9A0
:10D890000C33BDE8F081144B902404FB023202F1FA
:10D8A000480C01F144058C3200F1240E50F8043B81
:10D8B00052F804695CF8047B1C4687FB048441F839
:10D8C000044B86FB0343864545F80439EED1E0E777
:10D8D000D8E3CEB8281C310733C3BEB2CD3C410DCE
:10D8E0009A615FC9669EA0F6D08B07002DE9F047CC
:10D8F00002F001028BBB6AB3D0F88020D0F88072AE
:10D90000D0F88063D0F88054D0F88045D0F88016E5
:10D910005242C0F88020D0F880215242C0F88021C5
:10D92000D0F880275242C0F88027D0F880287F4264
:10D93000524276426D4264424942C0F88028C0F8A3
:10D940008072C0F88063C0F88054C0F88045C0F889
:10D9500080161A461046BDE8F0874FF00044DC40C0
:10D96000013C00F51067C3F11F06002A3DD00022DC
:10D9700094469646056845FA06F94FEAE578B9EB0C
:10D98000E57F18BF88EA04059D400560E04685EA0A
:10D99000E578A8EBE578D0F880506D4245FA06FAB4
:10D9A0004FEAE579BAEBE57F18BF89EA04059D40A7
:10D9B000C0F88050F14685EAE579A9EBE5790D6874
:10D9C00048EA090845FA06F9B9EBE57F42EA080298
:10D9D0004FEAE57818BF84EA080500F580709D409D
:10D9E000B84241F8045BC5D1B4E794469646056851
:10D9F00045FA06F94FEAE578B9EBE57F18BF84EA06
:10DA000008059D400560E04685EAE578A8EBE578E5
:10DA1000D0F8805045FA06FA4FEAE579BAEBE57F8F
:10DA200018BF84EA09059D40C0F88050F14685EA98
:10DA3000E579A9EBE5790D6848EA090845FA06F9A0
:10DA4000B9EBE57F42EA08024FEAE57818BF84EABD
:10DA5000080500F580709D40874241F8045BC6D1FF
:10DA600078E730B570B930BD21F813500133D0F8E4
:10DA7000C827D0F8C4475443D0F8BC276243934228
:10DA8000F2DBF0E700231D46F1E7034601390020F1
:10DA9000814202DC4FF0FF30704713F8012BFF2A60
:10DAA00004D11A7802F0E002E02AF5D00130EFE765
:10DAB0002DE9F04F87B000264FF0007C00900A68F7
:10DAC000CB6D64463546C2FB06456FF0730EC3FB53
:10DAD0000E45D1F8DC70D1F8800062463346C0FBB9
:10DAE0000623C7FB0E234FF4557A4868C0FB0A454E
:10DAF000834F886DC0FB0745D1F88400C0FB0A2323
:10DB0000D1F8D800C0FB072341F6D4798868C0FB60
:10DB100009457C4F486DC0FB0745D1F88800C0FB24
:10DB20000923D1F8D400C0FB072346F2B86EC868B9
:10DB3000C0FB0E45744F086DC0FB0745D1F88C0043
:10DB4000C0FB0E23D1F8D000C0FB07236F4F08693C
:10DB5000C0FB07456E4FA046AB46CC6CC4FB078BA1
:10DB60006A48D1F89050D1F8CC40C5FB0023C4FBE3
:10DB700007238F6C486944465D46C0FB0E4545F25D
:10DB80008408C7FB0845D1F8C870D1F89400C0FBE1
:10DB90000E23C7FB08234F6C8869C0FB094540F280
:10DBA0002C7EC7FB0E45D1F8C470D1F89800C0FB9D
:10DBB0000923C7FB0E230F6CC869C0FB0A454FF051
:10DBC000740EC7FB0E45D1F8C070D1F89C00C0FBA5
:10DBD0000A23C7FB0E234FEA946444EA8514009895
:10DBE00004804FEA926242EA831201F58053428038
:10DBF0001B684FF4D07465463246C3FB045201F5EE
:10DC000084536746D3F800E03346CEFB047341F2F9
:10DC1000040451F804E041F67C04CEFB045241F2C6
:10DC2000840E51F80EE0CEFB047341F2080451F863
:10DC300004E049F2FC74CEFB045241F2880E51F824
:10DC40000EE0CEFB047341F20C0451F804E0314CB9
:10DC5000CEFB045241F28C0E51F80EE0CEFB047361
:10DC600041F2100451F804E02B4CCEFB045241F277
:10DC7000900E51F80EE0CEFB047341F2140451F8FB
:10DC800004E06FF0B304CEFB045241F2940E51F85D
:10DC90000EE0CEFB047341F218044FF4127E51F8EB
:10DCA00004801446C8FB0E5441F2980251F80280D9
:10DCB0003A46C8FB0E2341F21C0751F807E06FF00B
:10DCC0001307CEFB075441F29C0E51F80EE0CEFB39
:10DCD00007234FEA956545EA8415A0F840504FEABE
:10DCE000926242EA8312034608330193CDE902C6E9
:10DCF00003464433DFF824E0A0F8422005930FE008
:10DD0000D4F8FFFF7CAFFFFF3CB6FDFF7894040022
:10DD1000C44902004CE803002464FFFF108E070092
:10DD2000DEE91089DDE9024CD1F80001D1F85C315F
:10DD3000C0FB084CDDE90226C0FB0926C9F1000A38
:10DD4000C3FB0A4CC3FB0826DDE90207D1F880B10A
:10DD50000492CBFB0807DDE90235CBFB0935D1F88E
:10DD6000DC21C2FB0A07C2FB0835DEE912B8D1F894
:10DD700004A1D1F85891CAFB0B4C049ACAFB08269F
:10DD8000C8F1000AC9FB0A4CC9FB0B260492D1F862
:10DD9000D891D1F88421C2FB0B07C2FB0835C9FB1F
:10DDA0000A07C9FB0B35DEE914B8D1F808A1D1F890
:10DDB0005491CAFB0B4C049ACAFB0826C8F1000A0E
:10DDC000C9FB0A4CC9FB0B260492D1F8D491D1F8B7
:10DDD0008821C2FB0B07C2FB0835C9FB0A07C9FB38
:10DDE0000B35DEE916B8D1F80CA1D1F85091CAFB79
:10DDF0000B4C049ACAFB0826C8F1000AC9FB0A4C5E
:10DE0000C9FB0B260492D1F8D091D1F88C21C2FB2A
:10DE10000B07C2FB0835C9FB0A07C9FB0B35DEE956
:10DE200018B8D1F810A1D1F84C91CAFB0B4C049A48
:10DE3000CAFB0826C8F1000AC9FB0A4CC9FB0B261D
:10DE40000492D1F8CC91D1F89021C2FB0B07C2FB10
:10DE50000835C9FB0A07C9FB0B35DEE91AB8D1F84A
:10DE600014A1D1F84891CAFB0B4C049ACAFB0826AE
:10DE7000C8F1000AC9FB0A4CC9FB0B260492D1F871
:10DE8000C891D1F89421C2FB0B07C2FB0835C9FB2E
:10DE90000A07C9FB0B35DEE91CB8D1F818A1D1F887
:10DEA0004491CAFB0B4C049ACAFB0826C8F1000A2D
:10DEB000C9FB0A4CC9FB0B260492D1F8C491D1F8D6
:10DEC0009821C2FB0B07C2FB0835C9FB0A07C9FB37
:10DED0000B35DEE91EB8D1F81CA1D1F84091CAFB80
:10DEE0000B4C049ACAFB0826C8F1000AC9FB0A4C6D
:10DEF000C9FB0B260492D1F8C091D1F89C21C2FB3A
:10DF00000B07C2FB0835C9FB0A07C9FB0B354FEAF3
:10DF1000946444EA8C14019A22F8044C4FEA90600D
:10DF200040EA871022F8020C049A4FEA926242EA11
:10DF300086120098A0F87C204FEA936343EA851389
:10DF4000A0F87E30019B059A04330193031F0093D0
:10DF5000019B93420EF1400E01F580717FF4E0AE1B
:10DF600007B0BDE8F08F00BF024B03480022C3F8A2
:10DF7000B8207047D04E0120A8E10600437882788F
:10DF80001B01120202F4E06203F030031343027833
:10DF900002F003021343C278120302F480521343C7
:10DFA0000279120402F4E02213434279120502F4CA
:10DFB000801213438279120602F080721343024AE0
:10DFC000C2F81835704700BF0070004010B5084A0D
:10DFD000002388214FF6FF7001FB03F4A45A84420A
:10DFE00004D10133052BF7D1024810BD0248FCE7EC
:10DFF00010470120A0E10600ACE1060001F06043FB
:10E00000B3F1005F70B502460E4663D10379324D1D
:10E01000242101FB0351496821B100684FF40474C5
:10E02000C0F80843242000FB03539C6954B1D8690D
:10E0300000283FD021B113684FF40472C3F80423C1
:10E04000264836E001219961DE60DC6110684FF4FA
:10E050008871FCF73DF84FF4A2711068FCF738F8AE
:10E0600013680121C3F83465C3F83815136824BB5D
:10E07000196011791368242202FB015252681ABBFD
:10E08000D3F81041D3F84421D3F82461144302D1CA
:10E09000002EF5D02246242303FB0155002310480F
:10E0A000AB61104B002E18BF18460733002A18BF6B
:10E0B000184670BD1E610124C7E7D3F8001241F075
:10E0C0002001C3F80012D4E74FF404720448C3F8E7
:10E0D0000423EEE70448ECE7E84D01200B00AD0B0C
:10E0E0000000AD0B0100AD0B0A00AD0B10B50378BD
:10E0F000012B0C4602D0022B00D010BD4168027AE1
:10E1000004F11000FCF721FA606804F11C01BDE87D
:10E110001040FFF773BF000013B5104B10481B6889
:10E1200000681A680121D1600E4A128892B2002458
:10E1300030F812001A68C2F84041D2F8402101922A
:10E14000019A1A684FF48034C2F804431A68C2F87E
:10E1500040051B68196002B010BD00BFA45101202A
:10E16000385101203C510120B0F5A07F08B524D1E1
:10E17000124B13481B6800881B6801225A60114A21
:10E18000138801339BB2138013889BB2984204D842
:10E19000BDE80840081DFCF7E5BC1388DB0708D480
:10E1A0004B685A681B7AC2F86035BDE80840FFF733
:10E1B000B3BF081DFCF7D6FCF7E708BDA45101204A
:10E1C0003E5101203C51012007B5019001A8FBF709
:10E1D0008FFC019B03F5E073890040F8231003B026
:10E1E0005DF804FB38B505460C460846FCF762FBB3
:10E1F0006C6020790021FFF7E7FF002038BD01297E
:10E2000006D08B1E5942594143681879FFF7DCBF8D
:10E210000321F9E710B5436802460C46187900213E
:10E22000FFF7D2FF21461046BDE81040FFF7E7BFD9
:10E230002DE9F34105793A4E24236B43F2180C463D
:10E24000517F8046002968D1F3580BB101235377E1
:10E2500094E80F00242707FB056707F10C0C8CE8F6
:10E260000F0097F82000FF2805D0BB7F1BB9FB7F6C
:10E27000C3B1FBF765FC226822B102F06043B3F141
:10E28000005F06D1A36883B103F06043B3F1005F80
:10E290000BD0242303FB0565224800236B7702B0D3
:10E2A000BDE8F081FBF759FCE5E7D8F8003061687C
:10E2B000C3F84425C3F84815D4E90212C3F834154D
:10E2C000C3F838250022C3F81821D3F8181101919A
:10E2D0000199C3F85025C3F8402501221A61242270
:10E2E0006A43B258AAB9D3F81821002AFBD02423D4
:10E2F00003FB056595F82000FF2805D0AB7F1BB90F
:10E30000EB7F1BB1FBF729FC0748C8E7FBF718FCBC
:10E31000FAE74022C3F80423F6E70448BFE700BF4A
:10E32000204D01200A00AD0B0000AD0B0B00AD0B22
:10E3300000F1804382B01A68002A14BF0120002037
:10E3400004D000221A601B680193019B02B0704741
:10E3500010B54FF08043D3F80443620707D54FF45C
:10E360008470FFF7E5FF10B11E4B1B689847A306AA
:10E3700008D54FF48A70FFF7DBFF18B11A4B002065
:10E380001B689847600608D54FF48C70FFF7D0FFE4
:10E3900018B1154B01201B689847210608D54FF48A
:10E3A0008E70FFF7C5FF18B1104B00201B6898470F
:10E3B000E20508D54FF49070FFF7BAFF18B10B4B88
:10E3C00001201B689847A3050AD54FF49270FFF708
:10E3D000AFFF28B1054BBDE810401B68022018476D
:10E3E00010BD00BFBC4E0120C04E0120C44E012014
:10E3F00040F20110814209D112F001000AD0064B0F
:10E40000D88980B2003818BF0120704716221A60E0
:10E410004FF0FF30704700BFA032012040F20110E2
:10E4200081420BD112F004000CD0074B587848B150
:10E430009B78002B0CBF00200420704716221A6026
:10E440004FF0FF30704700BFA032012008B5074BE6
:10E45000D3F80630B3F5966F06D14FF080434E22C5
:10E46000C3F81C25FAF744FF08BD00BF742601203D
:10E4700010B58478182104F07F030C22E409594375
:10E4800002FB0411114A0A44017911720122104958
:10E4900002FA03F07CB90C3302FA03F3C1F8043337
:10E4A000D1F814350343C1F81435BFF36F8FBFF3B0
:10E4B0004F8F012010BD023302FA03F3C1F8043379
:10E4C000D1F810350343C1F81035EEE7382F01209D
:10E4D000007002402DE9F843DDE908890C46164634
:10E4E0001F460025AE4201DC01200EE06378052BBB
:10E4F00004D1E37803F00303BB4208D00D4B186846
:10E5000010F0010001D000BE0020BDE8F8832046D5
:10E51000FFF7AEFF18B9BDE8F843FAF757BFA37885
:10E52000DA0914BF89F8003088F800302378013503
:10E530001C44D7E7F0ED00E0C208054900F00700F1
:10E5400001238340885C20EA03008854704700BFA1
:10E55000854E012038B5144C0546FBF765FE62195F
:10E5600092F9243092F82420072A9FBF0F4A03F51E
:10E57000A273002142F8231004EBD50305F0070233
:10E5800093F85530D340DB0705D52846FBF7CAFA88
:10E590002846FFF7D1FF2C4494F82400FBF736FE01
:10E5A000FF2384F8243038BD304E01200060004045
:10E5B00010B504460079FF281AD00E4B617900226D
:10E5C00043F8202043F82120FBF72EFE6079FBF76B
:10E5D0002BFE2079FFF7BEFF6079FFF7BBFF2079A4
:10E5E000FCF7ECF86079FCF7E9F84FF6FF73A380CD
:10E5F00010BD00BFBC44012008B5FFF7D9FF01489A
:10E6000008BD00BFA8E1060008B50868FFF7D0FF05
:10E61000004808BDA8E1060037B5204C2518024681
:10E6200095F92410072913DD214491F84C309B09FA
:10E63000032B09D1FBF7DBFD40B10321104603B0EA
:10E64000BDE83040FBF7C0BD012BF6D10221F5E754
:10E65000CBB2072B1FD88A0002F1804202F5C042DC
:10E660009B00D2F8100503F1804303F5C24340F04C
:10E670000100C2F8100500221A601B680193019B7B
:10E6800095F9243054F823302BB1012303FA01F11A
:10E69000034BC3F8041303B030BD00BF304E01205C
:10E6A00000600040044B054A5B8B05489BB2002B81
:10E6B00018BF1046704700BF74260120ACE1060069
:10E6C000A0E1060038B50C464942F9F773FC022177
:10E6D000F9F7F1FB5C230370447038BD73B50C4649
:10E6E00001210646F9F766FC04F110033F2B06D81A
:10E6F000A4F18001C9B2F9F7EDFB02B070BD14219D
:10E700000DF10505F9F7E6FB294604F07F00E3B2B9
:10E71000E4112A4605F8010D601C0128F5D80134E2
:10E7200003F0400312D11BB97F2305F8013C951E6D
:10E73000491B3046F9F7BFFB01AC01462B46A3420B
:10E7400008D15D1B9DF804204255D6E7002BEFD081
:10E750000023EAE713F8012B62F07F0201F8012B96
:10E76000EDE700000369272B2BD0222B29D0A3F142
:10E77000620113291ED8174ACA40D2071AD5426926
:10E78000272A1ED0222A1CD0722B1CD1662A06D121
:10E790008269272A15D0222A13D0722B15D14369FA
:10E7A000622B0CD1806927280BD0A0F1220358429C
:10E7B00058417047662BF0D14269722AE8D0002098
:10E7C000704701207047662BF6D0622BF7D1436962
:10E7D000722BE6E7110009002DE9F84F90F82E3072
:10E7E000468D934FDFF85082DA0748BF0162054635
:10E7F00048BF00F11801013E731C02D10846BDE874
:10E80000F88F6B6853F8364014F0030E11D123686B
:10E81000884A934240F0038194F85130B4F938C0EB
:10E82000B4F93C009B0706D0844502D0216404F172
:10E830003801013EE0E794F850305A0733D584455B
:10E8400031D0B4F94430B4F946209C45A8BF9C4669
:10E85000B4F94830A4F82CC09842B8BF1846B4F9AF
:10E860003A3020869342A8BF1346E385B4F94A2084
:10E87000B4F93E309342B8BF134604F12C096386C5
:10E880004846FCF7EEFE228A638A5343B0EB430FFF
:10E8900002D861634946CCE704F138032164E3649C
:10E8A00004F14401C5E76268930724D1DFF88C9135
:10E8B00013684B451FD1B2F91430B2F9189099453D
:10E8C00019D002F114094945D16114D0B4F8169059
:10E8D000B9F1010F29D1A385B2F91630E385B2F958
:10E8E00018302386B2F91A30638694F8503043F01A
:10E8F000010384F8503094F850309A071AD4A26873
:10E9000012F0030904D11368434516D192F80CE0C4
:10E9100094F850306EF3410384F85030DAB29B071C
:10E9200001D484450BD1E164BAE794F8503043F048
:10E930000203DEE74FF0010EEAE7CE46E8E7D20732
:10E940007FF577AFB4F90C00B4F92C90B4F930C06E
:10E95000A36AB4F90EB0B4F92E2093F904E0B3F829
:10E9600000A081448444B4F932005A44584493F8D6
:10E970000EB01FFA8EFE1FFA89F992B21FFA8CFCB4
:10E9800080B2BBF1000F2ED01EFB02A2A28593F92C
:10E9900005E01EFB09F9B3F802E0F144A4F82E905B
:10E9A00093F9042012FB00F01A881044208693F992
:10E9B00005205B8812FB0CFC9C44A4F832C0B4F91F
:10E9C0003230B4F92E2061639342BCBF6286E38586
:10E9D000B4F92C20B4F930309342BCBF2286A38511
:10E9E00004F12C0125E71EFB09AEA4F82CE093F9F5
:10E9F00005E01EFB02F2B3F802E07244E28593F9EF
:10EA0000042012FB0CFC1A889444A4F830C093F93B
:10EA100005205B8812FB00F018446086CFE7BB42FC
:10EA20007FF407AF2046FFF7D7FE014601E700BF9E
:10EA300034C5060058C9060040C70600A0C006003D
:10EA400070B5084D084E642445F00105336833B9AC
:10EA50004FF42070A847013CF8D1044870BD044829
:10EA6000FCE700BF10BC0600009102400700AD0BA0
:10EA70000000AD0BF8B53C4B5B791446054603F03E
:10EA8000FF02002B6ED1394E326019B34378023B3E
:10EA9000072B1FD8DFE803F0545250114E4C4A04A4
:10EAA000CB791B068A7943EA02434A7943EA022377
:10EAB0000A7913432E4AC2F83C36CB781B068A7873
:10EAC00043EA02434A7843EA02230A781343284A76
:10EAD000C2F83836264F0123C7F80833AB786A7876
:10EAE0001B0343EA02232A781343EA7843EA4233BA
:10EAF0002A7943EA82336A7943EAC233C7F8343663
:10EB0000FFF79EFF1B4B98422DD0002333603CB390
:10EB10006978D7F83C26D7F83836023907291FD844
:10EB2000DFE801F01D1B1917161412100023B9E7B6
:10EB30000023BAE70023BBE70023C0E70023C1E7B7
:10EB40000023C2E7110EE171110CA171110A61716C
:10EB500022711A0EE2701A0CA2701A0A62702370E7
:10EB6000054800E00548F8BD984E0120009102409C
:10EB7000009002400700AD0B0000AD0B0B00AD0B89
:10EB800007B5012300228DF800008DF801301146F1
:10EB900040F201136846ADF80230ADF80420FFF7EB
:10EBA00069FF034BC31A5842584103B05DF804FB98
:10EBB0000000AD0B07B540F20113ADF80230013291
:10EBC00000238DF800008DF8012068460A4619469A
:10EBD000ADF80430FFF74EFF034BC31A58425841BB
:10EBE00003B05DF804FB00BF0000AD0B07B50023C8
:10EBF0008DF80430012201A90520FFF7DBFF18B1D1
:10EC00009DF804309B07F5D103B05DF804FB0000CC
:10EC100007B501328DF800008DF8012040F2011394
:10EC200000226846ADF80230ADF80420FFF722FF5D
:10EC3000034BC31A5842584103B05DF804FB00BFB0
:10EC40000000AD0B0120704770470000004870477E
:10EC5000A8E1060040F20110814217BF162202F01F
:10EC600004001A604FF0FF307047000004288B68E2
:10EC700003D0052808D000207047064A06489BB2FA
:10EC8000002B08BF10467047044800EA430040F0DC
:10EC900001007047A0E10600ACE10600FEFF0100A4
:10ECA0008088400040F001007047C088400040F07C
:10ECB000010070472DE9F041164FDFF85C800646F1
:10ECC0000C460025738D9D4201D3BDE8F081736829
:10ECD00053F83500820708D10368BB4207D190F88A
:10ECE000513064F3410380F851300135EAE7434580
:10ECF000FBD190F82E30C3F3C002A242F5D064F3EA
:10ED0000C30380F82E305B07EFD42146FFF7D2FF14
:10ED1000EBE700BF58C9060034C50600004870473D
:10ED2000A8E1060000487047A8E106008068704727
:10ED30000079400040F0010070470000F0B58BB052
:10ED40006846F8F75DF90F4B0F4D1F680F4C104EDA
:10ED50002D1A07F5806001212844FAF729FE20606A
:10ED600070B9012105F5C840FAF722FE4FF4C043FF
:10ED7000206033602368074A1B681A600BB0F0BD3F
:10ED80003760F7E73C220120000004208C5101206D
:10ED9000CC490120EF29780110B50A4C206840B118
:10EDA000094B1A68094B1B689A4203D10368084A49
:10EDB0001A6010BDFAF79CFD00232360BDE81040E7
:10EDC000FFF7BCBF8C5101203C220120CC4901201F
:10EDD000EF2978010B6802480022C3E9012270473D
:10EDE000A8E106000B68024800225A60704700BF85
:10EDF000A8E106000E4B1A78C2F34000920716D520
:10EE00001A78510712D40B4A507880B100F07F0273
:10EE100003EB420303EBD01320335A78D20705D417
:10EE20005878C0F3400080F0010070470020704720
:10EE3000BC450120FC2F012008B5FBF7D1FC01489F
:10EE400008BD00BFA8E1060008B50868FBF7C8FCCC
:10EE5000004808BDA8E106000B68024800225A607D
:10EE6000DA607047A8E1060010B58368044643B134
:10EE70000430FBF7B5FC04F10C00BDE81040FBF7D3
:10EE8000AFBC10BD08B50868FFF7EEFF004808BD2D
:10EE9000A8E1060008B5FFF7E7FF014808BD00BF7D
:10EEA000A8E1060008B50868C36813B10430FCF790
:10EEB000A2F9014808BD00BFA8E1060010B58368AB
:10EEC0000446A3B10430FBF78BFC94F820309A077A
:10EED00003D504F10C00FBF783FC94F82030DB072A
:10EEE00005D504F11400BDE81040FBF779BC10BD56
:10EEF00008B50868FFF7E2FF004808BDA8E1060072
:10EF000008B5FFF7DBFF014808BD00BFA8E1060018
:10EF100043681A7A12B901201872704700207047AE
:10EF200041680A7A2AB901230B72416818460A72AD
:10EF300070470020704741680A7A2AB901230B7292
:10EF4000416818460A72704700207047084B03EB6F
:10EF5000411310B41C691CB95DF8044BFAF736BABA
:10EF60005969044B1961234611465DF8044B184753
:10EF7000B08C0600242F012008B5074B1B78012B0D
:10EF800002D9012800D0FEE7044B43EA0020044BDD
:10EF90001860FAF7ADF900BFC6490120AF0000AD17
:10EFA000B0510120F8B5284DB5F80832002B47D1F3
:10EFB000002845D0D5F8F810002942D0411A48BFA2
:10EFC0000F314FEA211CD5F8F4004FEADC010CF0B8
:10EFD0000704435C0122A24023EA020343544FEAA0
:10EFE0009C06D5F8EC40A05D374661460CF0030363
:10EFF0004FF0030E5B000EFA03F320EA0303E35520
:10F000000131D5F8EC408F0801F00303E05D5A00B0
:10F0100040FA02F202F00302022AEBD0A1EB0C014B
:10F02000082928BF0821813105EB81014B68B342D3
:10F03000D5F82C3288BF4E60B34238BFC5F82C6279
:10F04000F8BD0820FFF798FFD04E012010B5044608
:10F050004068FBF753F8607FFBF7B0FBA07FFBF73E
:10F06000ADFBFF236377A3772069FFF79BFF0023A6
:10F070006361238310BD000008B50868837FFF2B00
:10F0800001D0FFF7E3FF014808BD00BFA8E106007B
:10F0900008B50220FFF770FF08B50120FFF76CFFED
:10F0A00008B50A20FFF768FF10B5124B1B788BB12B
:10F0B000114B9A686AB1114A127852B9EFF3108075
:10F0C00072B60F491C680C605C684C609A6000B9AD
:10F0D00062B610BD0B4B1A6812B90220FFF74CFF45
:10F0E0001A68013A1A601B68002BF2D1BFF35F8FD8
:10F0F000EEE700BF8A51012020510120E04A0120A3
:10F1000000E100E00451012038B5FBF7EFFB044BB0
:10F11000D3E90045FFF7C8FF2046294638BD00BFA8
:10F120009851012038B505460C46FFF7EDFFC5E9BB
:10F130000001024B9B689B09236038BD10E000E092
:10F14000F0B585B001A9044602A8FFF7EBFF019DC9
:10F15000334BC5F57A700190002153F8042B12B19E
:10F160001679A64246D001310829F6D105B0F0BD86
:10F17000D2E90667029B991B538A548AA4B2A04223
:10F180009BB230D2508AC5F5FA6380B20129A3EB55
:10F19000000305D94FF47A7000FB0133A3F57A73AD
:10F1A0004FF6FE704FF6FF71834288BF0B46D18940
:10F1B000108A948980B210FA81F1B1FBF4F004FB5B
:10F1C0001011906820F81130138A91899BB29942EE
:10F1D0008BBF138AD389013301338BBF9BB29BB2A0
:10F1E0001382D38114E0C31A4FF47A70414311FAA9
:10F1F00083F3D5E7D379002BBAD02046FAF7F7FF8F
:10F200000038537918BF0120834201D00023D37105
:10F21000DDE90201BDF80430C2E906015382A5E729
:10F220009C44012008B5FFF76FFF07EE901AB8EE77
:10F23000677A07EE900ADFED096AF8EE677AE7EE83
:10F24000267A9FED077AC7EE877A17EE900A20F0AC
:10F25000030040F00200A0F1FF4008BD0000804F15
:10F2600000007A4410B50446FFF74EFF2369226F71
:10F27000C11A91429ABF9B18181A002010BD0000B5
:10F2800008B5FFF711FF014808BD00BFA8E106005F
:10F2900008B5114A136913B90620FFF76DFE196806
:10F2A000586011611846C468056946698769D0F8D5
:10F2B0001C80D0F82090D0F824A0D0F828B0D0F846
:10F2C0002CD090ED0C8B90ED0E9B90ED10ABD0F808
:10F2D00008E00120704700BFD04E012008B5024869
:10F2E000F9F7A1FBFFF7D4FF100207008068034A7B
:10F2F000034B002814BF104618467047ACE10600C7
:10F30000A0E106008968806A0909F8F7DBBE000001
:10F31000174B984210B502460C4623D0154B984225
:10F3200023D0C10708D5431000EE103AB8EEC00A4A
:10F3300084ED000A012010BD830707D101680E4B40
:10F34000994203D10430F8F7EDFBF1E71046F9F7E5
:10F350004DFA0028EFD002F1FF4222F0030300EE45
:10F36000103AE5E79FED050AE2E7B7EE000ADFE7AE
:10F37000A0E10600ACE10600800A070000000000E2
:10F3800010B50368044613B14068FFF70BFE204632
:10F39000BDE81040FFF706BE10B5037BDB0704464F
:10F3A00002D48068FFF7FEFD0023A36010BD022990
:10F3B000F8B5044605D0042923D001291CD100202A
:10F3C0002CE05668012E10D0022E10D000201568B7
:10F3D00029182CBF0127002766B1002D0ADA8842C0
:10F3E00038BF0021A1601160E9E78068EFE741685C
:10F3F0004868ECE7002FF5D016221A604FF0FF3076
:10F400000CE0456845B12B7BDB0702D4A868FFF709
:10F41000C9FD2846FFF7C6FD00206060F8BD2DE954
:10F42000F04316468BB0B207DDF848900746984681
:10F430003DD416F0040F0CBF0023202300930A468E
:10F44000139B202102A8F8F7CDFFF30504460DD544
:10F45000431C1F2B0AD80AAA1444252204F8202C86
:10F460000AAA1A44002102F8201C1C4616F0400586
:10F470001FD09DF808302F2B4FF000031BD801221E
:10F4800002A9CDE900323846F8F70CF909F1FF3945
:10F490000546013C0DF10901CDE9008933462246BC
:10F4A0003846F8F7FFF828440BB0BDE8F0832B236B
:10F4B000C4E702A9F0E702A91D46EDE710B504462E
:10F4C00038B18068FFF76EFD2046BDE81040FFF7B9
:10F4D00069BD10BD38B50A4D0A4C286838B1FAF735
:10F4E00007FA00232B600023C4F8C83038BDD4F8D5
:10F4F000F830002BF7D0D4F8C800FFF753FDF2E73F
:10F5000090510120D04E01204069FBF7E5B9837985
:10F51000012B14BF4FF48070202040F00100704791
:10F5200038B5044658B3006808B1FFF73BFD606882
:10F530000025256008B1FFF735FDA068656008B1BA
:10F54000FFF730FDE0680025A56008B1FFF72AFD50
:10F550002069E56008B1FFF725FD60690025256198
:10F5600008B1FFF71FFDA069656108B1FFF71AFD3B
:10F570000023A3612046BDE83840FFF713BD38BD26
:10F5800010B50446406808B1FFF7CAFF0023C4E97C
:10F590000133C4E90533A36210BD000008B5FFF7CD
:10F5A000EFFF014808BD00BFA8E1060008B50868E4
:10F5B000FFF7E6FF004808BDA8E10600154A38B588
:10F5C00000210446042352F8040B844208BF42F889
:10F5D000041C013BF7D1A268C2F80035A07E08B137
:10F5E000FBF7ECF8E07E08B1FBF7E8F8A068002133
:10F5F000FBF7D0F900250221A068FBF7CBF9E06802
:10F60000A560FFF7CFFC2069E560FFF7CBFC256123
:10F6100038BD00BFB446012008B5086883680BB147
:10F62000FFF7CCFF004808BDA8E1060007B5436816
:10F6300001291B79019301A80CBF07220322FAF7C5
:10F6400057FA019B120203F5E07342F0030240F8FF
:10F65000232003B05DF804FB00F01F0301229A4051
:10F6600043099B0003F1604303F56143C3F8802124
:10F670001A6070472DE9F8431D4B1B6807460E467C
:10F68000154693B300239AB2954202D80120BDE8F3
:10F69000F883B25CFF2A03F10103F4D0DFF8548051
:10F6A000DFF854900024FFF7A1FAF0B10620FFF72D
:10F6B00067FAD0B1331903F06042B2F1005F14D1A0
:10F6C0009A0712D13A19C8F81025C8F814354FF422
:10F6D0008073C8F818350820FAF7C8FD484504D1EA
:10F6E00004F58074A542DED8D0E70020CFE700BF44
:10F6F000CC4A0120009002400000AD0B436818790D
:10F7000009B9FAF72ABAFAF71BBA38B504460D4612
:10F710001146FFF78BFF29462046BDE83840FFF72A
:10F72000EDBF38B5044604340D46FBF7DFF820463C
:10F7300001220021FFF7E9FF002D14BF06203C2025
:10F74000FBF7CAF820460021FEF764FD002D14BF28
:10F7500040200A20FBF7C0F8BDE83840FFF7A4BC02
:10F7600001211030FFF7CABF70B51C464B1E59422D
:10F77000594105460830FFF7C1FF049AD5E90D103D
:10F7800023462244934200D170BDC1F80C056C6839
:10F7900013F8016B2670C1F80805F3E708B50021DE
:10F7A0001030FFF7ABFF012008BD000010B50A4B79
:10F7B00082699A420ED000F1180400212046FFF71A
:10F7C0009DFF0420FBF788F820460121FFF796FFF4
:10F7D000012010BD0020FCE7A80007002DE9F04142
:10F7E0002DED028B3B4A836E0126934286B0044680
:10F7F000B0EE408A80F8996012D1DFED377A60EE82
:10F80000277A6830FCEEE77A17EE903A99B2FBF768
:10F81000EAF8002384F8993084ED228A012517E064
:10F820002E4A93420CD1DFED2E7AB4EEE70AF1EEC8
:10F8300010FACCBF012100216830FFF75FFFE8E735
:10F84000B0F88C30B3F5807F08D1002580F899504E
:10F85000284606B0BDEC028BBDE8F08100F1080837
:10F860004046FBF78DFF0546E8B1DFED1E7A94F8C0
:10F87000971094F88C20676AA0688DF8142068EEC1
:10F88000277AFCEEE77ACDED037A9DF80C3081B152
:10F890008DF8153002230093324605AB0021B8479E
:10F8A0004046FBF770FF002384F89930002DCFD03D
:10F8B000B2E78DF81330324605AB00960391B84796
:10F8C0000399676AA06800960A460DF11303314652
:10F8D000E5E700BF001C070000FF7F4778BE060079
:10F8E000A4707D3F00007F4310B5044601211C3009
:10F8F000FFF704FF636800221A7210BD10B50A4BAF
:10F9000042699A420ED000F1140400212046FFF70C
:10F91000F5FE0420FAF7E0FF20460121FFF7EEFE96
:10F92000012010BD0020FCE7A800070007B54368D0
:10F9300001A81B790193FAF7DBF8019B03F5E0734B
:10F9400050F8230000F0010003B05DF804FB000054
:10F95000F7B5374E3318054693F92430002B0F4680
:10F9600064DA8B78C3F34003002B0BBF0824002418
:10F97000092108218C4202D12E4803B0F0BD56F86F
:10F980002400013042D1711946F8242081F8244026
:10F9900013B9331983F84C50BB785A0717D4D807DA
:10F9A00036D501A80195FAF7A3F8019B00EB830077
:10F9B000D0F8003723F00203C0F800371E49EA08E8
:10F9C00005F0070001238340885C03438B54BA7819
:10F9D0003B78910721D5A40004F1804404F5C0448C
:10F9E0002D02D4F8102522F44F3222F44072C4F8CC
:10F9F00010251B04D4F8102505F47C5503F440337E
:10FA00001D431543C4F810550C48B6E70134B1E75F
:10FA100079782846FEF7D8FBD0E7083C344494F8C0
:10FA2000545045EA831384F85430EDE70448A4E7C2
:10FA3000304E01200200AD0B854E01200000AD0BC1
:10FA40000B00AD0B2DE9F743002406460F4600F5E9
:10FA5000A0754FF48038A1462B688BB1D6F80433DB
:10FA600008FA04F21A420BD0C5F800902B680193F3
:10FA7000019BA30003F5A07398B2D7E90031984722
:10FA80000134042C05F10405E6D103B0BDE8F08390
:10FA900001490248FFF7D6BF744D012000A0004085
:10FAA00001490248FFF7CEBF684D01200090004099
:10FAB0007FB50222ADF814203B4A002303210493B2
:10FAC0008DF81630C2F8F0150121C2F8F435C2F8ED
:10FAD000001519461A0102F1804202F5E042013395
:10FAE000082BC2F81415C2F81015F3D104A8FEF7BC
:10FAF00045FA2D4B0922C3F81425C3F810250DF142
:10FB00000202C3F82C260122C3F830261A6003F53E
:10FB100080731A68002AFCD000221A601B680193C7
:10FB2000019B224B01221A6003F580731A68002A98
:10FB3000FCD000221A601B680293029B1C4B01221E
:10FB40001A601C4A1368002BFCD000231360126853
:10FB50000392039A144ADFED186AC2F80035BDF922
:10FB600002209A42B8BFADF80230BDF9023007EE6C
:10FB7000103AB8EEC77AC7EE267A9FED107A67EE94
:10FB8000877AF4EE677AF1EE10FA7DBF17EE903ABD
:10FB900023F0030040F00200094878BFA0F1FF40C5
:10FBA00007B05DF804FB00BF007000400470004027
:10FBB0000870004014710040FFA66A46333353407A
:10FBC000A8E10600044A8B881278DBB29A4201D081
:10FBD000F9F7FCBB01207047FC2F012007B54368F3
:10FBE00002461B79019301A8F9F782FF019B03F5F7
:10FBF000E07350F8233013F0010F536808D11879DF
:10FC0000FAF7F5FA003818BF012003B05DF804FBDD
:10FC10001B79019301A8F9F76BFF019BD0F804054C
:10FC2000D84000F00100F0E738B500F10C040121E4
:10FC30002046FEF7EFFA2046FFF7D0FF01220546E7
:10FC400011462046FFF761FD284638BD10B5044631
:10FC50000434FAF74BFE012200212046FFF755FD40
:10FC60000620FAF739FE00212046FEF7D3FA0620D7
:10FC7000FAF732FE2046FFF7B1FF04463720FAF7C5
:10FC80002BFEFFF711FA204610BD10B504460434D0
:10FC9000FAF72CFE012200212046FFF736FD4FF433
:10FCA000F070FAF719FE00212046FEF7B3FA46205D
:10FCB000FAF712FE2046FFF791FF04464FF4CD708D
:10FCC000FAF70AFEFFF7F0F9204610BDF8B52E4905
:10FCD000D1E90023541C43F10005C1E900452B4B39
:10FCE0001A685AB11A68012A15BF1A68284802F121
:10FCF000FF32027008BF4FF47A721A60254B1A68FF
:10FD00009AB1186801280DD1234A127852B1234ABA
:10FD100012783AB9224A147824B9224C04F13805F1
:10FD2000A56510701A68013A1A60D1E90001002334
:10FD300000F01F02134326D11A4BD3F8B81011B3A9
:10FD400011F003041FD10A68174B9A421BD10E1DF4
:10FD500001F12407012556F8040B38B1FFF73EFFE7
:10FD600000B12C436D00BE42EDB2F4D191F82630C3
:10FD70005C4091F8243091F825202340134381F80A
:10FD8000253081F82440F8BD98510120342201200B
:10FD9000C84A0120044701200847012009470120E3
:10FDA00065510120D04E012088D50600F8B5134FCB
:10FDB00006460A25002447F0010700220121306889
:10FDC000FFF7A3FC4FF42070B84700213068FEF71E
:10FDD00021FA42F20F713068FFF700FF28B9013DA8
:10FDE000ADB2002DE9D12046F8BD8C4202D80134D5
:10FDF000A4B2F0E742F21074F5E700BF00BC0600C1
:10FE000007B50121019001AA0248F8F705FEFFF7A6
:10FE10003FFA00BF40FF060008B5064B1B683BB128
:10FE20001B681A68044B9A4202D00420FFF7A4F81A
:10FE300008BD00BF8C510120EF2978012DE9F04168
:10FE40000025D0F800808D75836906460C46002B8E
:10FE500055D0C36A01330AD001F11607D8F8103023
:10FE600033F8150000284CD125440023AB7500233E
:10FE7000A07D19462E27F5696A5C202A01F101014F
:10FE800021D0052A08BFE522092904D1E51800B9C7
:10FE9000AF756F72013304EB030C8CF8092088B93D
:10FEA000A2F14105192D0BD8F569082995F80CE048
:10FEB0008CBF102508251EEA050F1CBF2032D2B2C8
:10FEC0008CF8162001330B29D5D130B9E218907582
:10FED000F269127B002A08BF0023234400225A72D1
:10FEE000F369DB7A2372F0691C30F9F71FFB20609D
:10FEF000F0691630F9F71AFBE080000CA080BDE82D
:10FF0000F0817F2802D9F9F767FB30B10135B5F5EB
:10FF1000807F02D007F8010BA0E70025A4E70000CE
:10FF2000034B044801221A70034B00221A707047D9
:10FF300008470120A8E106006551012038B50146B7
:10FF400000680E4C40F30730F9F7B0FD0B68002055
:10FF5000D3F80022C3F800020B684FF0FF32C3F859
:10FF600008230A68012313610A790C2505FB024264
:10FF700013720B7905FB0343187238BD684D0120DD
:10FF8000104B98420CD003F10802904215D003F1B7
:10FF90001002904213D01833984212D1032300E08C
:10FFA0000023094A0021D1540379084A0C2101FB9E
:10FFB00003231B7A2BB1FFF7C1BF0123F1E7022313
:10FFC000EFE77047482201202D510120684D0120A4
:10FFD00043687BB15A681B7AC2F86035064A002331
:10FFE00043601378013BDBB213701BB9034B1868F5
:10FFF000FFF7C6BF704700BF64510120A451012024
:020000023000CC
:1000000008B5FFF7E5FF014808BD00BFA8E10600FD
:1000100008B50868FFF7DCFF004808BDA8E1060046
:1000200007B5400040F00100019001AA01210248FB
:10003000F8F7F2FCFFF72CF92001070037B504466A
:10004000F9F727F8C56815B91620FFF7E9FF01ABE6
:10005000002201212046A847013001D10198F4E790
:10006000014803B030BD00BFA8E1060037B5044623
:10007000F9F70FF801ABC568002204212046A84714
:10008000013002D10198FFF7CBFF014803B030BD2A
:10009000A8E106000868FFF7E9BF10B5044600684C
:1000A000FFF7E4FF2046BDE81040FEF77BBF08687D
:1000B000FFF7DCBF38B5044600F10803456800F1DE
:1000C0000C0101220068A847A36813B11846FFF786
:1000D000A7FF00B92073207B38BD08B5838803F0E3
:1000E0003003302B02D11E20FFF79AFF08BD00001D
:1000F0001FB50223009303ABF8F7D0FF039B23B196
:100100000B2B08D01846FFF78BFF400040F0010092
:1001100005B05DF804FB0148FAE700BFA8E106005E
:10012000FFF7E6BF084BD3F8183182B04BB1074B4D
:10013000074800221A601B680193019B02B0F9F77F
:1001400019BD02B0704700BF0030024018310240B4
:10015000204D012010B50446C068FEF723FF0023A0
:10016000C4E901330148E36010BD00BFA8E1060007
:10017000074B1A78C2F34000920708D51B785B073B
:1001800004D4044B187900F0010070470020704738
:10019000BC45012074260120FFF7EABF08B5FFF730
:1001A000FBFF034A034B00280CBF1046184608BD4E
:1001B000A0E10600ACE1060038B50546FEF716FDE5
:1001C00010B90024204638BD0620FEF7D9FC0446AD
:1001D0000028F6D015F00302F4D1044B0C20C3F82C
:1001E0001C55C3F82025FAF741F8EBE700900240D0
:1001F00008B5436813211888FAF77AF9004808BD52
:10020000A8E10600436843B119880548054B4FF63D
:10021000FF72914218BF184670470148704700BFEF
:10022000A0E10600ACE1060073B5104D4FF46A245E
:100230004FF00106200B2E70F9F726FB08B9F9F7ED
:1002400035FB04F58054B4F5722FF3D1084B0193BC
:1002500001A901224FF46A20F9F738FB012201A914
:100260000448F9F733FB02B070BD00BF895101208B
:1002700031304442FC1F0F0010B54FF6FF720446A8
:10028000FF210120F9F728F938B1033424F00304E1
:10029000044B083404449C4202D9FFF7C5FF0248CE
:1002A00010BD00BFFB1F0F0004A00E0008B5FFF734
:1002B000BBFF014808BD00BFA8E1060010B5044619
:1002C000406818B1FAF78CFA00236360004810BD4B
:1002D000A8E1060008B590F82330FF2B01D0FAF70B
:1002E0008DFA014808BD00BFA8E1060008B5836883
:1002F0000BB1FFF763F9014808BD00BFA8E1060094
:1003000008B5837FFF2B01D0FEF7A0FE004808BD93
:10031000A8E1060007B520B90648F8F784FBFEF708
:10032000B7FF0B680348019301AA0121F8F774FB9A
:10033000F5E700BF88020700C28B4FF6FF739A42B1
:100340000AD04368188A172838BF1720033880B2AC
:10035000400040F0010070470020F9E74FF0102303
:10036000D3F80C220379D20703D5A3F10902012A9D
:100370000DD95909012203F01F0302FA03F3054ABC
:1003800052F8212013420CBF0120002070470020AA
:10039000704700BFBC490120084BD3F8183182B028
:1003A0004BB1074B074800221A601B680193019B61
:1003B00002B0F9F7DFBB02B0704700BF00F00240A7
:1003C00018F10240444D012008B5C36813B1043050
:1003D000FAF711FF004808BDA8E1060038B54368E8
:1003E000024618681B790624C0F800451C4CC0F86A
:1003F0008815342505FB0343022483F82D40002390
:10040000C0F84435C0F84835012303628360D0F852
:1004100050311BB9D0F82431002BF8D04FF4A8711B
:10042000F9F706FC01234361D0F80431002BFBD01F
:100430004FF48271F9F7FCFBD0F824316BB14FF423
:100440009271F9F7F5FBD0F8C434C0F8C434002435
:100450005068F9F7E3FD204638BD0124F8E700BFF6
:10046000804D01202DE9F04F89B005469DF8487078
:1004700016465FFA81F81C464BB94146FFF7AEFFBE
:10048000002814BF0020132009B0BDE8F08F426897
:10049000137912680621C2F800151C4A342101FBA9
:1004A0000323002F4FF0020183F82D10914614BF53
:1004B000002320234FF0000A4FF6FF77A74228BF02
:1004C0002746CDE9047ACDE9066A69688DF80CA063
:1004D00008798DF80D804FF0340C0968019303AA58
:1004E00000FB0C90F9F7E2FB094B9842834603D1DD
:1004F000E41B019B3E44DFD16868F9F78FFD584645
:1005000009B0BDE8F04FFAF73BB900BF804D0120BC
:100510000000AD0B2DE9F04700248AB0CDE904447A
:100520005F4B60486049012225461E6846B1D0F8FD
:100530000463164204D01D601E680196019E144398
:1005400004338B424FEA4202EFD1584B1A687AB11A
:1005500000221A601B680293029B4FF0A04344F0F4
:100560000044D3F810350493514BD3F8103505935C
:1005700014F0FF0F1AD04F4F01260025344210D03F
:10058000AB0003F1804303F5C043D3F81005D3F863
:10059000101557F8253023B1C1F30141C0F30520F0
:1005A00098470135082D4FEA4606E7D1002C70DA4E
:1005B00008AF002308937B604FF0FF33CDE906338B
:1005C0003C4EDFF8EC904FF0010896F9543096F865
:1005D0005420013322F0C0045BD00AAB03EBD401FA
:1005E00002F0070A11F8103C23FA0AF3D8074FEA81
:1005F000D40C4ED53319920993F9243056F8235070
:100600004DB9032A45D117F80C0008FA0AF3034341
:1006100007F80C3001E0032AF5D003A80394F9F79A
:1006200067FA039B11F8181C03F5E07321FA0AF12D
:1006300050F82330C907C3F3014307D5022B28D153
:10064000032A1CD02DB34FF0000A1CE0032B20D14D
:10065000032AF7D102212046F9F7B6FD8DB94FF0F4
:10066000A0430499D3F81025D9F81035914213D03E
:100670000492089ACDE90532099B0793A5E7114634
:10068000E9E74FF0010A11462046A847BAF1000FEA
:10069000E5D10AB0BDE8F08705999942F9D0E7E7BE
:1006A0000061004000600040206100407C6100402B
:1006B00000030050304E01202DE9F04F0025DFF8F7
:1006C000A0B085B004460E4690464FF4803700F542
:1006D000A079AA46D4F804333B4210D059F825300B
:1006E0006BB1C4F84873C4F8087349F825A059F8E9
:1006F00025300193019B5BF82630E8B2984701351D
:10070000A8454FEA4707E5D1D4F80433DA070ED5F8
:10071000D4F800315BB10023C4F80031D4F80031C3
:100720000293029B0E4B042053F826309847D4F8CE
:1007300004339B0711D5D4F8043173B10023C4F8F6
:100740000431D4F804310393039B054B53F826304E
:10075000052005B0BDE8F04F184705B0BDE8F08FA3
:10076000B04E0120024803220021FFF7A5BF00BFC1
:1007700000B00040024804220121FFF79DBF00BFE6
:1007800000100140024804220221FFF795BF00BF7C
:100790000040024010B4C3685A8B9B8B1344828E76
:1007A000541C1A4443798486042B04BFC36B43F85A
:1007B000221017215DF8044BF7F794BB38B50D46AE
:1007C0000121F7F7F7FB2946BDE83840FFF7E2BF04
:1007D0008968806AFFF7F2BF38B50D4601210446EB
:1007E000F7F7E8FB142D09D0152D09D0132D09D1E9
:1007F00010212046BDE83840F7F76CBB1121F8E71F
:100800001221F6E7BDE838400149FFF7C3BF00BF3A
:1008100074E10600F0B54468164D2668A468A1424C
:1008200028BF2146002455F83470B94209D305EB9E
:10083000C4046168C6F824152AB9003B18BF012317
:1008400005E00134EFE7002B14BF032302234268C5
:10085000022B126809D0032B09D0012B14BF0023EF
:100860000223C2F854350120F0BD0423F9E7062322
:10087000F7E700BF7CA3060070B543681E7A044604
:1008800086B901251D7290F8313090F83020C16A88
:100890004068FFF7BFFF04F11C003146FEF72EFF52
:1008A000284670BD0020FCE738B50D4B04460425F2
:1008B000002253F8041B8C4208BF43F8042C013D6E
:1008C000F7D1A36801225A60E068E57784F82050E8
:1008D000FEF768FB2069E560FEF764FB256138BD23
:1008E000B446012038B5084B1B6800250446C3F800
:1008F00000550079F9F762FF60792571F9F75EFF1D
:100900000248657138BD00BF44220120A8E10600FD
:10091000830710B5014611D102680E4B9A420DD1E2
:100920000D4B0340062B07D1C008F6F789FE40782F
:10093000400040F0010010BD8068F9E70846F7F775
:100940006BFF43691BB1BDE81040052018471846EE
:10095000F1E700BF0C060700070080FF38B5154B14
:100960009842044623D0144DA84201D1012038BD3D
:10097000124B98421BD0C20704D5430814BF012074
:100980000020F4E7F7F748FF43693BB12146042014
:10099000984718B1431B58425841E8E72046FFF7F3
:1009A000B7FF0028E2D0013818BF0120DFE70020A0
:1009B000DDE700BFA0E10600ACE10600A8E106000B
:1009C00010B504460846FFF7C9FF2071004810BD66
:1009D000A8E10600D1E9023249685B1A1344002AF3
:1009E000CCBF03F1FF330133042893FBF2F303D0B0
:1009F000052807D000207047054A0648002BC8BFCD
:100A00001046704723EAE370400040F00100704751
:100A1000ACE10600A0E1060010B5104A11F07F0419
:100A20004FEAD1100BBF012341F480715365C2F826
:100A30001815BFF36F8FBFF34F8F094B03EB4403C0
:100A4000034493F8212042F0020283F8212093F816
:100A5000212042F0010283F8212010BD00700240E5
:100A6000BC450120F8B5069D3C264FF461676E43F6
:100A70005F434D1E144B33F81550022904461544AC
:100A800003D9F8F7FDFD00B10135A4F2CD726FF482
:100A9000C863E1184FF4C870B1FBF0F101EB9201AB
:100AA0000A4BA4F26D726420B2FBF0F20798891A27
:100AB0000D44074903FB04042144394405483144EB
:100AC00000FB0510F8BD00BF10BB06008033E1013C
:100AD00080569C50805101002DE9F04190F82E3055
:100AE000448D264E264FDFF89C806FF300030546A9
:100AF00080F82E30013C631C01D1BDE8F0816B68A9
:100B000053F83400830726D10368B34230D1B0F9DB
:100B10003830B0F93C2093421FD090F8511089072B
:100B20001BD0838790F8503023F0070380F85030B3
:100B3000836813F0030105D1DFF84CC01A686245E1
:100B400008BF1973436813F0030204D119684145C3
:100B500001D19A821A83013CCDE790F850104907E1
:100B600001D49342DED1436C8363836CC363D9E7C2
:100B7000BB42F0D1FFF7B0FFEDE700BF58C9060058
:100B800034C50600A0C0060040C70600062837B5D9
:100B90000C4619D18D680D4B2B40062B12D1E8085D
:100BA000F6F74EFD007830B901A92846F8F770F83D
:100BB0000199F6F753FD23795840400040F00100B9
:100BC00003B030BD6868EEE70020F9E7070080FF5A
:100BD00038B50446F9F798FB236906480122002539
:100BE00083F821205D602169F8F75EFC02482561E9
:100BF00038BD00BFB1680300A8E10600F7B50446A0
:100C00000D46F8F743FE58B34E4E0127200B3770C0
:100C1000F8F73AFE10B1002003B0F0BDF8F746FE39
:100C20000228F8D04FF40072294620463770F8F7B2
:100C300029FE0028EFD1F8F739FE0228EBD04FF457
:100C4000007205F5006104F500603770F8F71AFED0
:100C50000028E0D1F8F72AFE023818BF0120DBE7B0
:100C60004FF080531A69B4FBF2F302FB134363B9EC
:100C7000354B0222C3F80425C3F80845D3F80024F5
:100C8000D007FBD50022C3F804252F4B0122C3F85F
:100C9000042514F0030351D04FF0FF32C3F10400D8
:100CA000019201AA2946E61A1A44054411F8017B6B
:100CB00002F8017BA942F9D1019A234FD7F8001419
:100CC000C907FBD53260BFF35F8F03F6FC730444A2
:100CD0009908DFF874C02E1F04EB8101224656F8F4
:100CE000047FDCF8000410F00100FAD042F8047B25
:100CF000BFF35F8F9142F2D199071AD023F003021C
:100D00004FF0FF36A118019604F0030401AE2A4407
:100D100034441D4412F8013B04F8013B9542F9D1DB
:100D2000019B094CD4F80024D207FBD50B60BFF31C
:100D30005F8F054B0022C3F804256DE74FF4805305
:100D4000C6E700BF8951012000E001402DE9F043D2
:100D5000DFF8A480DFF8A49085B005460C46002794
:100D600001266B8DBB4217D895F82E30DB070ED5C8
:100D7000002E3BD0B5F918302380B5F91A306380C6
:100D8000B5F91C30A380B5F91E30E380002686F04B
:100D9000010005B0BDE8F0836B6853F837008207A7
:100DA0000FD10368434513D1B0F93C20B0F9383076
:100DB000934214D0836B0193C38FADF80820ADF834
:100DC0000A3076B1019B2360029B6360002606E037
:100DD0004B45F6D101A9FFF7B9FF0028F1D1013742
:100DE000BFE701A92046FAF7EDFBEFE705F118018F
:100DF0002046FAF7E7FBCAE758C9060034C50600E3
:100E0000F0B5436853F8314014F0030785B0054648
:100E10002CD12368204A93422AD1B4F93C30B4F94A
:100E200038209A421EBFADF80830E38FADF80A3083
:100E300094F850301CBFA26B01926FF3041384F836
:100E400050304FF0000314BF01263E46A3626EB13E
:100E500095F82E30DB0718D4019BAB61029BEB6148
:100E600095F82E3043F0010385F82E3005B0F0BD23
:100E70000A4A9342FAD101A92046FFF767FF394693
:100E800006462046FAF766FBE1E701A905F11800DE
:100E9000FAF798FBE4E700BF58C9060034C506001E
:100EA00070B5438D013B4385436803EBC1030446A2
:100EB0005E680D46FFF7A4FF618D6368A94209D8FB
:100EC000002243F83120618D636803EBC103304693
:100ED0005A6070BD013503EBC50393E8030003E9D5
:100EE0000300E9E77FB5D0F8246105460C46002EE3
:100EF0005CD04FF49271F9F7EBF802238DF80030D3
:100F0000D0F88034C0F880340393D0F83C35029395
:100F1000E36801930023C4E906336846D4E900136B
:100F20009847D5F844317BB14FF4A2712846F9F7C0
:100F3000CFF8A36943B10023C4E90633E268D5F8CA
:100F40003C152046F9F7CCF8D5F82031ABB14FF479
:100F500090712846F9F7BCF80123EB60636963B12F
:100F6000D5F84C2502920023A2688DF80030636109
:100F70000192D4E9001368469847D5F858319BB1DF
:100F80004FF4AC712846F9F7A3F8636963B1D5F85B
:100F90004C2502920023A2688DF800306361019213
:100FA000D4E900136846984704B070BDD0F81031FA
:100FB000002BB6D04FF48871F9F78AF8A169D0F800
:100FC0003C359942ADD1E369E26873B1D0F80032A3
:100FD00023F02003C0F80032E369A3612369E360D2
:100FE000E6612046F9F77CF89BE7A361F9E700008A
:100FF00001490248FFF776BFE84D0120002000407C
:1010000001490248FFF76EBF0C4E012000800240EC
:101010002DE9F84F1E460379D2F800900F780D465F
:10102000A3B3B2F80AA0B2F80CB050465946FAF78A
:101030002DF9594680460AF12100FAF727F90BF1FC
:10104000210104465046FAF721F9102F4FEA194CB6
:10105000C9F307225FFA89F321D100F007000344A6
:1010600008F00708FF2BE04428BFFF2304F0030427
:10107000B8F1FF0F28BF4FF0FF081444FF2C28BF22
:10108000FF24240244EA084444EA0309102F1BD138
:101090004846FAF71FF930600123337151E0FF2110
:1010A0003941084053FA80F308EA0108FF2B5CFA43
:1010B00088F828BFFF230C40B8F1FF0F28BF4FF07E
:1010C000FF0852FA84F4D9E76B79002B40D04846E8
:1010D000FAF70CF9C7F1080738414FEA19423060B6
:1010E0005FFA89F08242144638BF044682421346B2
:1010F000C9F3072128BF03468B4228BF0B468C4209
:101100002CBFC3EB0403C3EB0103DBB2102B2C7920
:1011100003D8002CC0D13460BEE74846FAF7FAF88D
:10112000AB78181A80B200F10A039BB2142B05D9D0
:1011300000B210F1DB0F01DBDB2806DD1CB1002360
:101140003360BDE8F88F0123FAE7002CF9D1F6E708
:101150002B7953B1082F08D84846FAF7C7F8C7F1DA
:10116000080740FA07F7376096E7002395E7000085
:1011700079B3F8B5041F174E04EB8105032754F823
:10118000040F030719D1D6F8F830984215D3D6F8D2
:10119000FC20904211D2C01A48BF0F300011D6F87F
:1011A000ECC0810800F003031CF801E05B004EFA7C
:1011B00003F202F00302012A02D0A542DFD1F8BDFA
:1011C00007FA03F343EA0E030CF80130F6F75AF975
:1011D000F3E77047D04E0120F8B52E4CB4F8083232
:1011E00000220133A4F80832C4F80421251D04F1BB
:1011F000D806032755F8040F020719D1D4F8F830A0
:10120000984215D3D4F8FC20904211D2C01A48BF9E
:101210000F300011D4F8ECC0810800F003031CF873
:1012200001E05B004EFA03F202F00302012A1FD034
:10123000AE42DFD1D4F83002030718D1D4F8F83029
:10124000984214D3D4F8FC20904210D2C01A48BF60
:101250000F300011D4F8EC40810800F00303655C06
:101260005B0045FA03F202F00302012A09D0F8BD3F
:1012700007FA03F343EA0E030CF80130F6F702F91C
:10128000D6E7032202FA03F31D436554BDE8F84094
:10129000F6F7F8B8D04E012003071CD1124BD3F853
:1012A000F820904217D3D3F8FC10884213D230B400
:1012B000801A48BF0F300011D3F8EC40810800F0CD
:1012C0000303655C5B0045FA03F202F00302012AA6
:1012D00002D030BC70477047032202FA03F31D436B
:1012E000655430BCF6F7CEB8D04E012010F00F0296
:1012F0001DD11849D1F8F830984219D310B4D1F85B
:10130000FC40A0420FD2C31A48BF0F331B11D1F8C3
:10131000EC40990803F00300615C4000014101F0DA
:101320000301012906D010465DF8044B70470022E6
:101330001046704701329918880801F00301205CBB
:10134000490040FA01F101F003010229F2D0120133
:10135000E9E700BFD04E012021F00F012DE9F8434D
:10136000384A394C0F1AFF00A2FB07324FEA5228C5
:10137000A1EB881C4FEA8806C4E93EC1073600EBA2
:10138000080310F00301C4E93C834FEAD609C4F80E
:10139000EC0042D0B7F5037F36D34246002104F07B
:1013A00089FAD4F8F43013F003012DD1760906D070
:1013B000B6001846324604F07DFA0346334419F06D
:1013C000020F1CBF002223F8022B19F0010F01D0DD
:1013D00000221A70202200211C4804F06BFAD4F875
:1013E000F020D4F8F830501E03EB821301210022C4
:1013F000C4F82C02C4F80031A4F80822C4F8302242
:1014000084F80A12BDE8F883B9F1000FE2D04A4629
:101410001846002104F04EFADCE7D20A054604D053
:1014200097003A4604F046FA3D4418F0020F1CBFFC
:10143000002325F8023B18F0010FB2D000232B70D7
:10144000AFE700BFF32C23FAD04E0120DC5001207F
:1014500008B510F00103024663D03D284FEA60034F
:1014600007DC0C2B17DC022B4ED0052B4ED0012BAA
:101470004ED02D49002301EBC300406882424BD17E
:1014800051F83300C008F6F7F9F80378002B01464D
:1014900008BF002130E00D3B112BEAD801A050F825
:1014A00023F000BF1115030073140300731403002D
:1014B000731403001515030073140300ED140300E7
:1014C0007314030073140300FD140300731403006A
:1014D00073140300731403007314030073140300E4
:1014E0000115030073140300051503000F4803885A
:1014F000322BBED8F7F70EFF084608BD0C48F6E7BA
:101500000C48F4E70C48F2E70C48F0E70C48EEE72B
:101510000C48ECE70C48EAE70133172BABD100216C
:10152000EAE71946E8E700BF40EA0600344C070046
:101530001E54070006400700EE4E07000059070042
:101540008E4A0700743B07001C560700836813F996
:10155000012B002AFBDB13F9012B002AFBDB0433F0
:1015600013F9012B002AFBDB18887047136810B5AC
:1015700014463BB92B2905D1FFF7E8FFC00040F026
:101580000600206010BD136810B5144643B92B291E
:1015900007D14068FFF7DAFFC00040F00600206086
:1015A00010BD162904BF43681360F9E7024B1A699E
:1015B0000260186100207047D04E012040EA01030C
:1015C000F0B59C0709D0431E0A44914200D1F0BDFA
:1015D00011F8014B03F8014FF7E722F00303051F51
:1015E0009608CC18A1420DD1910744BF34F8021BD4
:1015F00020F82610034448BF0233D20744BF2278A4
:101600001A70E4E751F8047B45F8047FEAE713B564
:1016100004460193104629B9224601A9FFF7CEFFDF
:1016200002B010BD01AB23441444A242F8D013F819
:10163000011D02F8011BF8E738B5456895420446DC
:1016400028BF15462A460068FFF7B8FF236862687E
:101650002B44521B2360626038BD00002DE9FF4718
:10166000334B1B6806460C46154623B900273846FF
:1016700004B0BDE8F087FDF7B9FA07460028F5D0B9
:1016800014F003081ED00DF10C0909F06043B3F10A
:10169000005FEBD1274B0420C3F80465C3F808951D
:1016A000C3F80C05F8F7E2FD234B9842DED1C8F1F0
:1016B0000408204642464946FFF780FF444446441A
:1016C000A5EB080504F06043B3F1005FCED1A3079A
:1016D000CCD1DFF8608025F00309C8F80465042048
:1016E000C8F80845C8F80C95F8F7C0FD124B9842A9
:1016F0008246BBD1B5EB0902B9D003AD05F060431A
:10170000B3F1005FB2D104204E440192C8F80465E1
:10171000C8F80855C8F80C05F8F7A8FD5045A5D13C
:10172000019A294604EB0900FFF748FF9FE700BF35
:10173000CC4A0120009002400000AD0B10B50422FD
:10174000ADF5027D0DEB02010446FFF787FF78B18E
:1017500001AA042312F8011BFF2909D1013B9BB206
:10176000002BF7D14FF4007202A92046FFF776FF55
:1017700000200DF5027D10BD30B5C1B00C464FF410
:10178000807269460546FFF769FFA0B14FF4807289
:1017900069462046FDF76EFF68B14FF480726946D6
:1017A000A818FFF75BFF30B14FF480726946A018AC
:1017B000FDF760FF00B9002041B030BD2DE9F041D8
:1017C000194C236801332BD0184BDFF864801B6859
:1017D0001E680120A6F5805600250746D8F800208F
:1017E00007FA05F3134209D130B1206806EB452111
:1017F00000EB4520FFF7C0FF00F001000135082D88
:10180000ECD170B12068FEF7D7FC00252168701973
:10181000294405F50075FFF7AFFFB5F5805FF5D1F9
:101820000120BDE8F08100BFC8490120CC4A012059
:10183000D04901202DE9F84F2E4D2B680133074682
:1018400006D1002F53D1FDF745FE0120BDE8F88FEA
:10185000DFF8A490DFF8A4A000244FF00108D9F825
:10186000002008FA04F3134211D1E60006F1080B38
:10187000DAF8C830286899594FF4807200EB861066
:10188000FFF7ECFE0028E1D00436B345F0D1013477
:10189000082CE4D12868DFF86490DFF864A0FEF734
:1018A0008BFC4FF000081FE0D9F8C8302868995920
:1018B0004FF4807200EB8610FDF7DCFE57B9DAF8C2
:1018C00000303BB9D9F8F83023B1D9F8C83098596D
:1018D000FDF768FB0436B442E6D108F10208B8F11E
:1018E000100F04F10804ACD04FEA8806DCE7384654
:1018F000ACE700BFC8490120D0490120D04E0120EB
:101900009051012008B5074BD3F8C83033B9FFF721
:1019100055FF054B4FF0FF321A6008BD0120FFF75D
:1019200089FFF6E7D04E0120C849012008B50A4BCF
:101930004FF47A721A60FFF7E5FF084BD3F8C8300E
:1019400033B9FFF73BFF064B4FF0FF321A6008BD7B
:101950000020FFF76FFFF6E734220120D04E012070
:10196000C849012008B5FFF7E1FFF7F7C1FC000007
:101970002DE9F84F0346002940F0B180421E0C4685
:1019800000F2BD1002F8014F8242FBD1834A126877
:10199000106883F8BE41A0F58050440A1FBFFF22A3
:1019A00083F8BF2183F8C02183F8C1214FF00102E1
:1019B00002BF83F8BF4183F8C04183F8C14183F877
:1019C000C221002C40F0838083F8C34183F8C441D6
:1019D00083F8C541012283F8C62183F8CA41002259
:1019E000440C400E83F8C72183F8C82183F8C9212D
:1019F00083F8CD2183F8CE2183F8CF2183F8D0213D
:101A000083F8D12183F8D22183F8D32183F8D4211C
:101A100083F8D52183F8D62183F8D72183F8D821FC
:101A200083F8D92183F8DA2183F8DB2183F8DC21DC
:101A300083F8DD2183F8DE2183F8DF2183F8E021BC
:101A400083F8E12183F8E22183F8E32183F8E4219C
:101A500083F8E52183F8CB4183F8CC0183F8E621B4
:101A600083F8E72183F8E82183F8E92183F8EA2164
:101A700083F8EB2183F8EC2183F8ED2183F8EE2144
:101A800083F8EF2183F8F02183F8F12183F8F22124
:101A900083F8F32183F8F42183F8F52183F8F62104
:101AA00083F8F72183F8F82183F8F92183F8FA21E4
:101AB00083F8FB2183F8FC2183F8FD21552283F86C
:101AC000FE21AA2283F8FF210846BDE8F88FFF22F5
:101AD00083F8C32183F8C42183F8C5217AE7013A4A
:101AE0002E4FDFF8C080DFF8C0904E1E0446551818
:101AF000AE4201D10021E7E73B681868A0F5805CA1
:101B0000B6EB5C2F01D30121DEE7D9F8002008EA0B
:101B1000462393424FEA46203BD100280346B8BFF4
:101B200000F2FF135B125A4202F0070203F00703B0
:101B30001B4958BF5342DBB2012209689A40D2B216
:101B40000A4226D0DFF864A0DAF8C810B9B14FEA2B
:101B5000430B4FF4807251F82B102046FFF72EFDF7
:101B6000DAF8C8100BF101034FF4807251F823101A
:101B7000A018FFF723FD04F500740136B8E74FF411
:101B8000007221460CEB4320FFF768FD0028F2D1DC
:101B9000B9E74FF400722146F6E700BFCC4A0120B6
:101BA000D049012000F0FFFFC8490120D04E01209C
:101BB00010B58389C288044600689BB202FB03000B
:101BC000FFF7FCFCA389A1889BB20133B3FBF1F2C0
:101BD00001FB12339BB2A38163899BB2994215BF6B
:101BE0006389A38901339BB216BF9BB2E3816381F2
:101BF00010BDF8B5037A04460E46154633B942893E
:101C000083889B1A9BB29D4228BF1D460027BBB20A
:101C10009D4201D82846F8BD31462046FFF7C8FF4F
:101C2000E38801371E44F2E738B50446154632B959
:101C30000378012B02BF104B8022C3F88420E38974
:101C400022899BB29A4204F1040001D1237B73B133
:101C5000FFF7AEFF75B901252378012B02BF064BB4
:101C600080225A6035B9BDE83840F7F7AFBB002D88
:101C7000F9D1F1E7012038BD00E100E04378023BF3
:101C80000A46032B10D8DFE803F00225141C124B80
:101C900019786FF30001197019786FF34101197009
:101CA00019786FF3820119700C4B01461868FFF721
:101CB000BBBF094B1978C9070CD5197841F004014D
:101CC000F1E705490B78DB0704D50B786FF3820346
:101CD0000B70E9E7704700BFBC450120F0450120CB
:101CE0001FB50023CDE9013301218DF8050001A8BE
:101CF00003938DF80430FFF7C1FF05B05DF804FBD6
:101D0000012813B5044600F0A18002284DD1634B91
:101D1000D3F800241205FBD54FF40062C3F8002469
:101D2000BFF36F8FBFF34F8F5D4B1B68082B0AD13A
:101D30005C4B5D4A1868002840F0828049F275319A
:101D4000196010601960F7F781FE48B1554B574A8A
:101D50001868002877D149F2753119601060196050
:101D60004F4B1B68082B09D1514B40F2E3721A60AC
:101D700040225A60BFF36F8FBFF34F8F474C4D49DE
:101D80008022C4F81C25C4F804134B49C1F88421EF
:101D90004A60F7F771FE0028FBD00123C4F8043530
:101DA000BFF36F8FBFF34F8F48E0002846D13B4B06
:101DB000D3F80025002A41D14FF40062C3F8002473
:101DC000BFF36F8FBFF34F8FF7F740FE48B1354B2E
:101DD000364A1868032128BB49F275301860116033
:101DE00018602F4B1B68082B09D12E4B2E4A186800
:101DF000C021C8B949F27530186011601860274BCE
:101E00000124C3F80045BFF36F8FBFF34F8FF7F77F
:101E100033FE98B9F7F73AFD40B102B0BDE8104083
:101E2000F7F724BE1160DCE71160E8E7234B186088
:101E30001B680193019B4FF080431C6002B010BDF2
:101E4000002313607FE70023136089E7134BD3F867
:101E50000025002AF2D00022C3F80425BFF36F8FBB
:101E6000BFF34F8F14498020C1F88400D3F80013CA
:101E7000C3F80813C3F80025BFF36F8FBFF34F8F6C
:101E8000F7F704FD38B1F7F7F3FD022002B0BDE823
:101E90001040FFF725BF0A4B1C60F6E700700240B8
:101EA0003001001000EC064014EC064014ED064032
:101EB000007802400514800100E100E000010040CC
:101EC0000400004013B5274C402384F827330DF15C
:101ED000030000238DF80330F7F7B2FA9DF80330C2
:101EE000EBB10120F7F7A6FA0120F7F7A1FA0120DC
:101EF000F7F7A2FA01A8F7F7A1FA1B4B1A7862B11B
:101F000000201870019BDA0701D5FFF7F9FE019B4D
:101F10009B0702D50220FFF7F3FE02B010BD134B62
:101F20001A788AB94FF08041C1F88025C1F8782528
:101F30002268D10706D4E02284F800230122C4F8E5
:101F40008021226001221A70094B0A4A1A604FF060
:101F500080434FF46072C3F80423D3F838340193FC
:101F6000CBE700BF00E100E0382201202C51012026
:101F7000C44E0120011D03001FB50024CDE901441A
:101F80008DF8040007208DF805008DF8081001A8D1
:101F9000194603928DF80940FFF770FE04B010BD9A
:101FA0001FB5124B93F8C020BAB1114A5268C2F360
:101FB000080272B10023019308238DF805300D4B00
:101FC0000121CDE9023001A8FFF758FE05B05DF808
:101FD00004FB93F8C020002AFBD1012283F8C02023
:101FE0000260BFF36F8FBFF34F8FEFE7382F0120F1
:101FF00000ED00E0A11F0300F8B5104D104E00F5F4
:102000009473182455F823304443142202FB0052E1
:10201000DDB20C4B3159C2F8001703EB8000C2F857
:102020000457FFF7BDFF335937192B443351FB8851
:1020300015FA83F39BB2FB80F8BD00BF007002402D
:10204000382F01202870024010B4104B182101FBDA
:1020500000314A8A0B8ACC689B1A0A7D9BB2934254
:1020600028BF13461422424302F1804202F51C327B
:10207000C2F80046C2F804362344CB60044B5DF836
:10208000044B03EB8000FFF78BBF00BF382F01200C
:1020900004700240F8B50446182300F07F001E4D7E
:1020A0001646E70903FB00F20C2303FB0723EA189B
:1020B000E95000239680D3802A4698B996B91748EC
:1020C000FFF76EFF95F8C0304BB9F7F7A7F900237B
:1020D0001A4621461846FFF74FFF0120F8BD85F844
:1020E000C060F4E7AFB9182303FB00235B7A13B198
:1020F000FFF782FFF1E70A4B30B90122DA64BFF340
:102100006F8FBFF34F8FE8E700F5947043F82070AE
:10211000F5E7FFF799FFE0E7382F01205070024004
:102120000070024010B50C46204611461A46FFF7D3
:10213000B1FF60B1064B04F07F0103EB410303EBF9
:10214000D41191F8213043F0010381F8213010BD02
:10215000BC450120F7B58B79062B06460C46174681
:1021600002D1CB79502B08D0154B1B68DA0702D46B
:10217000002003B0F0BD00BEFAE7124D097805F16A
:102180002E03019305F12F03009302231A462144E5
:10219000FCF7A0F928B90A4B1B68DB07E8D500BE9D
:1021A000E7E7A37885F82D3017233B8095F82F10AB
:1021B0001F232A463046FFF7B5FF0028D9D1EAE7AA
:1021C000F0ED00E05C44012070B4104A104B4FF475
:1021D0000B6444431519E97801F07F0003EB4003D9
:1021E00003EBD11393F8210010F001000CD16E8B9A
:1021F000AB8A9B1B9BB23F2B06D904F50364224498
:10220000402370BCFFF78EBF70BC7047742601205E
:10221000BC450120F7B58B79022B0746154607D040
:10222000274B1B68DB0700D500BE002003B0F0BDC4
:10223000CB79073BDBB2F72BF2D9224EB378002BD8
:10224000EED18B7833700C7809230C44138005E0B1
:1022500023782A8813442B8023781C446378242B0A
:10226000F6D0052B11D12046FCF702F928B9144B02
:102270001B68DA07D9D500BED8E7A3787370237836
:102280002A8813442B8023781C446378042B12D1B2
:1022900063790A2B0FD10C4B217801930133009302
:1022A00002231A4621443846FCF714F90028DED0F0
:1022B0002B8817332B800020FFF786FF0120B5E71E
:1022C000F0ED00E0742601207626012008B5084BC9
:1022D0001B6899420AD1074B002058839883D88302
:1022E000FFF772FF044B03F128029A6508BD00BF97
:1022F000CC4E012074260120D04E0120F8B51A4A98
:10230000D0788842144612D11646D51802F110072B
:10231000AE4211D1154B2BB1638B9BB213B1002090
:10232000AFF300800020FFF74FFF012003E0937818
:102330005B1A58425841F8BD638BA28A9BB29A42FD
:1023400006F5036101D1237E13B13846FFF730FC57
:102350006379FF2B06D096F83018994202D10020FD
:10236000FFF7B4FF0136D3E7742601200000000018
:1023700008B5074A93788B4208D110231832FFF72B
:10238000D1FE20B9BDE80840F7F720B8002008BD0D
:10239000FC2F01202DE9F341244B5C7807460D46C4
:1023A00090461E46002C3BD10A781144996291F860
:1023B00001C0BCF1210F0BD1AC5C5A1C023301925D
:1023C000009321442A790323FCF784F8044650B98A
:1023D000174B1B68DA0704D40024204602B0BDE87E
:1023E000F08100BEF9E7AB79012B04BFEB79F37004
:1023F00000233371AB783370B36AB3F80730F380DE
:102400002B79C3EBC3031233A8F80030B17800294D
:10241000E3D0084A10233846FFF784FE0028DCD1B9
:10242000034B1B68DB07D7D500BED5E7FC2F012087
:10243000F0ED00E0143001202DE9F8431A4C1D4660
:10244000A3788B42064611D115F0030705D104F29B
:102450002D1904F10408BD420BD8144AA178402379
:102460003046FFF75FFE08B9F6F7D8FF0020BDE859
:10247000F88319F8012C02F00F03052B12D00F2B53
:1024800010D002F00B02022A04D00C3B012B94BFA7
:102490000222032249464046FFF7ABFB043709F10D
:1024A0000409D8E70122F5E7A0320120CC3301204E
:1024B0002DE9F8438B79012B80460D46164608D14D
:1024C0000A7809213180AA5C0A4432801846BDE8A6
:1024D000F883032B01D00020F9E7CB79002BFAD148
:1024E0001E4F97F80190BA7859EA020934D18B78D7
:1024F0003B700C7809230C4433802B794B4508D86A
:10250000174AB97840234046FFF70CFE0028DED179
:1025100006E06378052B18D12046FBF7A9FF28B900
:10252000104B1B68DB07D6D500BED0E7A378DA09CD
:1025300014BF7B70BB7023783288134433802378B8
:1025400009F101091C445FFA89F9237832881344A0
:10255000338023781C44D0E71B70FFDEA0320120BB
:10256000CC330120F0ED00E010B5154A0446507B55
:10257000F6F778FF936892F82F1068B993620123F9
:1025800082F82C3042F2077382F83E00938720468F
:10259000BDE81040FEF740BA926B9B1AB3F5805F1E
:1025A00028BF4FF48053074A9BB22046FFF7BAFD7D
:1025B00020B9054B1B68DB0700D500BE10BD00BF6E
:1025C0005C4401205C340120F0ED00E010B40A4CC2
:1025D00008680B464968224603C20022C4E9022269
:1025E00093F900305DF8044B93421146ACBF802054
:1025F0001046FFF74FBD00BF242F012013B5124B2B
:102600009889D98993F90040421A92B2402A28BF8A
:102610004022002C0EDA884212D099680B480192B1
:10262000FEF7CCFF0949019A802002B0BDE81040B6
:10263000FFF730BD88424FF0000003D10021F4E7DE
:102640008020FBE70149F0E7242F01207C45012091
:10265000F8B51B4E0D46844608684968B260374697
:1026600003C714460022F281E9888B4228BF0B463B
:10267000B381A3B13CB9134B1B68DA0701D4002026
:10268000F8BD00BEFBE76046FFF7B8FF08B10120C8
:10269000F6E70C4B1B68DB07F1D500BEF0E795F9B8
:1026A0000020002AACBF802000201A461946FFF700
:1026B000F1FC0028EBD1BDE8F840F6F787BE00BF7B
:1026C000242F0120F0ED00E037B50B7803F0600314
:1026D000202B05460C4621D14B78FE2B06D0FF2B34
:1026E0001CD1FFF773FF012003B030BD01238DF82B
:1026F00007300B4B1BB1AFF300808DF807009DF83E
:1027000007000028F0D0431E8DF807300DF10702B6
:10271000012321462846FFF79BFFE4E70020E3E77B
:102720000000000038B50B7803F06003202B0C4646
:1027300009D10F4A8B8815789D4204D14B78212B03
:1027400003D81F2B0ED8002011E0222BFBD14B8881
:102750001371FFF73BFF608810F0010007D1FBF712
:1027600075FE03E007230632FFF772FF012038BD34
:1027700074260120F0B50B7803F01F05012D85B0FC
:1027800006460C4601D000201AE04A4A8F8892F88B
:1027900000C0FFB2BC4517466AD0474B1B68DB0739
:1027A000F1D500BEEFE76378062BECD163881B0AF6
:1027B000212B07D1926A002AE5D01378FFF748FF52
:1027C00005B0F0BD222BDED1D3883C4AFFF740FF95
:1027D00035E063881A0A012ADFD1DAB2384B0021CA
:1027E00018461D7A954210D10C22E388019302FB12
:1027F00001011A4649683348FEF7E0FE019B002BB1
:10280000CBD0304A21463046E0E70131042903F1BC
:102810000C03E6D100235B68FFDEE388102BB2D8FF
:10282000294AEFE76088294B000A78711BB1AFF3A2
:1028300000800028A7D021463046FFF7C7FE0120C0
:10284000BEE7234A0123DDE73B79C3F101038DF89D
:102850000F300DF10F020123D4E760881D4B0138C2
:1028600018BF01203871002BE5D0AFF30080E2E7FC
:1028700013F0600397D0202B85D16378013B0A2B9E
:1028800081D801A252F823F0D32703004328030084
:1028900049280300872703008727030087270300B1
:1028A00087270300872703001B2803002528030030
:1028B0005B280300FC2F0120F0ED00E094D6060019
:1028C000DC2301200430012014300120000000002E
:1028D0000130012000000000F7B50E46144600F15B
:1028E00008054FF0FF37042C2246314628BF04224A
:1028F00001A80197FEF762FE012201A92846F6F71A
:10290000E5FF042C04D9043CA4B204360435EAE7FC
:1029100003B0F0BDF7B50288112A04460D464FF00A
:10292000000344D0262A40D0102A64D1334988209D
:102930004FF6FF760A4600FB03F77F5AB74203D0F3
:102940000133052BF7D104232D4E88204343D118A2
:10295000A088D6F8D070D0522A48C865C1E918714D
:102960000020294F81F85A00A1F876008F6603F104
:1029700060011144C6F8D01004F10801A86151F8B3
:10298000080F6C334968134403C36846F7F7B4FC77
:10299000BDF80030228A9A4202D8628A9A4203D253
:1029A000A0886946F7F7A2FC0023EB6020E0134AF9
:1029B00081881746882000FB03F6B65A8E4203D062
:1029C0000133052BF7D1042388265E43B9190E483D
:1029D000F6F76AFD4FF6FF73BB530023CA6D81F80B
:1029E0005A3008498A421EBF5360217A1172AB6186
:1029F000012003B0F0BD1846FBE700BF10470120DF
:102A0000D04E0120A8E106006960030038B50388B4
:102A1000362B0C4615D1B1B182888B899A4212D1DE
:102A2000C388CB81C5894A68954228BF154600F105
:102A300010012A462068FEF7C1FD0120A560207420
:102A400038BD0020FCE70120FAE700002DE9F04F37
:102A500015464268DFF860A01368DFF86080DFF891
:102A600060B087B081460E4601930DB901201BE08E
:102A7000D9F80420019BD768AF4228BF2F465345A1
:102A800015D13A4631464046FEF798FD4246D9F800
:102A90000400002402A9CDE90227CDE90444FBF794
:102AA000C7FB584505D0204607B0BDE8F08F324639
:102AB000EDE73E44ED1BD8E700F0024000000120A6
:102AC0000000AD0BF8B51C464B1E59421746594144
:102AD00005461430069EFCF711FE012F17D126443F
:102AE00005F11C07B44200D1F8BD012221466868F7
:102AF000FFF7ACFF01213846FCF700FE0120F7F795
:102B0000EBFE00213846FCF7F9FD0134EAE768687E
:102B100032462146BDE8F840FFF798BFF0B5ADF565
:102B2000805D81B0044617461E460D4649B9B2F590
:102B3000805F06D11946FEF761F80DF5805D01B0A2
:102B4000F0BD4FF4805221466846FEF737FD31460E
:102B50003A460DEB0500FEF731FD69462046EAE7EF
:102B6000F8B544680C44C4F30B0116461D46641ABC
:102B70000DB90120F8BDC1F58057AF4228BF2F46DF
:102B800033463A462046FFF7C9FF0028F2D0ED1B36
:102B90003E4404F580540021EAE72DE9F04184B079
:102BA00002AF0C463A6A054619460CBB5300D81DC5
:102BB00020F007006E46ADEB000D02A84FF0800C30
:102BC0000DF1090E94420BD10122A98B009202460D
:102BD0006868FDF747FCB5460837BD46BDE8F0819B
:102BE00011F8048000F814C00EF814800134E9E7ED
:102BF00002F1080020F007006C46ADEB000D40200C
:102C0000531C8DF808000DF109007B60FEF7D6FC1F
:102C10000122A98B009202AE7B6868683246FDF7FC
:102C200021FCA546D8E7F8B54589ADB204460E4665
:102C300055B143899BB29A428ABF45891546ADB2C8
:102C40000027BBB29D4201D82846F8BDE389E2883F
:102C500021689BB202FB03113046FEF7AFFCE3890B
:102C6000A1889BB20133B3FBF1F201FB12339BB29B
:102C7000E3816389013B9BB26381E38801371E4492
:102C8000DFE700002DE9F047564C23780F469046C9
:102C9000002B40F0A08000252846BDE8F0871A09E7
:102CA000A2F10801032901D90E2A23D184F8242195
:102CB00084F829610135A84549D094F828017B5D45
:102CC00094F8241100286AD14FF0020C042984F8EA
:102CD000253184F828C1E2D1F72B06BF052384F8FB
:102CE000243184F8281194F8282194F829319A4243
:102CF000E0D123E0A2F10C01012905D884F82421B8
:102D0000032384F82931D5E70F2A40D1F02B02D1D3
:102D100084F82461CCE703F0FD02F12A02D184F8A3
:102D200024C1EDE7F22B03D1032384F82431BFE75C
:102D3000052384F82431022384F829312A48042207
:102D40005146FEF756FF032842D8002839D1627851
:102D5000264B02F07F0103EB410303EBD21393F800
:102D6000210010F0010697D121494022A1F5AC7055
:102D7000FFF759FF034600288ED01D4A6178304680
:102D8000FFF7D0F9002887D1F6F720FB84E70F235F
:102D900084F82431A4F8260184F829C1CEE722184A
:102DA000042982F8243100F10102D2B284F82821EA
:102DB00099D1F72B97D1043084F8240184F8292184
:102DC000BCE70C4B1B68DB077FF565AF00BE62E715
:102DD00084F828916EE70025042604F5927AA94626
:102DE00069E700BFA0320120B4320120BC450120B8
:102DF0000C340120F0ED00E008B510461AB102488D
:102E000092B2FFF710FF08BDA4320120814210B436
:102E100010D28B1898420DD2531E194403449A1AAB
:102E20009A4202D15DF8044B704711F8014903F84A
:102E30000149F5E75DF8044BFEF7C0BB38B5044621
:102E4000154662688A42084603D929448A4201D855
:102E5000606038BDA368521A18441944FFF7D6FFC2
:102E60006268521B6260F4E72DE9F04F2DED028B92
:102E700083B00C460092F2B901F10C05D4F800A021
:102E80000AF10203EB1808EE103A574606464FF0D7
:102E900000094FF0610B33780BB1292B0DD1B9F13B
:102EA000000F58D0002D56D02368013BA3EB090337
:102EB00005F809304FE00025E0E73F2B00F02981BD
:102EC00013D8243BDAB20A2A19D822680A2B16D85A
:102ED000DFE813F0AF01150015001500D90015004B
:102EE000420172011500150075005E2B00F09981FA
:102EF00015D85B2B06F1010169D05C2B28D027681F
:102F0000002D59D07B1C23600123EB5523685A1CEC
:102F100022603278EA546368013363603BE07C2BC3
:102F2000EDD1B9F1000F00F06181002D00F0618159
:102F30002368013BA3EB090305F80930226818EE6A
:102F4000100AA2EB0A0205EB0A01FFF75FFF50E14E
:102F5000737833B90026304603B0BDEC028BBDE870
:102F6000F08F276843F02000642807F1010205D0A4
:102F700023F0040343F02003732B0ED1CDB10523BE
:102F80002260EB5523685A1C22607278EA54636809
:102F9000013363600E4601367DE755B1012322609F
:102FA000EB5570782668F3182360F6F75CF9A8559E
:102FB000EDE7BB1C2360EAE7BB1C2360ABE7531CB7
:102FC00017462360002DA6D00223AB54A3E7276841
:102FD00072787B1C5E2A236015D10DB10423EB555A
:102FE000B11C2368013323606368013363600E46BC
:102FF0004FF0000831785D290AD1002DCBD0EB19B4
:1030000083F80180C7E7002DEBD00323EB55E8E7F9
:1030100000299FD023685C2903F1010225D1019387
:10302000711C05B370782260F6F71DF9019BE85416
:103030004B782D2B03D18B785D2B18BF02310E46B8
:10304000236816F8010B5C2803F1010215D10193E6
:103050008DB148782260F6F706F9019BE8540136F5
:1030600008F10108C6E72260E2E722600DB132787C
:10307000EA543146DCE72260F1E722600DB10A78BC
:10308000EA540E46EBE773783F2B174627D1B37807
:103090003A2B24D1002302369846701C009A0193E3
:1030A0002146FFF7E1FE064600283FF453AF0278C1
:1030B000292A7FF44FAF019B002B3FF46CAF2368AC
:1030C0002DB35A1C22607E22EA5423684FEA480836
:1030D0005A1C08F10108226005F803801BE7A36869
:1030E00003F10108C4F8088075B1531C23607E23E6
:1030F000AB5423685A1C22604FEA4802EA546368C2
:10310000013363600123C8E702322260F7E702332C
:1031100053E72268BA423FF41DAF2DB1B81CD21B51
:10312000E9192844FFF772FE23680233236073789D
:103130003F2B07D10DB16223EB55013635B96368DA
:1031400001332CE0002DFAD005F807B02368EA1906
:10315000023BDF1B5770F2E7BA423FF4FBAE2DB1E2
:10316000B81CD21BE9192844FFF750FE236802332C
:1031700023603DB16022EA542368EA18C3F1FE03DC
:103180003B44537023680233236073783F2B09D18B
:103190000DB16223EB55013645B9636802332768E8
:1031A0006360F8E6002DF8D005F807B02368EA1947
:1031B000023BDF1B5770F0E7BA423FF4CBAE7378A7
:1031C0003F2B08D10DB105F802B001363DB9276893
:1031D000023727609FE6002DF9D06223AB542368A5
:1031E000EA18C3F1FE031F445770F0E7002D7FF487
:1031F000A5AE2368DA1C226015B12B4460229A70B8
:10320000D4F8009009F101032360002DC5D005F822
:103210000AB0236805EB0A02023BA3EB0A035370D2
:10322000BBE72268531C2360002D88D05023AB5489
:1032300085E7531C2360002D81D05123F7E7000060
:103240002DE9F04F2DED028B0D4608EE103AD1B06E
:1032500016468346002802F012830968F9F720FD1C
:10326000031E0293C2F20F832B6803442B60DBF82A
:103270000080B8F1000F0BD1584618EE101AFAF77B
:10328000F0FB6FF0060051B0BDEC028BBDE8F08F93
:10329000DBF80470002FEFD098F8004098F81C205D
:1032A000002C3CD1032A4FF009010CBF4FF011094B
:1032B0004FF0200939A8CDE93934CDE93B49F9F778
:1032C00095FC386098F81C30032B0CBF05210321B6
:1032D00039A8F9F78BFC07F1180A7860DBF8BC37DE
:1032E0009C420CDB4FF0000ADBF8C4379A4580F2B1
:1032F000C780902303FB0A740023039391E0AAF193
:103300001003012139A80393F9F770FC039B43F8DC
:10331000040B5345F5D101340AF1100ADEE7032A04
:103320004FF008010CBF4FF009094FF01109399314
:1033300039A80023CDE93A33CDF8F090F9F756FCDF
:10334000386098F81C30032B0CBF0121022139A8EA
:10335000F9F74CFC7860C5E70C2139A8F9F746FC71
:103360000921A06239A8F9F741FC0821E06239A8D7
:10337000F9F73CFC206398F80030002B0CBF0421C7
:10338000092139A8F9F732FC0121606339A8F9F75E
:103390002DFCA063002855D0022139A8F9F726FC9E
:1033A0000121E06339A8F9F721FC0521206439A83F
:1033B000F9F71CFC0521606439A8F9F717FC002314
:1033C000E364A064032139A8F9F710FC0321206508
:1033D00039A8F9F70BFC0321606539A8F9F706FC59
:1033E000E36BA0652BBBC4E90A336363E36DC3F1F0
:1033F0001403236698F80030002B3FD1012139A82F
:10340000F9F7F4FB6066012139A8F9F7EFFB012118
:10341000A06639A8F9F7EAFB039BE0660133039342
:103420004834DBF8BC37039A9A4295DB0AF1010A6B
:103430005AE7022B04D1236C13B90823E365D5E7BF
:103440000723FBE7C4E90F00052139A8F9F7CEFBF4
:103450000521606439A8F9F7C9FB0521A06439A8E2
:10346000F9F7C4FB0421E06439A8F9F7BFFB032195
:10347000E06539A8F9F7BAFB2066BBE70020C1E791
:103480003B68CBF8D8372B684B442B60029B03EB8F
:10349000090433681B1B3360DBF8B827DBF8B0374F
:1034A00072B1002B59D1DBF8CC2733689A4264DD26
:1034B000584618EE101AFAF7D4FA4FF0FF30E2E649
:1034C000002B4AD10123CBF8B037D5F80080D6F8CD
:1034D00000A0A8EB0404474651463846FAF7D5FA4F
:1034E000002807EB000324DB395C227891421BD1D2
:1034F00059786278914217D1A1789A784A4012F0AF
:10350000FC0F11D18F0748BF03F1FF33A3EB080372
:10351000002BCBF8B4370FDA584618EE101AFAF72A
:10352000A0FA6FF00200AEE60330DF1CAAEB000A3F
:10353000D2E74FF0FF33EBE7029ADBF8C4171A44E7
:103540009144DBF8C027DBF8C83702FB09F2D20050
:103550004B4392FBF3F2CBF8B827DBF80030DBF8F3
:10356000B4273BB15B69003B18BF01231344CBF880
:10357000CC3798E74FF0FF33F8E7DBF8DC07DBF8F0
:10358000D8370BF11C01984208913EDBC11A1A464C
:10359000089B19441846FFF739FC089BDBF8D8074D
:1035A000DBF8CC2729681844FEF708F8DBF8CC17BD
:1035B000DBF8D8270A44CBF8DC272B680B442B60B8
:1035C0003368DBF8CC279B1A3360DBF8DC37DB0091
:1035D00011930BF5FC6319934FF0FF331093002305
:1035E000CDE905330293DBF8C437029A9A4282F29E
:1035F0004E81902353431793059B0493199B149377
:10360000179B13934FF0000AE4E3089B29680344D7
:103610001846FDF7D3FFDBF8CC17DBF8DC270A44AC
:10362000CBF8DC272B680B442B603368DBF8CC2706
:103630009B1A584618EE101A3360FAF712FA6FF018
:10364000010020E6B8F1000F00F0A382DBF804309F
:103650000393002B00F09D82DBF80840002C00F063
:103660009882089B23930023CDE92433069A119B6B
:103670009A18D31D48BF02F10E03DB102693069B58
:103680001BB1194623A8F9F7B1FA029B98F800601C
:1036900090225343482202FB0A32039B1A44536B85
:1036A000D16B002E40F03E819D4810F8135000EB86
:1036B000430302295F785CD1D2F84080B8F1000F53
:1036C0000DD0049B04EB0308294623A8F9F78EFAD2
:1036D0000136082E08F8010BF6D14FF00308059BC0
:1036E0003E2606FB0A3608EB48031E4426440DF12D
:1036F0008C0929464846F9F779FA2946F075484673
:10370000F9F774FA294630764846F9F76FFA08F166
:103710000108B8F1060F707606F10306E9D1049BA3
:10372000E61839464846F9F761FA394686F829001D
:103730004846F9F75BFA394686F82A004846F9F711
:1037400055FA08F10108B8F10C0F86F82B0006F1C4
:103750000306E6D1029A7C235A433E2303FB0A2345
:103760001C44002384F83D3084F83C3084F83B301E
:103770001AE0029B002B4BD13E2303FB0A44029E1E
:10378000A1460DF18C0829464046F9F72FFA01367B
:103790000B2E09F8010BF6D139464046F9F726FA07
:1037A000A0550136152EF7D1029A90235A4348238B
:1037B00003FB0A23039A1A44936A149A1360239A08
:1037C000089BD31A259AC2EBC302D31002F007025A
:1037D0000A92069A14980A99C2EBC3020A4450F856
:1037E000041B1490881A0390089818440E9011989E
:1037F000002BA0EB02021A9202DB884280F2D081F9
:10380000584618EE101AFAF72CF96FF007003AE54F
:103810004FEA0A13039A083302EB0308D658D6B1CD
:103820003E2303FB0A430622109813F8011B195488
:10383000013AF9D1D8F80430D3B9049B062604EB39
:103840000309294623A8F9F7D1F909F8060001363A
:103850000B2EF6D11FE0049B04EB0309294623A895
:10386000F9F7C4F90136062E09F8010BF6D1E1E7A4
:10387000029D3E2303FB0AF37C20E21800FB053384
:10388000234491799971D179D971117A1972517A48
:103890005972927A9A72D8F808302BB33E2303FB00
:1038A0000A430B330B22109813F8011B19540132F1
:1038B000102AF8D1D8F80C3023B33E2303FB0A4377
:1038C00010331022109813F8011B19540132152AD5
:1038D000F8D1029A7C235A433E2303FB0A231C445B
:1038E00000236375A3755FE7049B0B2604EB0309B4
:1038F000394623A8F9F77AF909F806000136102E9F
:10390000F6D1D7E7049B102604EB0308394623A819
:10391000F9F76CF908F806000136152EF6D1D8E74C
:10392000908B0600D8F8206016F0010603D0BAF19B
:10393000010F00F0A580B3F5C87F6CDA18110522DD
:1039400090FBF2F2279202EB8202821A2892002068
:10395000C3F3810203F0030329922A93024603462C
:10396000022940F0C280029D4FF0900C0CFB05FC38
:103970004827039D07FB0AC72F443F6C002F08BF51
:10398000012102EB4202854F114417F821203992A0
:1039900007EB81014A783A928A783B92CA783C9246
:1039A000A6B1BAF1010F11D127AE04F1FC0239A979
:1039B00004F5867756F804CB42F804CB51F804CBD3
:1039C000C2F80CC0BA42F5D1C4F8F80002999022AE
:1039D0005143482202FB0A1203990A445366D36BEF
:1039E000022B40F0CC80176C002F00F0A980049BC4
:1039F0000026E718279923A8F9F7F8F80136062ECC
:103A000007F8010BF6D103230127059A4FF03E0971
:103A100009FB0A258CE0B3F5FA7F12DAA3F5C87327
:103A200098100522B0FBF2F2279202EB8202821A72
:103A300003F003030020289229932A9003460122D1
:103A40008EE7A3F5FA730322B3FBF2F202EB420016
:103A50001B1A0298039D27924FF0900C0CFB00FC60
:103A600000274820CDE9297700FB0AC02844289385
:103A7000006C10B1CDE928233846012302226FE7FC
:103A8000B3F5B47F03F001004FEA630210DA242794
:103A900092FBF7F307FB13220627279392FBF7F31A
:103AA00007FB13222893002329922A93032257E726
:103AB000F32A0CDCB43A13112793C2F38103289341
:103AC00002F00302002329922A93042248E7F43AE1
:103AD0000323B2FBF3F3279303EB4303D21A002330
:103AE0002892CDE9293305223AE7002149E727AB9F
:103AF00023A853F827100791F9F778F8079930753C
:103B000023A8F9F773F80799707523A8F9F76EF8E9
:103B100008F10108B07539AA08EB090352F827101B
:103B2000884506F10306E2DB0137042F3FF412AEAD
:103B300003EB43062E44994626444FF00008EAE77B
:103B40003B4662E727AB23A853F82610F9F74EF857
:103B500008F8010B013755F826108F4207EB0903CF
:103B6000F0DB0136042E0DD1029A7C235A433E230A
:103B700003FB0A231C440023A375637514E600238A
:103B80001E4639AD9946049B09EB0308A044002763
:103B9000E1E7069B0A934FF0FF331AE6198B060004
:103BA000DBF80040002C00F0B581DBF80430069310
:103BB000002B00F0AF81DBF80830002B00F0AA8169
:103BC000DBF80C00002800F0A581039B002BC0F25D
:103BD000A181029B616B90255D434822069B02FBFD
:103BE0000A551D44AB6B002B00F02081EB6B022BC0
:103BF00040F01C812B6C002B40F00081EB6D032208
:103C0000013393FBF2F301EB4303B3F92E2002EBF4
:103C100042024FF41071029B90245C43482303FB43
:103C20000A43069C2344DC6A6300B3F5107FA8BFF7
:103C30004FF410739342D4BF3A933A9200EB8A0246
:103C40000793169202F590528B42D4BF3B933B915F
:103C50003C9307990023399311604FF4106202FBE3
:103C60000A020F9239AA0D920A9A0B920C930E9A9D
:103C7000139B0892069A4033D3181B930D9B1C6824
:103C80000C9B01330C930D9B53F8045F0D932D1B7C
:103C9000002D40F36F82039B002BC0F23B810C9AF6
:103CA0001B9B089953F82260B44B03EBC6031B79A6
:103CB00009930B9B09985B4213F007031EBF11F891
:103CC000017BC3F1200207FA02F20F9F08BF1A46D8
:103CD00007EB8404002840F0BB80231D002244F839
:103CE000202043F8202002308542F7DC13460B9A4F
:103CF00008991A4401EBE20102F007020B92039AC1
:103D00000891D31A03930C9B032BB7D1039B002B71
:103D100040F3B282029B079D90225A43482303FB43
:103D20000A23069A1A444FF00009D36E944A52F8B7
:103D30002300944A52F823600B9B5B4213F0070365
:103D400017BF11F8014B0899C3F1200204FA02F2DF
:103D50000F9C04EB85040694039CC6F12006A4EB9B
:103D60000305079C0796884EC4F50F74304408BFBE
:103D70001A464F4601340990BC4200F30182169B5B
:103D800003F5905213681F4417600023B7F5107FA6
:103D9000C0F27482039A0B9B134403F0070206924D
:103DA000089A02EBE303139A48321392049A3E32C4
:103DB00004920E9A9B1A00F1AD800E9A1A44089252
:103DC0000A9AC2EBC303069A13441A9AD31A1193A0
:103DD0000AF1010ADBF8BC37DBF800809A45FFF6F0
:103DE00031ACB8F1000F40F05182584618EE101A6D
:103DF000F9F737FE6FF00900FFF745BA23785BB992
:103E0000029C9023634302FB0A32069B1A44D36D43
:103E1000013331F91320FCE6B1F93630B1F9342021
:103E20009A1AB1F90C3003EB4202F2E6029A90239F
:103E30005343482404FB0A34069B1C44E36D246E60
:103E4000013331F913202344013331F91310E2E631
:103E50004E4F57F826C04E4F07EB4C001190039879
:103E6000A0EB030E0998012840F0948037F81C60FD
:103E700006F00F064FF00008C6F12006BEF10F0F46
:103E800051DD0F46C3F1180017F802CB49780CFA40
:103E900000F0C3F1100C01FA0CF101430A43103396
:103EA000AEF1100E394604F1080722FA06F0119C13
:103EB000013034F81000040B10F0F00F02FA04F295
:103EC000A3EB103318BF02F00044C0F3031C1EBF65
:103ED000520003F1FF3344EA0C0C10F4706FC0F38E
:103EE00003241FBF03F1FF3302F0004020435200C0
:103EF00008BF204643450DDB023D002D47E902C0C7
:103F00003C4635DCA3EB0803039A7344D31A002B19
:103F100080F23181584618EE101AF9F7A2FD6FF0C1
:103F20000800FFF7B0B90EEB03000028F2DDBEF188
:103F3000000FC1BF11F8017BC3F1180C07FA0CF791
:103F40003A43BEF1080FC1BF11F8017BC3F1100362
:103F500007FA03F31A434FF00047431E47FA03F3EF
:103F60001A404FF00B0800F10B034FF0000E9AE7D8
:103F70000A2B07F1080798DC80E700BF2C690700CF
:103F80003892070030920700409207002C6A070021
:103F9000AC6A07000998871E012FBBD8BA48119F49
:103FA00050F836C0002012900CF101001590CCF1B1
:103FB00020001890BEF10F0F2ADD8846C3F11806C5
:103FC00018F8029B497809FA06F6C3F1100901FABC
:103FD00009F131430A431033AEF1100E41460A2B6A
:103FE000E8DDB7F8008008F00F08C8F1200622FAD3
:103FF00006F6013637F816605FEA16392FD107EB5F
:104000004607A3EB080302FA08F226463446E6E721
:104010000EEB0306002E7FF77DAFBEF1000FC1BF90
:1040200011F8018BC3F1180908FA09F842EA0802ED
:10403000BEF1080FC1BF11F8018BC3F1100308FADC
:1040400003F31A434FF00040731E40FA03F30B20B2
:104050001A40129006F10B034FF0000EBFE7C6F3B3
:104060000318B8F10F0FC6F30326A3EB090302FAF6
:1040700009F2374627D10998032827D1159803EB71
:104080000E09002E18BF0130484580463FF742AF69
:104090009845A9EB030E56DCBEF1000F0ADA734413
:1040A00003F1FF3E4FF0004040FA0EFE02EA0E021E
:1040B0004FF0000E189822FA00F808F10F08A3EB51
:1040C0000C0302FA0CF2B8F1000F05D002F000491F
:1040D00049EA08085200013B0F2E21D10998032814
:1040E00043D1159803EB0E0948453FF713AF1598D8
:1040F0009842A9EB030E30DCBEF1000F08DA7344DE
:104100005E1E4FF0004040FA06F632404FF0000EBF
:10411000189822FA00F70F37A3EB0C0302FA0CF2FF
:1041200027B102F0004637435200013B1298834208
:10413000FFF6F0AE2646023D002D46F8088B67607C
:1041400015DD119F62E711F801EBC3F118000EFABB
:1041500000FE42EA0E0208339AE711F8016BC3F140
:104160001807BE4032430833C1E73746D9E7129AF1
:104170009B1AC9E60023039A93427FF7B8ADC9E6BC
:104180000F2D57DD0E46C3F1180016F802CB497803
:104190000CFA00F0C3F1100C01FA0CF101430A43D0
:1041A0001033103D3146069E1036079822FA00FC67
:1041B000099810F80C004FEA101C02FA0CF210F0EB
:1041C0000808A3EB10131FBF02F0004803F1FF33F0
:1041D000520048F0010810F0040E1FBF02F0004E1C
:1041E00003F1FF3352004EF0010E10F0020C1FBF1E
:1041F00002F0004C03F1FF3352004CF0010C10F0C0
:1042000001001FBF02F0004003F1FF3340F0010046
:1042100052004B45FFF6B3AD0437A74246E9048E82
:1042200046E902C00696BFF6A7AD092B06F11006B7
:10423000BBDCA1E5E81800287FF7A1AD002DC1BFC8
:1042400011F8016BC3F1180C06FA0CF63243082D75
:10425000C1BF11F8015BC3F1100305FA03F31A4360
:104260004FF00045431E45FA03F31A404FF00A0988
:1042700000F10A03002596E7002780E50F9A42F82F
:104280002730013782E500BF2C690700DBF8047096
:10429000002F3FF4AAADDBF808300793002B3FF462
:1042A000A4ADDBF80C90B9F1000F3FF49EADDBF844
:1042B00010A0BAF1000F3FF498AD09F590530A939E
:1042C000029B179A7C246343503216931744079B32
:1042D000169A13440C93002354460B93DBF8BC3717
:1042E0000B9A9A424EDBD8F82030002B40F06881C0
:1042F000D8F820305A10039240F0AA81D8F8203024
:10430000D90740F1A68209F5905298F8005010683C
:104310005B100493DAF83033002D40F09783002BC4
:1043200040F0DB81DAF84443D8F83420DAF82C5333
:1043300009930134013532F91410049EAB4A079FEA
:10434000A0EB010A1C2000FB0622059E0A923E36C5
:10435000BE190E96049FA64E002206EBC7060392D6
:104360000F96AC4203DABAF1000F00F3CF81079C3D
:1043700005985534201814909D4C049804EBC00007
:1043800015905FE20B9B4FF4106202FB03931393B3
:1043900057F8143C022B46D157F8106C002E46D02B
:1043A00098F800300322002B03920CBF0826062643
:1043B00000233993BB69D8F8202001335B001293A6
:1043C00057F8203C520818BF023B9A1C17920C9ACF
:1043D0000E92C3F1D0030022099215460492149361
:1043E000B54226D10023C4F81833399AC4F81C33D7
:1043F000C4E9C833C4F82833039BC4F82C230B2B1F
:104400004BDD0998F9F736F80A9B013898600B9B49
:1044100001330B930A9B04330A930C9B3E331834ED
:1044200048370C935AE70D2303931626C0E70396EB
:10443000BEE76B1C0F93D8F8343003EB4502B2F99A
:10444000021033F915208B1A0E9A0D9312F8013BC6
:104450000E927A6922B1674A691C0A4412F8012C4B
:1044600004981399134401EB8001129A149802FBEB
:1044700003030D9A0846F9F709F8049A0D9B1344B3
:10448000049300B13995099B049A034309930A9B4D
:104490001B689A42A6DA0F9DA2E7039B3B93CDE9E6
:1044A00039330C9B14331893039B0F9301330F9AEA
:1044B0000393D8F83430159703EB42030026B3F981
:1044C0003010B3F92E20039B8A1A189903EB43038B
:1044D000CB181493930004990E93139B03EB81055F
:1044E000179B0D95C3F1D20351461A93159850F8B6
:1044F000043B1590149810F801CB14901A9800EB17
:10450000C303129800FB0C330D98CDE91B12F8F78A
:10451000BDFFDDE91B1220B10DF1E40C0F9B4CF83F
:104520002630099B03430993DDE90D30013603442E
:10453000032E0D930144D9D1049902EB420319448F
:104540000346534404911E460AEBC20100239A42DB
:1045500005F10C0526DC0A9B049A1B689A4202DAD4
:10456000039B0D2BA0D10A9B1A46049B136057F89E
:10457000103C002B14BF02230123C4F81833399BCD
:10458000C4F81C333A99C4F820138B423B9AC4F800
:104590002423B8BF0B469342ACBFC4F82833C4F8F9
:1045A00028232EE75AF8230045F80C0C56F8040B84
:1045B00045F8080C51F8040B45F8040C0133C6E724
:1045C00041F2082359F80330002B06DD41F20C2399
:1045D00059F80330002B3FF78BAE09F59053064C8A
:1045E00019686FF04040002310E000BFE466070048
:1045F000D466070060190700010000C059F82320A5
:10460000B2F1404F19DC49F8234001338B42F5DB0E
:1046100041F20423674D59F80300002209F51063A5
:104620006FF040448242BFF663AE1968B1F1404F6B
:1046300009DC1D6001320433F4E7B2F1804FA8BFFA
:1046400049F82300E1E7B1F1804FA8BF1C60F1E712
:10465000D80737D5DAF83023D8F834304ABBDAF83F
:104660004423013233F912300022A9F104010392EC
:1046700015461646AB427FF741AE51F804CFD1F84C
:1046800000490CEB0407ACEB04040F60C1F80049CF
:10469000B44687EAE77CACEBE77C039840EA0C0081
:1046A0000390374684EAE477A7EBE4773A43013591
:1046B000E0E7DAF8402303EB4203B3F9303003EBD1
:1046C0004303D1E741F2042309F5905259F803104E
:1046D00013688B42B8BF0B46C6E7013B012B10D8CD
:1046E000DAF82823DAF8401301320992D8F8342096
:1046F00002EB41024B1CB2F930102C4601EB410198
:104700001BE609952B462C46294616E60E9E365D7D
:10471000072E274623D10498274E56F830C00F980D
:104720004068D8F834600C9006EB470E36F91760F5
:10473000BEF902E00B91AEEB060001340D9009EBDF
:10474000810700260D980B99B0423144AAEB060E62
:1047500003DD56450AD14FF0000EF24601E60A98F5
:1047600050F826C08669A6EB0C00DAE757F8041B60
:104770000C9880FB01E18900C7F8FC184FF0000E8F
:1047800081EAE17EAEEBE17E57F8041C42EA0E02BC
:104790008CFB01E1890047F8041C4FF0000E81EA10
:1047A000E17EAEEBE17E039941EA0E010391013611
:1047B000C8E700BF010000C0D4660700149803EBEF
:1047C00043060644002516F8014B072C40F0D5801F
:1047D00004989D4C54F8304027A840F8254015987F
:1047E000446839A840F825400135032DEBD1D8F8AD
:1047F00034400791013304EB430504EB4C0CB5F94D
:104800002E50BCF92E40281B0B9039980C902798FD
:104810000D903A980E9028980F903B981290002790
:104820002998139009EB8104BC46079807EB4701D0
:1048300001440B98B84205DDBAF1020F04F10C04F3
:1048400000F3A580099883429C4602DABAF1020F70
:10485000B4DCD8F82030E3B10398F8F70BFE41F24E
:104860000823013849F803001046F8F703FE41F227
:104870000C23013849F8030041F2042209F5905154
:1048800059F8023008688342B8BF03460B6049F804
:10489000023000230393039ADBF8BC379A42C0F23C
:1048A0001182029ADBF8C847544318EE102A5C4381
:1048B00002EB4404DBF80C20002A00F0D787DBF879
:1048C00014200392002A00F0D187DBF81850002D45
:1048D00000F0CC87022B02F5D85303F1180307939D
:1048E00040F03A8605F1800302F5D85907EE903A78
:1048F0001746002605F5085809F11C09079B1B6897
:10490000009306F0010A3846D8F80020534629469D
:10491000F8F79CFAD9F80030009317EE901A07F5D3
:104920001060D8F800205346F8F790FAD8F8003015
:104930004FF4886101FB0A3104EBC61005EB8101DD
:10494000F9F7B6F8D8F800300136A3EB0A0303F004
:104950000703122EC8F8003007F18007CED1029B62
:1049600001330293059B7C330593199B08331993FC
:10497000109B7C331093FEF736BE0A9850F82470D3
:1049800027A840F825700A988469E41B29E754F8A1
:104990000C1C0C9880FB01518900C4F8F418654682
:1049A00081EAE175A5EBE17554F80C1C0D9880FBCC
:1049B00001618E0044F80C6C614686EAE671A1EB59
:1049C000E67154F8086C0E9880FB06E6B000C4F857
:1049D000F808664680EAE076A6EBE07635430F9865
:1049E00054F8086C2A4380FB0656B60044F8086C5D
:1049F000654686EAE675A5EBE67529430398129DA0
:104A000008432E4654F8041C86FB01518900C4F863
:104A1000FC18654681EAE175A5EBE175139954F838
:104A2000046C2A430D4685FB0616B60044F8046C58
:104A3000614686EAE671A1EBE67101430391AAF1B2
:104A4000030A0137F1E600BFD4660700079A04990C
:104A5000D2F8F82001EB4202A04901EB8212099240
:104A6000079A002402F1FC0102F5867C4FF0010E4A
:104A700051F8042B39AD0EFA02F2CE6805EB84072B
:104A8000013A0025B54251DB002EA8BFA4198C4580
:104A9000EED10121002B40F08580D8F8342003931B
:104AA000CDE94E11DAF84413DAF82C430B940131B6
:104AB0000DF1E40E32F911701A46059B03F13E0424
:104AC000079B2344C51B0C930498854B03EBC00341
:104AD0000D930B9B8B42FFF6BCAE0C9B5C5C5EF8AF
:104AE00021309C420E4625D17D4B049853F830303E
:104AF0000A930D9B5B680793D8F8343003EB4604A8
:104B000033F91630B4F90240E41AAC4201F1010164
:104B1000A8BF2C4609EB87064FF0000C64451CDC4F
:104B2000002CA8BF3F192D1BD3D192E647F8042BC8
:104B30000135A7E7631C5B1014F00104099814BF4A
:104B40004FEA830CA44650F80C000A901CB99B0055
:104B50000998C358CFE70023FAE756F8043B0798B3
:104B600080FB03A39B00C6F8FC384FF0000A83EAE1
:104B7000E37AAAEBE37A56F8043C0A9842EA0A027E
:104B800080FB03A39B0046F8043C4FF0000A83EA35
:104B9000E37AAAEBE37A039B43EA0A0303930CF15B
:104BA000010CBBE70AF54773169C0A93079B4591D6
:104BB0005534234404991C46494B002203EBC1039E
:104BC000039294460D930A9B1846996950F8043B4A
:104BD0000C93D8F834300A9003EB41034D1C1E8E21
:104BE000032316FB03C60C9BAB4207DA0CF1010C46
:104BF000BCF1030F04F10104E5D12AE605EB4503FE
:104C00002F4614F803E039AB53F825108E451FD119
:104C1000334B049953F831300B930D9B5B6807932A
:104C2000D8F8343003EB47030135B3F93010B3F94A
:104C30002E3009EB8607C91A4FF0000E714507F1B7
:104C40000C071ADC21EAE17101EB41010E44CAE7CD
:104C50000EF101031EF001014FEA6303099814BF2E
:104C60004FEA830E8E4650F80E000B9019B99B0048
:104C70000999CB58D3E70023FAE757F80C3C07987B
:104C800080FB03A39B00C7F8F4384FF0000A83EAC7
:104C9000E37AAAEBE37A57F80C3C0B9842EA0A0253
:104CA00080FB03A39B0047F80C3C4FF0000A83EA0B
:104CB000E37AAAEBE37A039B43EA0A0303930EF138
:104CC000010EBBE7DBF8003063B9584618EE101A46
:104CD000F8F7C7FE6FF00A00FEF7D5BA1C670700A9
:104CE000D4660700DBF804200D92002AEDD0DBF833
:104CF0000C200492002AE8D0DBF81450002DE4D0F8
:104D00005A6B1B780398002B0CBF08230623122133
:104D100032F91330029A93FBF1F30C9390235A4328
:104D2000482303FB00230D9A1344DA6B022A00F098
:104D3000E380049A00F5906352F8236040F2262342
:104D40009E42CFBF2023073696FBF1F14B1C0B93FD
:104D50000B9B5A1E039BDFF8A49407924FF4106A32
:104D60000AFB03FA049B534414930799002900F3A8
:104D7000CB80DDE9033101EB830000F59054122173
:104D800023680D9E4A4308329A42B8BF1A462260F1
:104D9000113292FBF1F31593039B05EB83030A9306
:104DA00003F5D85341F608321B681A930A9B9B58A7
:104DB000169341F610320A9B9B581793039B4FF0B2
:104DC000480909FB03F1029B90225343CC18344459
:104DD000246C002C0C9C08BF00240C9441F2082485
:104DE0000059129003984FF4906404FB005404F5AA
:104DF00090501B9005EB0A0013901298C0F1070029
:104E00000990129806280998C8BF002007EE100ADA
:104E1000139800F508600F9014983C300E90CDE97F
:104E20001E911B980790CDE9202300200490824614
:104E30000B9B534500F3228123EAE377149A1E9BD0
:104E4000079703FB07291B9B242404FB07331493B8
:104E500003EB0408139B03EB87030B93A8F12403D4
:104E600007EE903A079A159B934200F32382BB42C8
:104E7000A3EB07004FF02404149B04FB00F4AEBF27
:104E80000646002400263E4423441C46B0463546D0
:104E900000271A9BAB4200F30183B342B8BF3346ED
:104EA0001E4600221F2E40F34583049B002B00F07A
:104EB00051830022049B002B80F247830A9B0299B6
:104EC000039803F5D853C3F800809023594348232F
:104ED00003FB00130D99194441F60830CB6B0A9976
:104EE0000B5041F610300C9B0B50531E41F61832FC
:104EF0008B50039B0133CDE41A6C1AB10C9B0B93BE
:104F00005A1E27E70B9225E75C6CB04E214686FBC4
:104F10000171AF4E9F6C304686FB07C7C91B490025
:104F20005964AA4E996C86FB017180FB04740C4491
:104F300064009C641C6CA74E214686FB017100F145
:104F4000AF6000F5A430DF6C9F3080FB07C7C91B42
:104F500049001964D96C86FB017180FB04740C4410
:104F60006400DC64DC6B9C48214680FB01719B4E35
:104F70001F6D86FB07C7C91B4900D963196D80FBEC
:104F8000017186FB04740C4464001C6500F18960A7
:104F90009C6B00F5FA20214600F50D7080FB017135
:104FA0008F4E5F6D86FB07C7C91B49009963596D1A
:104FB00080FB017186FB04740C4464005C655C6BCF
:104FC000214689FB0171874FD3F858C087FB0CEC51
:104FD000A1EB0C0149005963996D89FB01C187FB65
:104FE00004C40C4464009C651C6BDFF814C22146A9
:104FF0008CFB01717C4FD3F85CE087FB0E8EA1EB3C
:105000000E0149001963D96D8CFB01E187FB04C4D3
:105010000C446400DC65DC6ADFF8E8C121468CFBE7
:105020000171724FD3F860E087FB0E8EA1EB0E0189
:105030004900D962196E8CFB01E187FB04C40C4462
:1050400064001C669C6ADFF8C0C121468CFB0171BC
:10505000674FD3F864E087FB0E8EA1EB0E01490089
:105060009962596E8CFB01E187FB04C40C440799DB
:10507000640001395C660791483376E6219A1F9BEC
:1050800013440D9A1344D3E90F731BB10C9B534582
:10509000C8BF0027DDE916325245C8BF0023984635
:1050A0000F9BA3F508631893129B062B2FAB7CDC98
:1050B000079A0E9C002602F124003246A168099D41
:1050C0002941891A62682A418E1B521A5E6243F88E
:1050D000042950F8041D2941016007998142A4F177
:1050E0000804EBD1309B5B103093279B27A85B1003
:1050F0002793F8F79BFA30A8F8F798FA57EA0804CC
:1051000000F0848039AE424607983146F8F764FBD8
:10511000209B384803FB07004AAB00241D93364B05
:105120001C9300F1480922460DF1BC0E3146A04601
:105130001C9DDEF8243055F804795EF804691C954E
:1051400087FB03C3079DC3EBA60C03EBA60345F83F
:10515000223050F822608CFB06361D9D51F822301B
:1051600059F8047D334455F804691D959B008CFB68
:105170000757189D3E44D701B600EB516FF07F05ED
:1051800005FB02F70F9DEE51474683EAE377A7EB55
:10519000E377434686EAE673A3EBE67301321F43E7
:1051A000092A44EA0704C3D16DE00E980024224680
:1051B000A0F148068168891A426808380C1B521A07
:1051C00086425C6243F80429F4D18BE7F053C26D48
:1051D000AA0025BEE4EBDC70736E8D794A3FE3D7FD
:1051E0007611B7E82FFEE4F3C7A3C1FAC6BD2EFEC1
:1051F0005DC286FFD08B0700D0B60600B7206D7F5A
:10520000407EE47F63B2FC7F94C6FF7F079FA04E81
:10521000DFF8849220460DF1BC0CA646DCF8242071
:1052200059F804395CF8041983FB0282A2EBA1034C
:10523000D7F8008002EBA10247F8042BC8F1000167
:1052400056F8082BC91A81FB025203EB820256F86A
:10525000043C81FB03534142189D6A500F99C8EBEF
:1052600083030B50714682EAE271A1EBE271724650
:1052700083EAE372A2EBE3728038114310F5906F7A
:1052800044EA0104CAD117EE103A52460799189819
:10529000F8F72CFB049B204303430493079B243320
:1052A00007930F9B04330F930E9B48330AF1010AB7
:1052B0000E93BDE5DDE9163107988142C8BF002392
:1052C0001A46129B062B13DC17EE901A4B4609F177
:1052D00048041868099D284118605868284158609A
:1052E00051F8040B083328419C4241F8040CF0D1DA
:1052F00027A948460E92F8F723FA2DA909F10400D0
:10530000F8F71EFA33A909F10800F8F719FA0E9A0E
:1053100017EE900A39A9F8F75FFA29AA0E920B9AAC
:105320005C49002002F5C07639AB27AD0F901F967F
:1053300053F8046B0446B60086EAE674A4EBE67400
:1053400016609E681894B600044686EAE674A4EBDC
:10535000E674C2F8806151F8046BD5F80CE01B9438
:1053600086FB0EAE5E6904460EEB860686EAE674A0
:10537000A4EBE674DDF838E0C2F800631C94DEF8B4
:105380000CA08C6884FB0A6A1E6A04460AEB860637
:1053900086EAE674A4EBE674C2F880641D94AEF16C
:1053A00004044E69DEF800E00E9486FB0EAED5F8DC
:1053B00024A051F8044C84FB0A6ADE6AD6440EEB42
:1053C0008606044686EAE674A4EBE674C2F8006634
:1053D000D5F800C00E6A1E94043586FB0CEC0E9CBA
:1053E0008E68D4F828E086FB0EAE9E6BF4440CEB7E
:1053F0008606844686EAE67CACEBE67C189CC2F81E
:105400008067A6461B9C4EEA040A1C9C4AEA040AD2
:105410001D9C4AEA040A1E9C4AEA040A0F9C4AEAB6
:105420000C0A44EA0A040F941F9C803294427FF4D1
:105430007FAF2D9B9B1048F8243C2E9B9B1048F877
:10544000203C2F9B9B1048F81C3C33A9A8F1180363
:1054500051F8042B921043F8042B4345F8D117EE72
:10546000103A079A0B9817EE901AF8F73FFA0F9B2D
:1054700003431846049B03430493079B013307939C
:105480000B9B043309F1480908F124080B93E5E468
:10549000D0CD0600F08C0700D0B60600DDE916314D
:1054A000A942C8BF00231A4639A92046F8F794F943
:1054B000139B03EB850105F00103099304F120031D
:1054C00045F3000A39A8A4F1040E4FF0000C0B9329
:1054D00003684FEA8309C1F800903B4689EAE97303
:1054E000A3EBE973079343688AEA83031A46099B8F
:1054F0001A4449EA02094CEA090CC1F88020B9466D
:1055000082EAE279A9EBE279079B4EF8047F43EA4D
:105510000902049B134304930B9B734500F108009D
:1055200001F58071D4D1BCF1000F18BFA846243416
:105530000135AEE4139B03EB86000023D901013350
:10554000122B4250FAD10136ACE4049B5B000132CD
:105550000493AFE42022B1E405F508531E344FF064
:10556000000A04930AF001030993079B049A1B683D
:10557000039800932946099B126800EBCA10F7F7BD
:1055800065FC049B09991A684FF4886303FB0123A7
:1055900005EB83074FF0000C55F82310FA6D4FF020
:1055A00000736046C1FB003C6FF07301C2FB013C1D
:1055B0004FF455797968BA6DC1FB093CB549C2FB16
:1055C000013C41F6D478B9687A6DC1FB083CB24918
:1055D000C2FB013C46F2B860F9683A6DC1FB003C81
:1055E000AE49C2FB013CAE4A3969C1FB023CAD4940
:1055F000FA6CC2FB013C7969BA6CC1FB003C45F214
:105600008401C2FB013CB9697A6CC1FB083C40F2E1
:105610002C71C2FB013CF9693A6CC1FB093C742155
:10562000C2FB013C4FEA936343EA8C1324F81E3C0F
:1056300007F580534FF0007219684FF4D0700023C3
:10564000C1FB002341F2040141F67C007958C1FB03
:10565000002341F2080149F2FC707958C1FB002394
:1056600041F20C0190487958C1FB002341F210012E
:105670008E487958C1FB002341F214016FF0B3004A
:105680007958C1FB002341F218014FF41270795888
:10569000C1FB002341F21C016FF013007958C1FBDC
:1056A00000234FEA926242EA8312A4F11E030A9396
:1056B000DFF8FCC1628004F122030B93DCF844E0C4
:1056C000D7F85C91D7F80031DCF840104FF0007249
:1056D0000020C3FB01204FF00073D7F800610021C8
:1056E000C6FB0E31CEF1000EC9FB0E20DCF8406087
:1056F000C9FB0631D7F80461DCF84C90D7F858E1C3
:10570000B046DCF84860C8FB0620C8FB0931C9F187
:105710000009CEFB0920DCF84860CEFB0631D7F843
:105720000861DCF85490D7F854E1B046DCF85060DA
:10573000C8FB0620C8FB0931C9F10009CEFB0920CE
:10574000DCF85060CEFB0631D7F80C61DCF85C90D9
:10575000D7F850E1B046DCF85860C8FB0620C8FB1B
:105760000931C9F10009CEFB0920DCF85860CEFBF5
:105770000631D7F81061DCF86490D7F84CE1B046F8
:10578000DCF86060C8FB0620C8FB0931C9F10009DC
:10579000CEFB0920DCF86060CEFB0631D7F814613F
:1057A000DCF86CE0D7F84891B046DCF86860C8FBDC
:1057B0000620C8FB0E31CEF1000EC9FB0E20DCF82E
:1057C0006860C9FB0631D7F81861DCF874E0D7F8D7
:1057D0004491B046DCF87060C8FB0620C8FB0E316F
:1057E000CEF1000EC9FB0E20DCF87060C9FB06315B
:1057F000D7F81C61DCF87CE0D7F84091B046DCF8C3
:105800007860C8FB0620C8FB0E31CEF1000EC9FB44
:105810000E20DCF87860C9FB06314FEA926242EA5A
:1058200080120A9820F8022F0A904FEA936343EA05
:1058300081130B9A22F8023D84420B920CF1400C2A
:1058400007F580777FF43AAF049B099A1B680AF149
:10585000010A9B1A049A03F00703BAF1120F1360AE
:1058600004F140047FF47EAEFFF779B8584618EE95
:10587000101AF8F7F6F86FF00B00FDF704BD6FF0A3
:105880000400FDF700BD6FF00500FDF7FCBC002033
:10589000FDF7F9BCD4F8FFFF7CAFFFFF3CB6FDFF7E
:1058A00078940400C44902004CE803002464FFFF1C
:1058B000108E070000F0030370B553EA010406D010
:1058C00002440346934213D003F8011BFAE722F087
:1058D00003039608034405469D420AD1910742BF3F
:1058E000002120F826100233D20701D500221A70B9
:1058F00070BD45F8044BEFE770B531220021064634
:105900000E480F4DFFF7D6FF1022FF210D48FFF77D
:10591000D1FF1022FF210C48FFF7CCFF0B481422C7
:105920000021FFF7C7FF0024AB680BB13046984752
:105930000134042C05F12005F6D170BDBC450120D1
:10594000B08C0600BD450120CD450120242F01204B
:105950002DE9F04FBA4B87B01B780093002B00F075
:10596000CC82B84EB84FB94B1C682378012B02BFCC
:10597000B74B8022C3F88420B4F80E801FFA88F851
:10598000B8F1000F18D0638A628961689BB202FB8C
:10599000031103A8FBF712FE638A2189DDF800805A
:1059A0009BB20133B3FBF1F201FB12339BB2638272
:1059B000E389013B9BB2E3812378012B02BFA44B17
:1059C00080225A60B8F1000F00F073829DF80D300C
:1059D000013B072B00F2248201A252F823F000BF02
:1059E000015A0300015A0300175F030067590300BF
:1059F000675903000B5A0300E75D0300315F0300A2
:105A00009DF80C00FFF778FFADE7924C9DF80C5025
:105A1000237843F00103237000233B619DF810308D
:105A200003F06002602AA14605D13368D90740F12E
:105A3000E58000BEE2E0402A0FD1874B002B00F04A
:105A4000DD80864B03B13B6104A92846AFF300809B
:105A50008046B8F1000F86D1D0E003F01F03012B80
:105A600000F03881022B00F05281002BDDD1002A9A
:105A7000DBD19DF81130092BD7D801A252F823F0C1
:105A8000BF5C0300AF5C03002B5A03009F5C030064
:105A90002B5A0300A95A0300E95B03002B5A0300A9
:105AA000D75A0300F15A030006AB13E903000022A2
:105AB000C7E9022287E80300694BD3F80014D3F842
:105AC00000040143C3F80014C3F858214FF48002C6
:105AD000C3F8042347E72378C3F340038DF80A3063
:105AE00001230DF10A0204A92846FCF7B1FD3AE7AB
:105AF00023789DF812A0C3F340029B0718D4BAF193
:105B0000000F15D02378DFF870B1019223F0300335
:105B100043F0100323709BF801300B2B16D19BF838
:105B200000309B444F4B9B45F5D34F4B00221A70DE
:105B3000BAF1000A237818BF4FF0010A6AF3410353
:105B4000237004A92846FCF741FD0CE7042B14D16F
:105B50009BF80530022B08D0082B14D0032B15D04E
:105B6000012B0AD14FF0030801E04FF000089BF829
:105B700002304B445A78FF2A0BD03368D8077FF5A0
:105B800054AF00BE51E74FF00108F0E74FF00208B4
:105B9000EDE783F80180019BADF80A30334B03EB4E
:105BA00048130DF10A02DB68594628469847002839
:105BB000E3D0BDF80A000828DFD95A4600235178FF
:105BC000052909D192F802C00CF07F0109EB4101CF
:105BD00001EBDC1181F8118011780B449BB29842E3
:105BE0000A44ECD883449DE7BDF81230190A032912
:105BF00047D010D8012918D002293FD0184B0122D4
:105C00005A65BFF36F8FBFF34F8F5A65BFF36F8F26
:105C1000BFF34F8FA7E60F29F0D1154B002BEDD026
:105C2000AFF300804388024601E0124A122304A920
:105C30002846FCF70DFD00287FF495AEDEE700BF97
:105C400028300120F0ED00E0242F0120F045012054
:105C500000E100E0BC450120000000000000000061
:105C6000007002400239070030220120B08C06008B
:105C7000000000000239070031380700B04ADA237B
:105C8000D5E7DBB2EE2BB9D00B2B3FF6CEAEAD4A4B
:105C900052F82320002A3FF4C8AE1378C7E7BDF8B6
:105CA0001230012BAAD1237843F0080348E7BDF84E
:105CB0001230012BA2D123786FF3C30340E723787E
:105CC000C3F340129B0803F002031343ADF80A30FC
:105CD000022306E79DF814100F298FD80C44617831
:105CE00003298BD82AB99DF811000A2806D00B2861
:105CF00007D004AA2846F9F729F99CE78DF80A206D
:105D0000EFE69DF81230002B7FF48FAE19E79DF877
:105D1000141011F0780C7FF488AE01F07F0004EBD2
:105D2000400404EBD1144FEAD11E94F811A04FEABD
:105D3000400B002A55D19DF81120012A27D0032AB3
:105D400047D0002A7FF471AE94F82120C2F34002BC
:105D5000ADF80A2004A90DF10A022846FCF778FCE8
:105D6000BAF1FF0F0BD0BAF1030F3FF65EAE04AAF3
:105D700051462846F9F7EAF8002818BF80469DF8F2
:105D8000103013F060037FF464AE3B6161E6BDF850
:105D90001230CBB950B16C4BC3F8181541F4807177
:105DA000C3F80C15BFF36F8FBFF34F8FD944CE44A8
:105DB0009EF821306FF341038EF821309EF8213098
:105DC0006FF300038EF8213004A92846FCF7FEFB90
:105DD000C6E7BDF81230002BF6D12846FAF71CFEB4
:105DE000F2E7E046BCE79DF81010584B01F07F0445
:105DF00003EB440303EBD1134FEAD11C93F82120AA
:105E00006FF3000203F1200083F82120002C48D119
:105E10003B789DF80C80059DBCEBD31F0FD02DB1B6
:105E20003368DB077FF59FAD00BE9CE5484B002B38
:105E30003FF499AD39464046AFF3008093E597F9BA
:105E40000030002B07DBB86800283FF48CAD4149D7
:105E50002A46FBF7B3FBBA68FB892A442B44BA6095
:105E6000FA889BB29A42FB8101D03F2D15D83B693D
:105E70006BB997F900300022002B1146B4BF2046C1
:105E80008020FCF707F900287FF46DADC8E739469C
:105E9000404698470028ECD1B0E64046FCF7AEFB00
:105EA000F1E75A7C032A2BD92B4B1B68DA0700D564
:105EB00000BE2A4C254BA27802F07F0103EB410380
:105EC00003EBD21393F8210010F0010515D104F56E
:105ED0000761402204F12000FCF7A5FE014660B1F5
:105EE000FAF746F948B10B4604F50762A17828464F
:105EF000FCF718F908B9F3F769FA07B0BDE8F08FB5
:105F0000174B9DF80C0003EB42139DF811209C6980
:105F1000059BA04727E5124D0024EB6913B19DF8BE
:105F20000C0098470134042C05F12005F5D11AE541
:105F3000049B002B3FF417AD0598984713E500BF6D
:105F4000283807005029070000700240BC45012096
:105F5000000000007C450120F0ED00E074260120E7
:105F6000B08C0600024840220021FFF7A3BC00BF0E
:105F70005C440120024840220021FFF79BBC00BF87
:105F80005C440120054B00225A831A609A831A71DF
:105F9000DA835A859A85DA85704700BF7426012016
:105FA00008B5134B4FF40B6200211846FFF782FC33
:105FB0004FF44241C180012101810821FF22017378
:105FC00000F130014271016100224FF48231034639
:105FD0004283428182834161C283027600F58660FA
:105FE000C3E908015A8583F828209A85DA8508BD17
:105FF0007426012002482C220021FFF75BBC00BF61
:10600000FC2F01200020FFF7F5BF0000044B002209
:10601000DA811A601A825A82DA831A845A847047A3
:10602000A03201200E4B10B54FF4D6720021184655
:10603000FFF740FC00F124020346426009489860E3
:1060400003F1A404C3E9054000220121DA81197398
:106050001A8219775A82DA831A845A8410BD00BFD3
:10606000A03201208000010030B50388A3F11002A6
:106070001F2A89B00C4606D88188228891421AD1FD
:10608000242B16D907E0A3F150021F2A0FD88188CC
:10609000228891420FD1503B9AB2072A0BD8072B86
:1060A00009D8DFE803F061087908084E0846242B78
:1060B00032D8102B01D80020B6E0113B132BFAD8B0
:1060C00001A252F823F000BF33610300B96103005D
:1060D000CB6103002D620300B7600300B7600300CB
:1060E000B7600300336103000F62030071620300B5
:1060F000B7600300B7600300B7600300B760030038
:10610000A7610300B760030025610300336103004A
:1061100037610300336103003A2BBCD14389A1F8F6
:10612000763006E000238088ADF800306946F4F749
:10613000EFF8012078E0002220881146F4F7EAF811
:10614000F7E7B4F87610C38841B9172B38BF172387
:10615000B3F5007F194628BF4FF400712088A4F8DA
:106160007610F4F7D3F9E4E722884FF6FF739A42EA
:10617000DFD094F85A30022BDBD183684E4A23F0EB
:106180007F4393424FF00105D3D184F87850F8F75C
:10619000BBFFC4E92001CCE7002320881A4619463A
:1061A000F3F796F9C5E7012500F1080184F874506A
:1061B0002088F4F79BF8BCE750F8083FE366436893
:1061C0002367002384F87430B3E704F108035022F6
:1061D00000211846FFF76EFB04F12403002104930D
:1061E00004F14003CDE90531A37800908B424FF6CE
:1061F000FF72A4F858202088304A03916B4618BFDC
:106200000A46CDE901110791F4F776F991E7037A8F
:1062100084F85B309BBB638BA4F8583001200223C9
:1062200084F85A3084F8790009B030BD028AA07829
:106230000121F3F751F9A0B1C288502A11D104F11C
:10624000080500F108012846FBF7B8F922460023AB
:1062500032F8400B2946F4F751F9638BA4F8583013
:1062600067E7002320881A461946F4F747F960E7E4
:10627000037A03F00F02012A05D81F2B03D800234D
:1062800084F85A3055E7B4F85820A0780221F3F783
:1062900023F938B9002320881A461946F3F718F96C
:1062A0000223EDE7C28800F1080103232088F3F7F9
:1062B0000FF90028F4D0EDE7022901003E14070091
:1062C0002DE9F04FA84BA94AD3F80003002385B06D
:1062D0001C4601251E4605FA03F1084209D052F872
:1062E000237037B10C4342F82360BFF36F8FBFF3C5
:1062F0004F8F0133192BEED1E7071AD50022114633
:10630000930003F1804303F51C330132082A5960DE
:106310009962F5D1944B59629964954BC42200213E
:106320001846FFF7C7FA4022027502720120FBF7F8
:10633000D7FCA60202D50320FBF7D2FC650213D5D9
:10634000894ED6F8005405F44073E805C6F80034C9
:1063500005D50420FBF7C4FC0123C6F82C35A9059C
:1063600002D50520FBF7BCFC824B814E234033B1A4
:1063700096F8C030002B40F0D380F3F74FF822029C
:106380003BD5794BD3F880E4D3F88424D3F8881430
:10639000D3F88C74D3F89054D3F894045FFA81FC4A
:1063A000D3F89814D3F89C341EF07F0F5FFA8EF860
:1063B000D2B2FFB2EDB2C0B2C9B2DBB201D1052A8E
:1063C0001BD04FF0000EADF806E08DF80D004FF435
:1063D000C06E8DF80E1001A80121ADF804E08DF813
:1063E00008808DF809208DF80AC08DF80B708DF8A3
:1063F0000C508DF80F30FBF741FC5D4FDFF86891D2
:10640000B84600254FF0010A4FF0140B05F10C03BC
:106410000AFA03F32342E9B21BD00BFB05930020D9
:10642000D3F80827182303FB0563D2B2587298F8F3
:1064300008C094457DD1DB88B8F804209BB29A420D
:1064400077D9002D70D1C9F84CA0BFF36F8FBFF37F
:106450004F8F0135082D08F11808D7D1464B23403E
:10646000002B5AD0404BD3F86C84C3F86C84BFF334
:106470006F8FBFF34F8F14F4806407D0D3F880443C
:10648000D3F880341B06C4F3C0145FD54FF0000A64
:10649000DFF8DC9000254FF0140B0123AB4013EA2A
:1064A000080FE8B201D1ADB9A4B12F4B0BFB0533F6
:1064B000D3F80416182303FB05635A8A11FA82F2F3
:1064C00092B25A825A8AB9F8101092B2914240D9C7
:1064D000FBF7BAFD0135082D09F11809DDD10024BB
:1064E00001254FF0180904F1100305FA03F313EA2C
:1064F000080FE0B203D15CB9BAF1000F08D009FB74
:106500000462B988D3889BB299422BD9FBF774FDFA
:106510000134082C07F11807E5D105B0BDE8F08F6C
:10652000002386F8C0302AE705F5947349F8230064
:106530008BE7182303FB05630020DA88A8F8042002
:10654000DA88012392B2FBF717FD82E74FF0010AC8
:106550009EE75A8A40F08001012392B20020FBF7A7
:106560000BFDB7E75572D3E700700240007102409F
:10657000382F0120FCFB1F000004000110B502446D
:10658000904201D1002010BD10F8014B11F8013BE1
:106590009C4202D3F4D90120F5E74FF0FF30F2E737
:1065A0002DE9F84F80460D46F1F758F8134B5C691A
:1065B00007460CB920461EE0E36804F1100B0BEB14
:1065C00083095E464E45B24601D32468F1E756F88A
:1065D000040B0378BB42F5D14378AB42F2D12A4693
:1065E00041460230FFF7CAFF0028EBD16068AAEBF2
:1065F0000B0A00EBAA00BDE8F88F00BFD04E0120C7
:10660000884237B504460D4608D1F2F7EFF828B9AD
:10661000A10766D12268374B9A4262D1364B9C4221
:1066200002D1002003B030BD9D42FAD0E20704D56C
:10663000EB07F6D423462C461D46304B2F4A234009
:10664000062B02EA050205D0A00733D120682C49A9
:1066500088422FD1062A46D0A907E2D128682849C6
:106660008842DED1062B05D1E008F0F7E9FF01787A
:106670006B6806E0062A6168FAD1E808F0F7E0FFE7
:10668000037811B10BB19942CBD169462046F2F79C
:10669000FFFA01A904462846F2F7FAFADDE90023D9
:1066A0009A420146BDD12046FFF768FFB0FA80F05C
:1066B0004009B7E7062AB4D0AB0703D12A68104BCC
:1066C0009A42AED02046F2F7A7F88369002BA8D0F3
:1066D0002A462146022098470028A2D0094CA04211
:1066E00004E001209EE7062BC4D1AC4214BF002079
:1066F000012097E738070700A8E10600070080FFA0
:10670000040E0700ACE10600F8B51746044600EB9E
:1067100081060025B44203D1680040F00100F8BDB5
:1067200054F8040B3946FFF76BFF0028F2D001350F
:10673000F0E7000007B501910549F2F724FCD0E924
:106740000210019A03B05DF804EBFFF7DDBF00BF54
:10675000BC0A07000A46083050F8041CFFF7D4BFF3
:10676000022838B50D46144613D1930701D00A48C4
:1067700038BD1268094B9A42F9D1A168A868FFF7A1
:106780003FFF0028F3D022792B799A42EFD10448B9
:10679000EEE70020ECE700BFA0E106003CA8060001
:1067A000ACE106002DE9F0479942DDF820A08046D3
:1067B00091461E4613D3BAF1010FA1EB030416BF95
:1067C00025460025002408EB050732464946384691
:1067D000FFF7D4FE20B1A54201D05544F3E70027CE
:1067E0003846BDE8F08770B50446022C049E154675
:1067F000184610D1B24226D1024608461146AE4292
:10680000324628BF2A46FFF7B9FE022C0ED1B0FA55
:1068100080F0400970BD2CB1032C05D032462E46C5
:106820001546E9E70124EAE70424E8E700280ADB43
:106830000BD1AE4203D02CBF01200020EAE7601E3E
:1068400018BF0120E6E70020E4E70120E2E72DE998
:10685000F74F9DF8306007468A46904699460024D7
:106860004C4502D386F0010619E018F804B0013453
:10687000002508EB0401554501D35C44F0E77B5D3E
:106880000135002BF9D09B450DD85A467819019354
:106890000091FFF773FEDDE9001320B92EB13046F9
:1068A00003B0BDE8F08F002EF9D01D44E3E70000EF
:1068B0002DE9F04F03881B2B89B005460C460ED1FD
:1068C000057A012D4FF0000006D1486081F8215073
:1068D0003548F2F7E9FD284609B0BDE8F08F1D2BD9
:1068E00060D1F8F711FC04F1080602460B46CDE929
:1068F0000623A98CA3892F7A95F80A80ADF8161083
:106900003046039395F91BA0D5F82090F3F781FD4D
:10691000039B1331181A814207F0010B4FEA580804
:10692000C7F3C00734DAE3699A4531DBA36943B1A1
:1069300001220092BDF8161062694846FFF787FFF2
:1069400030B359460FB14BF002013046F3F74FFD1B
:10695000082206A93046F3F7F8FD5FFA8AF13046BF
:10696000F3F745FD062205F10B013046F3F7EDFD87
:1069700041463046F3F73BFD02220DF11601304649
:10698000F3F7E3FD9DF8162049463046F3F7DDFDA9
:1069900061680020F3F7B6FC012308B184F82130C8
:1069A000184699E7002097E7B168030003460020E6
:1069B0001A5C02B970470130FAE700002DE9F04F88
:1069C000814689B0144600260B461D4613F8012B5C
:1069D00082B9A94211D30B78002B00F03A81013122
:1069E00020234FF000080A4612F8015B7DB94FF0F2
:1069F0000A0C2AE0252AE8D1EBE76F1AD9F804300F
:106A0000D9F800003A4698473E442946E3E72D2D41
:106A100003D148F001081146E5E72B2D02D148F0DB
:106A20000208F8E7202D02D148F00408F3E7212DF1
:106A300002D148F00808EEE7302D21D148F0400897
:106A40002B46E8E70CFB0525303D0F4611F8012BDE
:106A5000A2F130000928F5D92E2A41D17A782A2AC4
:106A600010D000204FF00A0C0F4611F801BBABF11B
:106A70003002092A09D80CFB00BBABF13000F3E768
:106A80000025B4E754F8040B023720EAE07B3A789B
:106A90006C2A08BF013797F800A0BAF1000F00F088
:106AA000D880BAF1780F6AD8BAF1570F1BD8BAF16B
:106AB000470F61D8BAF1440F61D9073424F00704B5
:106AC000F4E802010593F0F76DFCCDE9005B00EE00
:106AD000100A059B424651464846F8F7A0FC62E082
:106AE0004FF0FF3BD3E7AAF15802202A47D801A173
:106AF00051F822F0316C03007F6B03007F6B0300C1
:106B00007F6B03007F6B03007F6B03007F6B0300D1
:106B10007F6B03007F6B03007F6B0300916B0300AF
:106B2000B36B0300156C0300BB6A0300BB6A030070
:106B3000BB6A03007F6B03007F6B03007F6B030066
:106B40007F6B03007F6B03007F6B03007F6B030091
:106B50007F6B0300476C0300C76B03007F6B030070
:106B6000EB6B03007F6B0300036C03007F6B030080
:106B70007F6B0300316C0300BAF1500F63D0D9F87A
:106B80000430D9F8000001223946984701360BE05D
:106B900054F8042BCDE9003543463AB12F4904227D
:106BA0004846F0F77FFD0644791C0DE72C49052285
:106BB000F6E754F8042B8DF81C20CDE900350122AE
:106BC000434607A9ECE707A954F8040B0593F0F72F
:106BD0005AFDBBF1FF3F059B014601D1DDF81CB01A
:106BE000CDE900355A464346DAE7BBF1FF3F54F89A
:106BF000041BF5D108460593FFF7D8FE059B834695
:106C0000EEE7CDE9023561230093CDF804800A2335
:106C1000002207E0CDE9023561230093CDF804801E
:106C20000A23012254F8041B4846F0F799FDBAE7FD
:106C3000AAF1170ACDE90235CDF804805FFA8AF38C
:106C400000931023E4E7CDE90235CDF804806123F9
:106C5000F6E7304609B0BDE8F08F00BF5257060096
:106C6000575706000EB403B503AA52F8041B01924D
:106C7000FFF7A4FE02B05DF804EB03B0704700001C
:106C800013B5044608460191FAF760FC019B0449DC
:106C90000246204602B0BDE81040FFF7E3BF00BF48
:106CA0005D57060010B504468868FAF74FFC0246A7
:106CB0000B4620460249BDE81040FFF7D3BF00BF96
:106CC000735706004A680149FFF7CCBFFD5706001D
:106CD00030B4064B0D68064C0A4606498D420CBF7F
:106CE0002146194630BCFFF7BDBF00BFA4570600C0
:106CF00091570600400E0700CA880149FFF7B2BF4E
:106D0000B65706000A460149FFF7ACBFC357060055
:106D10004A680149FFF7A6BFCB57060013B50446E2
:106D200008460191F1F7AFFD019B04490246204658
:106D300002B0BDE81040FFF795BF00BFDA5706006C
:106D40004A680149FFF78EBFE557060007B5094BB2
:106D50008B4214BFD221A32140F22B130191009347
:106D6000054940F2551340F2A912FFF77BFF03B02B
:106D70005DF804FBC8B50600F457060007B5074BDD
:106D80008B4214BFB221D62100918623044940F2E0
:106D9000F512FFF767FF03B05DF804FB18BF0600AC
:106DA000F757060007B5084A40F225138A4214BF78
:106DB0001946D42100918823044940F2F512FFF7C7
:106DC00051FF03B05DF804FB78BF0600F7570600DB
:106DD00007B5084B8B4214BF4FF4AB718221009171
:106DE00040F23113044940F2F512FFF73BFF03B0C4
:106DF0005DF804FBFCBF0600F757060010B586B02F
:106E0000044603AB084604AA05A9F4F76DF8039BF2
:106E10000093054940F2F52340F2BB222046FFF7DC
:106E200021FF06B010BD00BFF75706000B4B99427B
:106E300007B50FD00A4B994214BFCC2172210091A3
:106E400040F23D13074940F2BB22FFF70BFF03B0AE
:106E50005DF804FB4FF4A071F1E700BF7CDD060094
:106E60004CDD0600F75706001FB50C46114602AA76
:106E70000092094A0192CDE902041A466846FFF7DA
:106E80009DFD24B1DDE902321AB903F8012C04B0EA
:106E900010BD00221A70FAE7391603000CB407B5CA
:106EA00004AB53F8042B0193FFF7DEFF03B05DF84A
:106EB00004EB02B0704700000FB407B504AA054800
:106EC00052F8041B0192FFF779FD03B05DF804EB63
:106ED00004B07047E8EB060038B505460846FFF7F2
:106EE00065FD044618B102466B682868984720463D
:106EF00038BD00002DE9F0478CB0044600AF0846CD
:106F00000E46F2F729F850B32A4B1B6823B11B68D1
:106F10001A68294B9A4222D107F10802391D3046DE
:106F2000F1F786FD7B68D3B1E8468AB0694623480D
:106F3000DFF89490F2F7EEF907F118012048F2F724
:106F4000E9F907F10C011F48F2F7E4F96946204618
:106F5000FFF7C2FF7D68033D002D0DDAC546022212
:106F60003146204608F0EAF917492046FFF7B4FFFA
:106F70003037BD46BDE8F087BA6802EB850307F1FC
:106F800018015B6852F825202046FFF76BFEBB68AE
:106F90004FEA850A53449A682AB949462046FFF7C2
:106FA0009BFF033DD8E707F10C012046FFF75AFE8F
:106FB000F7E700BF8C510120EF29780194470700C3
:106FC000FA5E0700B63B07006D62060010B594B08C
:106FD000044602A80191F0F73DFA38B9019920461C
:106FE00002F0B2FEF0F72EFA14B010BD0248039979
:106FF000FFF780FF0020F7E7E8EB06002DE9F04FF0
:107000006A4ED6F80431D6F8F08085B0002B6AD0ED
:1070100000254FEA88024046C6F80451002A50D0A5
:107020000024D6F8EC70A10804F00303795C5B003F
:1070300041FA03F303F00303032B32D001349442EB
:10704000EFD3D6F80431002BE6D18046D2B34FF00F
:10705000000E75464FF003094FF0020B04E0012BC0
:107060004FD0013595422DD2D6F8EC10AF0805F07F
:107070000304C85D640040FA04F303F00303022B29
:1070800001EB950C32D0032BE9D10BFA04F420EA82
:107090000400C855D6F8F0804FF0000E4FEA880281
:1070A000DFE72046F0F7EEF9D6F8F0000134B4EB54
:1070B000800F4FEA8002B4D3D6F80431002BABD155
:1070C000C3E78046202200213948FEF7F3FBB6F8DB
:1070D000082208F1FF33013AC6F82C32A6F808223C
:1070E00005B0BDE8F08F4FEA8802AFE7BEF1000FB0
:1070F000B7D009FA04F420EA0400C855D6F8F080A5
:10710000CCE7D6F8F4104FEAD50A05F0070811F8D5
:107110000A3043FA08F2D20701EBD50128D5D6F898
:10712000F8002A01825800EB05100090AAB1002354
:107130000022CDE90223F1F76FFBC369019013B37D
:10714000009802AA0C219847029810B10399FFF702
:107150003DFFD6F8F41051440B78012202FA08F8EA
:1071600023EA08030B70D6F8EC30D85D03EB070C6C
:1071700009FA04F420EA04008CF80000D6F8F08044
:107180004FF0010E8AE7019A906B0028E4D01A466E
:107190000430662111F010FF0028D5D0426802AB00
:1071A000DDE900010AF02CFCCEE700BFD04E012043
:1071B000DC50012030B58BB0FAF70EF86846EFF7D7
:1071C0001FFF164C054604211548F9F7D1FF236C23
:1071D0002BB1144A934214D1E06CFAF75DF81248CF
:1071E0000A21F9F7C5FF1148AA21F9F7C1FF104993
:1071F000491B89082846F9F7BBFFFFF7FFFE0BB0D4
:1072000030BD0C4A9342EAD1E06CFAF745F8D4F865
:10721000B400FAF741F8D4F8BC00DEE7D849012001
:10722000A84F0120A8C20600BC2101201047012060
:107230000000042094C306002DE9F04F0F3087B002
:1072400005090591029200F09080B44BD3F8F82024
:10725000002A00F00281B149B1F80832002B40F059
:107260008480D1F8003191F80AE29B1A029A48BF53
:107270000F33002A14BF032100214FEA231314BF48
:107280004FF0FF384FF001080193082D4FEA4103FA
:107290002A46039328BF0822A04B0091813203EBBA
:1072A00082038EF0010E0493049BD3F80490029B9A
:1072B000002B5FD1994BD3F82CA24E46974BD3F8B5
:1072C000ECB000220324B14549D8564547D8B8F15F
:1072D000FF3F1BF806104FEA860052D0B8F1010FAD
:1072E00079D0009BBEF1000F00F08D805C0003237D
:1072F000A3401940002942D101329542FCD8009B9D
:1073000003440299002940F0AB805C1C072DA4EBDC
:10731000020422D8814F05EB030107EB85064FEAF3
:1073200091013046C6F80812C6F80C1215D0062D89
:10733000C0F8101211D0052DC0F814120DD0042D74
:10734000C0F8181209D0032DC0F81C1205D0012D69
:10735000C0F8201201D1C7F828121D4688E09542D6
:1073600040F2D980BEF1000F18D00023184607B0B4
:10737000BDE8F08F694BD3F82C62B2469EE700223D
:10738000B8E70323BEF1000F0DD15F0004FA07F741
:107390000F4213D0019F1A18BA425BD2FFF70AFFBF
:1073A0004FF0010E80E75F0004FA07F70F420DD09F
:1073B000013B00225F1CF6D1464484E70132AA4219
:1073C0009ED2013B5F1CE0D146447CE701329542EE
:1073D00096D9013BEEE7BEF1000F2AD1734607E0D4
:1073E000019F1A189742D9D901330022042BE3D008
:1073F0005F0004FA07F70F42F2D1013295427FF69F
:107400007FAF0133F2E7DDF80CC004FA0CF70F424E
:107410000AD00133042B4FF00002CDD04FEA430CC9
:1074200004FA0CF70F42F4D1013295427FF668AFAF
:10743000EBE7002303E001330022042BBCD05F0004
:1074400004FA07F70F42F6D1013295427FF658AFA2
:107450000133F2E7013B0022B4E70820F7F78CFD87
:107460002E48591E8908D518C0F82C12013D1C461B
:10747000A00804F0030359001BF8006001238B40AF
:10748000611C33438D420BF8003011D30227234B8C
:107490008808D3F8EC6001F0030316F800C05B0025
:1074A00007FA03F3013143EA0C038D423354EED261
:1074B0001A4B0299D3F8F850260105EB041331B1A9
:1074C0001648D0F80011994288BFC0F8003113F077
:1074D00003014FEA021219D000211AB11846FEF733
:1074E000E9F90346059A002A3FF440AF0022AA5169
:1074F0000A4AE108D2F8F40004F00704455C0122CE
:1075000002FA04F444EA050242542FE79008002AE4
:10751000E8D08200E2E74FF0FF33F2E6D04E0120E0
:107520000A460021FFF788BE2DE9F34100240E46EC
:107530000746194630464FF6FF73904600942246A0
:1075400003F04AFC21461020FFF7EAFF0F4DA0424E
:1075500018BF05462F60AC602EB90D4CEC60284674
:1075600002B0BDE8F081B71CBF0021463846FFF7E6
:10757000D7FF04460028F0D0064BA7F10802C0E967
:10758000003641460830FAF719F8E7E7E84E0120DF
:1075900098E10600B80E07002DE9F04F0D4687B0C0
:1075A000002100AF064610209046FFF7B9FFB5F85E
:1075B00000A00AF1010A044600215046FFF7B0FF7F
:1075C0004CB92346224621463046FFF7ADFF1C3713
:1075D000BD46BDE8F08F07F1080968B9C4E90200AB
:1075E000184B2360D4E90210F0F738F800236060EC
:1075F0004A46BC600121E7E701233B72124B7B60E6
:107600002B88C7F80CA00733EB46DB08ABEBC303B2
:107610009D464FF0000A6946C7E904A02846C7F80E
:107620000090F1F777FE424669463846FFF7C6F903
:10763000D7E9043202F803A03B69A3607B69E360E9
:10764000DD46CDE7040E0700016805000EB403B562
:1076500003AA52F8041B0192FFF79EFF02B05DF8E7
:1076600004EB03B0704708B519B9F1F7DCF9F7F787
:107670000FFEFFF7EBFFFAE7014608B50148FFF7F9
:10768000F2FF00BF60FD0600136870B593B904688F
:10769000E56B4034AB4200D170BD54F8046BB1428D
:1076A00001D00133F6E7591CF6D0023350F82330ED
:1076B0001360F1E70148FFF7DFFF00BFD253070077
:1076C00007B5436802461B7900936846F2F710FA43
:1076D000536801461B79019301A8F2F709FA019B4F
:1076E00003F5E07350F82330DA0702D50948FFF7B5
:1076F000C3FF009B03F5E07351F82300C0F3810042
:10770000012805D0C31E5842584103B05DF804FB60
:107710000220FAE74E4F070008B50148FFF7ACFF1B
:107720005E5C0700014608B50148FFF79CFF00BFFB
:10773000D401070007B5064A1368526801A95B1A0D
:107740009A4202D80348FFF7EDFF03B05DF804FB4F
:10775000D04E0120C64607002DE9F74FDDF83080F6
:1077600004460D4617469B46FFF7E4FF4FF002091B
:107770004FF0010A20784F2803D87B68AB4240F2D3
:10778000A880512804F1010600F0A5800ED8052834
:1077900007D848B1831E032B23D8DFE803F027293D
:1077A0002945502800F091803446E3E7622868D0EC
:1077B00011D8602860D06128F6D1A61C5B46647899
:1077C000CDF800803A4629463046FFF7C5FF30B96C
:1077D00046FA84F6E8E77E2861D07F28E4D10120CC
:1077E00047E02A7863789A4273D1A61C0135DBE71B
:1077F000637804341A461AB9033818BF01200BE025
:10780000297814F802CC8C450BD814F801CC8C459F
:1078100007D3C21E5042504158B319FB03A31E4464
:10782000E4E70234013AE6E7637843F02001642993
:107830004FEA5312C3F340102B7806D1303B092B8B
:1078400015D9D04300F0010011E0732904D1202B99
:107850000DD0093B042BF3E723F02001413919290E
:1078600005D9A3F13001092901D95F2BE9D10028FD
:10787000BBD103B0BDE8F08F94F901600236264415
:1078800092E794F90100CDF80080A61C5B463A46C9
:1078900029463044FFF760FF0028A0D184E7A61CEA
:1078A0006478444580DA24B2CDF800805BF82490F7
:1078B0004BF824505B463A4629463046FFF74CFFCA
:1078C00000288CD14BF82490D3E73B68AB423FF4BF
:1078D0006BAF0020CDE77B68F8E7000008B50148F2
:1078E000FFF720FF0E56070070B505460C468E18B0
:1078F000B44200D170BDD5E900039847431C01D1C3
:10790000FFF7ECFF04F8010BF2E738B50446002559
:10791000D4E900039847421C01D1FFF7DFFF00F0D4
:107920007F0343EAC5150306F2D4284638BD00009C
:1079300008B50148FFF7F6FEDA56070008B501481A
:10794000FFF7F0FE3057070008B50148FFF7EAFEE1
:107950007E4A070008B5037A0BB9FFF7F5FF08BDAB
:1079600008B5037A0BB9FFF7EFFF08BD08B5037F31
:107970000BB9FFF7E9FF08BD08B50148FFF7D2FED4
:10798000784D070008B50148FFF7CCFE3A400700E4
:1079900008B5F7F7B3FF08B9FFF7F4FF004808BDD3
:1079A000A8E1060008B5F7F701FF08B9FFF7EAFFFD
:1079B000004808BDA8E1060008B50148FFF7B2FE7F
:1079C000DC460700014608B50148FFF74CFE00BF42
:1079D00004FF0600014608B50148FFF744FE00BF5A
:1079E0007803070008B50148FFF7F4FF8A4C070049
:1079F00070B5054608466E680EB9FFF7F3FF746868
:107A0000A9688C420DD9641AB368944228BF144601
:107A100019442246F9F7D2FDAB682344AB602046F7
:107A200070BD0024FBE70000402808B567D00DD8E2
:107A300000F0FD003C2809D1782907D8612908D831
:107A4000422968D04839CBB2092B3CD96248FFF7AC
:107A5000C1FF62391629F9D801A353F821F000BFFC
:107A6000177B03004D7A0300F97A03004D7A030077
:107A7000BD7A03004D7A0300CF7B0300BD7A03007B
:107A80004D7A03004D7A0300BD7A03004D7A03005E
:107A90004D7A03004D7A03004D7A0300F97A030012
:107AA0004D7A03004D7A03004D7A03004D7A0300AE
:107AB0004D7A03004D7A0300177B03000121042057
:107AC00002B1116008BD0929C0D801A353F821F003
:107AD000CF7B0300BD7A03004D7A03004D7A03008B
:107AE000BD7A03004D7A03004D7A03004D7A0300FE
:107AF0004D7A0300F97A030001210820E0E7782994
:107B0000A4D8612909D85129A0D847293CD80129EE
:107B100059D042299AD1012155E06239162995D8C8
:107B200001A353F821F000BF177B03004D7A030037
:107B3000CB7B03004D7A0300857B03004D7A030065
:107B4000D57B0300857B03004D7A03004D7A03004B
:107B5000857B03004D7A03004D7A03004D7A0300C4
:107B60004D7A0300CB7B03004D7A03004D7A03006E
:107B70004D7A03004D7A03004D7A03004D7A0300DD
:107B8000177B030004219AE7483909293FF65EAFC5
:107B900001A353F821F000BFD57B0300C57B030090
:107BA0004D7A03004D7A0300C57B03004D7A030034
:107BB0004D7A03004D7A03004D7A0300C17B030028
:107BC00008219AE7042108467AE70821FBE701210A
:107BD000022075E70221F6E7E64D070070B50D4675
:107BE0000179044601F07F01164640200022FFF78C
:107BF0001BFFE2682A60A36843436B60237903F0AC
:107C00007F03AB602168094B99420BD194F9043092
:107C1000002B01DBB30707D46368C3F3172300FB12
:107C200003202860002070BD0120FCE7340B070012
:107C300008B50369002219794020FFF7F5FE4000DE
:107C400040F0010008BD000008B50148FFF7C2FE82
:107C5000605B070008B50148FFF7BCFEBE440700A3
:107C600008B50148FFF7B6FE963B070008B5014886
:107C7000FFF7B0FEFE4C070008B50148FFF7AAFE6B
:107C80007E54070008B50148FFF7A4FE1065070001
:107C900008B50148FFF79EFE0E50070008B50148E1
:107CA000FFF798FEAE48070008B50E4B98424FF01C
:107CB000804314D00C4A904209D00C4A904202D022
:107CC0000B48FFF787FE5722C3F81C2505E000226A
:107CD000C3F81C25074B084A1A60084808BD002253
:107CE000F2E700BF78DD06007CDD06004CDD060013
:107CF00010540700B0510120AF0900ADA8E1060003
:107D000008B50148FFF766FE5C3F070008B5436809
:107D10000BB9FFF7F5FF08BD13B50446FFF7F6FFF3
:107D20000DF10700F2F72AFB04F10C00F2F771FBEA
:107D300004469DF80700F2F77DFB600040F001006B
:107D400002B010BD13B50446FFF7E0FF0DF10700C8
:107D5000F2F714FB00239DF807006382A382F2F779
:107D600069FB014802B010BDA8E1060008B54368F0
:107D70000BB9FFF7C5FF08BD10B50446FFF7F6FFC6
:107D80002046F7F7D3FD034A034B002814BF1046E3
:107D9000184610BD18BF0600F4BE060010B5044614
:107DA000FFF7E4FF2046F7F719FF034A034B0028CB
:107DB00014BF1046184610BDACE10600A0E1060055
:107DC00038B50D460446FFF7D1FF0A4B9D4205D159
:107DD00000212046F6F71EFA074838BD074B9D42A2
:107DE00005D1002211462046F7F78FFCF4E704483E
:107DF000FFF7F0FDF4BE0600A8E1060018BF06007C
:107E0000E244070038B504460D46FFF7AFFF2046B1
:107E1000F7F78CFD10B90648FFF72EFC2846F8F757
:107E20009DFD01462046F7F769FC024838BD00BFBA
:107E30008C600700A8E1060013B50446FFF796FF23
:107E40002046F7F773FD08B9FFF766FC636801A8E1
:107E50001B790193F1F74CFE019B074A03F5E07390
:107E600050F823300548C3F30223063B012B98BF8B
:107E7000104602B010BD00BF78BF06007CBF0600F0
:107E800038B504460D46FFF771FF2046F7F74EFD63
:107E900008B9FFF741FC04496B1A59422046594181
:107EA000F7F7C4FB014838BD78BF0600A8E106001B
:107EB00010B50446FFF75AFF2046F7F737FD0128B3
:107EC00002D10848FFF7D8FB2046FFF7F9FB01284D
:107ED00006D0054B054A022814BF1846104610BDAF
:107EE0000348FCE7D03B0700A8E10600FCBF060002
:107EF0005CC0060038B505460C46FFF737FF28463C
:107F0000F7F714FD012802D10C48FFF7B5FB0C4B25
:107F10009C4208D00B4B9C420BD00B4B9C420AD08E
:107F20000A48FFF757FD01212846F6F768F9064889
:107F300038BD0221F8E70021F6E700BFD03B07007B
:107F40005CC00600FCBF0600A8E106007046070002
:107F500010B586B00446FFF709FF334B9A88ADF899
:107F600014201868314A9B798DF816300323049049
:107F70000121C2F8F0350023C2F8F435C2F800152B
:107F800019461A0102F1804202F5E0420133082B42
:107F9000C2F81415C2F81015F3D104A8F5F7EEFFD6
:107FA00063685A79214BC3F81425C3F810250DF1E5
:107FB0000202C3F82C260122C3F830261A6003F50A
:107FC00080731A68002AFCD000221A601B68019393
:107FD000019B174B01221A6003F580731A68002A6F
:107FE000FCD000221A601B680293029B114B0122F5
:107FF0001A60114A1368002BFCD00023136012682A
:108000000392039A094AC2F80035BDF902209A4248
:10801000B8BFADF80230BDF80200800080B2400069
:1080200040F0010006B010BD185706000070004077
:1080300004700040087000401471004008B5FFF75C
:1080400095FE014808BD00BF3233D3C008B590F893
:108050002330FF2B01D1FFF753FE08BD10B50446B6
:10806000FFF7F4FF054B064801225A6094F82630CA
:1080700043F0040384F8263010BD00BF00500240D6
:10808000A8E1060010B50446FFF7E0FF0A4BD3F85D
:10809000082142B194F826206FF3410284F826208B
:1080A0000022C3F8082194F82630044813F0020F88
:1080B000034B08BF184610BD00500240ACE106005B
:1080C000A0E1060010B50446FFF7C0FF94F8263083
:1080D000034813F0080F034B08BF184610BD00BF3C
:1080E000ACE10600A0E1060010B50446FFF7AEFFC4
:1080F00094F8263003481A0744BF6FF3C30384F88B
:10810000263010BDA8E1060010B50446FFF79EFF1B
:108110000C4BD3F8082142B194F826206FF34102AA
:1081200084F826200022C3F8082194F826309A0704
:1081300001D4FFF703FC43F00803034884F826301A
:1081400010BD00BF00500240A8E1060008B543681A
:108150000BB9FFF7D5FD08BD10B50446FFF7F6FFD4
:10816000A06A400040F0010010BD10B50446FFF7C2
:10817000EDFFA07E400040F0010010BD10B50446A8
:10818000FFF7E4FF94F82400400040F0010010BD28
:1081900008B543680BB9FFF7B3FD08BD10B5044639
:1081A0002C34FFF7F5FF14F8082C0023D9B29142C4
:1081B00001D3054810BD54F8041B89680133002918
:1081C000F4D00248F6E700BFA0E10600ACE10600EB
:1081D00010B50446FFF7DCFFA06A10BD10B50446D9
:1081E000FFF7D6FF6069400040F0010010BD08B500
:1081F00043690BB9FFF784FD08BD10B50446FFF7CE
:10820000F6FFA06A10BD10B50446FFF7F0FF606AE4
:10821000400040F0010010BD08B5FFF7E8FF212045
:1082200008BD10B50446FFF7E2FF94F82D004000AA
:1082300040F0010010BD000010B50446FFF7D7FF65
:1082400094F82C00236A9FED127A04EB80045908FD
:10825000626923F001031344934210D1F1EEC76A1F
:1082600007EE901AF8EEE77AC6EEA77A17EE900AB4
:1082700020F0030040F00200A0F1FF4010BD32F9F1
:10828000020B07EE900AF8EEE77AA7EEA77AE3E78B
:108290000000000008B583680BB9FFF731FD08BD89
:1082A00010B50446FFF7F6FF2046F8F7FDFA01483F
:1082B00010BD00BFA8E1060010B50446FFF7EAFFB5
:1082C0002046F2F751FA034A034B002814BF104628
:1082D000184610BDACE10600A0E1060010B504464A
:1082E000FFF7D8FF94F82000034A044B002814BF7E
:1082F0001046184610BD00BFACE10600A0E1060024
:1083000010B50446FFF7C6FF94F820307BB1A36890
:108310000421002284F82020C3F80012A368D3F8B7
:10832000041121B1C3F80421A36801229A60014815
:1083300010BD00BFA8E1060010B50446FFF7AAFF74
:108340002046F2F711FA08B9FFF7F8FA012384F88A
:108350002030A36802480222C3F8002210BD00BFEB
:10836000A8E1060008B583680BB9FFF7C9FC08BD92
:1083700010B50446FFF7F6FFF2F7B8FA237F1BB1FA
:10838000F6F792FE034810BD01232377F6F78CFE23
:108390000148F8E7A0E10600ACE1060010B504468C
:1083A000FFF7E0FF00230148237710BDA8E1060096
:1083B00008B583680BB9FFF7A3FC08BD10B50446E8
:1083C000FFF7F6FF2046F7F760FC034A034B00284F
:1083D00014BF1046184610BDACE10600A0E106002F
:1083E00010B50446FFF7E4FF2046F7F72FFC034AD9
:1083F000034B002814BF1046184610BDACE1060020
:10840000A0E1060038B50D460446FFF7D1FF284627
:10841000F8F7A4FA01462046F7F783F9004838BD7B
:10842000A8E1060008B583680BB9FFF769FC08BD31
:1084300010B50446FFF7F6FFF2F758FA94F820302B
:10844000DB0603D5F6F730FE054810BD94F8203062
:1084500043F0100384F82030F6F726FE0148F4E7D5
:10846000A0E10600ACE1060010B50446FFF7DAFF14
:1084700094F8203002486FF3041384F8203010BDC4
:10848000A8E1060008B5837AFF2B01D1FFF738FC7D
:1084900008BD000010B50446FFF7F4FF237A1BB9AE
:1084A00001230248237210BD0148FCE7ACE106003D
:1084B000A0E1060010B50446FFF7E4FF00230148E1
:1084C000237210BDA8E1060008B5C3680BB9FFF719
:1084D00017FC08BD10B50446FFF7F6FF201DF7F79F
:1084E000D4FB034A034B002814BF1046184610BDA6
:1084F000ACE10600A0E1060010B50446FFF7E4FF7A
:10850000201DF7F7A3FB034A034B002814BF1046B6
:10851000184610BDACE10600A0E1060038B50D46D6
:108520000446FFF7D1FF2846F8F718FA0146201D48
:10853000F7F7F7F8004838BDA8E1060008B5437A18
:10854000FF2B01D1FFF7DCFB08BD000010B504468E
:10855000FFF7F4FF00230148237210BDA8E10600D5
:1085600010B50446FFF7EAFF63681B68D3F82435AB
:10857000B3F1805F23D013D8B3F1006F21D00BD8B3
:10858000B3F1007F1FD01348B3F1806F18BF0020F4
:10859000400040F0010010BD0F48B3F1206FF5E737
:1085A000B3F1804F11D006D8B3F1A05F0FD00B48C4
:1085B000B3F1005FEAE70A48B3F1004FE6E7094884
:1085C000E6E70948E4E70948E2E70948E0E709483F
:1085D000DEE700BF90D003000024F40080841E007A
:1085E00000127A0040420F0020A1070048E8010075
:1085F00000093D000048E80108B5837FFF2B01D149
:10860000FFF77EFB08BD10B50446FFF7F5FFA06835
:10861000400040F0010010BD10B50446FFF7ECFF2C
:1086200004F11000F1F7F5FE400040F0010010BD2C
:1086300010B50446FFF7E0FFD4ED037A9FED077A0B
:10864000F8EE677AC7EE877A17EE900A20F00300FB
:1086500040F00200A0F1FF4010BD00BF00007A44CE
:1086600010B50446FFF7C8FF6368186840F3073089
:10867000F1F71CFA0023E3822383636806481B6832
:10868000012143F30732C3F3043301FA03F3520920
:10869000024941F8223010BDA8E1060000E100E0E7
:1086A000F8B50F461E4605461446FFF7A5FF40F2F3
:1086B00001139F4216D114F0010006D005F11000FD
:1086C000F1F7A7FE003818BF0120630709D56B68D2
:1086D000074A1B79242101FB03235B690BB940F096
:1086E0000400F8BD162333604FF0FF30F9E700BFF8
:1086F000E84D012008B543680BB9FFF701FB08BD41
:1087000010B50446FFF7F6FF6089400040F0010015
:1087100010BD10B50446FFF7EDFFE068400040F0E3
:10872000010010BD08B50379FF2B01D1FFF7E8FA6E
:1087300008BD000010B50446FFF7F4FF2079F1F7FB
:1087400073FD01230148A37110BD00BFA8E106001D
:1087500010B50446FFF7E6FFA37913B92079F1F7C6
:1087600063FD0023E3812382A37913B92079F5F710
:1087700053FF014810BD00BFA8E1060038B504460C
:10878000FFF7D0FF238A9BB213B91248FFF71AF9FB
:10879000A37913B92079F1F747FDE389A268A1898C
:1087A0009BB232F81350E3899BB20133B3FBF1F271
:1087B00001FB12339BB2E381238A013B9BB22382EC
:1087C000A37913B92079F5F727FF680040F001007D
:1087D00038BD00BF7461070010B50446FFF7A2FF63
:1087E000A089400040F0010010BD000010B5044613
:1087F000FFF798FFA079034A034B002814BF1046E7
:10880000184610BDACE10600A0E1060038B50D46E3
:1088100004460846FFF786FF2B8A042C9BB203D040
:10882000052C07D0002038BD044A0548002B18BF8E
:108830001046F8E7580040F00100F4E7ACE106000C
:10884000A0E1060008B543680BB9FFF759FA08BD67
:1088500010B50446FFF7F6FF201DF7F7A7FA2189A8
:10886000034A044B814234BF1046184610BD00BF76
:10887000ACE10600A0E1060010B50446FFF7E2FFF8
:10888000201DF7F793FA400040F0010010BD10B52D
:108890000446FFF7D7FF2089400040F0010010BDDB
:1088A00008B503790BB9FFF72BFA47F6015008BD5D
:1088B00008B543680BB9FFF723FA0069400040F0A0
:1088C000010008BD222808B508D8431E1F2B09D86F
:1088D0001138012806D90448FFF77CF8312801D067
:1088E0004128F8D108BD00BF323B070070B50E46E5
:1088F000054617493046F0F746FB08350446D8B917
:1089000014493046F0F73FFB044610B91248FFF710
:1089100061F890F85030D90601D51048F7E723F0F8
:10892000140343F01403856280F85030F2F758FDC9
:10893000F2F799FD204670BD90F82E309A07ECD4DE
:1089400043F0020380F82E302946F2F703FEF1E7E8
:1089500034C5060058C906008C3F0700BC5E0700FE
:10896000F8B51646838D428D9A4204460D4602D1D3
:108970000E48FEF7D7FE3146FFF7B8FF628D074677
:10898000AA42636809D843F83570616801EBC501F4
:108990004E60638D01336385F8BD03EBC20313E9B9
:1089A0000300013A83E80300EAE700BFAC3B07009D
:1089B0007FB50446C08A984202D82948FFF70AF8D2
:1089C00094F85000050745D504F12405208B02FBDF
:1089D0000050435494F85030258BD807238CA1EBDA
:1089E000030191FBF5F305FB13110EB254BF04F123
:1089F0002C0001A8002EA38BBCBF6D182EB213FB58
:108A000006F39BB20380A18B0B448380638C618B44
:108A1000D21A92FBF1F301FB132215B2002DE38B66
:108A2000BCBF89180DB213FB05F39BB24380E28BE8
:108A30001344C38094F85030DB0704D501A904F136
:108A40002C00F2F7BFFD94F8503043F0010384F896
:108A5000503002E0656A002DB8D104B070BD00BF8F
:108A600044500700F8B50025C0E901250446C1605F
:108A70000582E3681A8BAFB2BA4215D84FF4803240
:108A80001A6293F8502042F0020283F85020F8BD99
:108A900000233946FFF78CFF0136E068438BB2B202
:108AA0009342F5D80135E4E70026F6E72DE9F047D3
:108AB000B0F80A8004460E460D468F184FF00009A4
:108AC000BD4202D3A81BBDE8F0872846EEF7AAFEF8
:108AD00001462846EEF7C3FE7F29054678D8A1F166
:108AE00020035E2B0BD86068F2F7B4FF034662895F
:108AF0002189E068FFF75CFF238901332CE00D2911
:108B00001ED1A4F80890E36821891A8B8A4208D8FC
